
 Start         Length     Name                   Class
 0001:00401000 0004CF70H .text                   CODE
 0002:0044E000 00000D94H .itext                  ICODE
 0003:0044F000 00001340H .data                   DATA
 0004:00451000 000051B8H .bss                    BSS
 0005:00000000 00000014H .tls                    TLS


Detailed map of segments

 0001:00000000 00008A75 C=CODE     S=.text    G=(none)   M=System   ACBP=A9
 0001:00008A78 0000010D C=CODE     S=.text    G=(none)   M=SysInit  ACBP=A9
 0001:00008B88 000008F5 C=CODE     S=.text    G=(none)   M=Windows  ACBP=A9
 0001:00009480 00000338 C=CODE     S=.text    G=(none)   M=SysConst ACBP=A9
 0001:000097B8 00000158 C=CODE     S=.text    G=(none)   M=RTLConsts ACBP=A9
 0001:00009910 000001D0 C=CODE     S=.text    G=(none)   M=Character ACBP=A9
 0001:00009AE0 00000131 C=CODE     S=.text    G=(none)   M=StrUtils ACBP=A9
 0001:00009C14 0000C99B C=CODE     S=.text    G=(none)   M=SysUtils ACBP=A9
 0001:000165B0 000007D3 C=CODE     S=.text    G=(none)   M=VarUtils ACBP=A9
 0001:00016D84 0000818C C=CODE     S=.text    G=(none)   M=Variants ACBP=A9
 0001:0001EF10 0000180B C=CODE     S=.text    G=(none)   M=TypInfo  ACBP=A9
 0001:0002071C 000173A0 C=CODE     S=.text    G=(none)   M=Classes  ACBP=A9
 0001:00037ABC 000008D3 C=CODE     S=.text    G=(none)   M=SyncObjs ACBP=A9
 0001:00038390 000000B3 C=CODE     S=.text    G=(none)   M=Rtti     ACBP=A9
 0001:00038444 0000BB90 C=CODE     S=.text    G=(none)   M=ceflib   ACBP=A9
 0001:00043FD4 000000FC C=CODE     S=.text    G=(none)   M=IOUtils  ACBP=A9
 0001:000440D0 0000007F C=CODE     S=.text    G=(none)   M=IniFiles ACBP=A9
 0001:00044150 000030A2 C=CODE     S=.text    G=(none)   M=Registry ACBP=A9
 0001:000471F4 0000062A C=CODE     S=.text    G=(none)   M=Contnrs  ACBP=A9
 0001:00047820 00001784 C=CODE     S=.text    G=(none)   M=ceffilescheme ACBP=A9
 0001:00048FA4 00003FCA C=CODE     S=.text    G=(none)   M=cefclient ACBP=A9
 0002:00000000 000000AA C=ICODE    S=.itext   G=(none)   M=System   ACBP=A9
 0002:000000AC 00000016 C=ICODE    S=.itext   G=(none)   M=Windows  ACBP=A9
 0002:000000C4 000000B4 C=ICODE    S=.itext   G=(none)   M=SysUtils ACBP=A9
 0002:00000178 0000000F C=ICODE    S=.itext   G=(none)   M=VarUtils ACBP=A9
 0002:00000188 000000AA C=ICODE    S=.itext   G=(none)   M=Variants ACBP=A9
 0002:00000234 00000008 C=ICODE    S=.itext   G=(none)   M=TypInfo  ACBP=A9
 0002:0000023C 0000009D C=ICODE    S=.itext   G=(none)   M=Classes  ACBP=A9
 0002:000002DC 0000000F C=ICODE    S=.itext   G=(none)   M=SyncObjs ACBP=A9
 0002:000002EC 0000004C C=ICODE    S=.itext   G=(none)   M=Rtti     ACBP=A9
 0002:00000338 00000012 C=ICODE    S=.itext   G=(none)   M=ceflib   ACBP=A9
 0002:0000034C 00000460 C=ICODE    S=.itext   G=(none)   M=IOUtils  ACBP=A9
 0002:000007AC 00000008 C=ICODE    S=.itext   G=(none)   M=IniFiles ACBP=A9
 0002:000007B4 00000008 C=ICODE    S=.itext   G=(none)   M=Registry ACBP=A9
 0002:000007BC 000005D8 C=ICODE    S=.itext   G=(none)   M=cefclient ACBP=A9
 0003:00000000 000009F0 C=DATA     S=.data    G=DGROUP   M=System   ACBP=A9
 0003:000009F0 00000024 C=DATA     S=.data    G=DGROUP   M=SysInit  ACBP=A9
 0003:00000A14 0000000C C=DATA     S=.data    G=DGROUP   M=Windows  ACBP=A9
 0003:00000A20 00000100 C=DATA     S=.data    G=DGROUP   M=Character ACBP=A9
 0003:00000B20 000002DC C=DATA     S=.data    G=DGROUP   M=SysUtils ACBP=A9
 0003:00000DFC 00000008 C=DATA     S=.data    G=DGROUP   M=VarUtils ACBP=A9
 0003:00000E04 00000152 C=DATA     S=.data    G=DGROUP   M=Variants ACBP=A9
 0003:00000F58 0000000C C=DATA     S=.data    G=DGROUP   M=TypInfo  ACBP=A9
 0003:00000F64 00000058 C=DATA     S=.data    G=DGROUP   M=Classes  ACBP=A9
 0003:00000FBC 00000008 C=DATA     S=.data    G=DGROUP   M=Rtti     ACBP=A9
 0003:00000FC4 00000028 C=DATA     S=.data    G=DGROUP   M=ceflib   ACBP=A9
 0003:00000FEC 00000010 C=DATA     S=.data    G=DGROUP   M=IOUtils  ACBP=A9
 0003:00000FFC 0000000C C=DATA     S=.data    G=DGROUP   M=IniFiles ACBP=A9
 0003:00001008 00000024 C=DATA     S=.data    G=DGROUP   M=Registry ACBP=A9
 0003:0000102C 00000030 C=DATA     S=.data    G=DGROUP   M=ceffilescheme ACBP=A9
 0003:0000105C 00000010 C=DATA     S=.data    G=DGROUP   M=cefclient ACBP=A9
 0004:00000000 00002C34 C=BSS      S=.bss     G=DGROUP   M=System   ACBP=A9
 0004:00002C34 0000000C C=BSS      S=.bss     G=DGROUP   M=SysInit  ACBP=A9
 0004:00002C40 00000008 C=BSS      S=.bss     G=DGROUP   M=Windows  ACBP=A9
 0004:00002C48 0000001C C=BSS      S=.bss     G=DGROUP   M=Character ACBP=A9
 0004:00002C64 00002240 C=BSS      S=.bss     G=DGROUP   M=SysUtils ACBP=A9
 0004:00004EA4 0000005C C=BSS      S=.bss     G=DGROUP   M=VarUtils ACBP=A9
 0004:00004F00 00000040 C=BSS      S=.bss     G=DGROUP   M=Variants ACBP=A9
 0004:00004F40 00000004 C=BSS      S=.bss     G=DGROUP   M=TypInfo  ACBP=A9
 0004:00004F44 00000048 C=BSS      S=.bss     G=DGROUP   M=Classes  ACBP=A9
 0004:00004F8C 00000014 C=BSS      S=.bss     G=DGROUP   M=SyncObjs ACBP=A9
 0004:00004FA0 00000010 C=BSS      S=.bss     G=DGROUP   M=Rtti     ACBP=A9
 0004:00004FB0 00000194 C=BSS      S=.bss     G=DGROUP   M=ceflib   ACBP=A9
 0004:00005144 00000024 C=BSS      S=.bss     G=DGROUP   M=IOUtils  ACBP=A9
 0004:00005168 00000004 C=BSS      S=.bss     G=DGROUP   M=IniFiles ACBP=A9
 0004:0000516C 00000004 C=BSS      S=.bss     G=DGROUP   M=Registry ACBP=A9
 0004:00005170 00000048 C=BSS      S=.bss     G=DGROUP   M=cefclient ACBP=A9
 0005:00000000 00000008 C=TLS      S=.tls     G=(none)   M=System   ACBP=A9
 0005:00000008 0000000C C=TLS      S=.tls     G=(none)   M=Classes  ACBP=A9


  Address             Publics by Name

 0001:00048FA4       cefclient..TCustomClient
 0001:00049264       cefclient..TCustomDisplay
 0001:0004910C       cefclient..TCustomLifeSpan
 0001:000491C0       cefclient..TCustomLoad
 0001:00049484       cefclient..TExtension
 0001:0004931C       cefclient..TScheme
 0004:00005174       cefclient.backWnd
 0003:00001060       cefclient.brows
 0003:00001064       cefclient.browsrHwnd
 0004:0000518D       cefclient.canGoBack
 0004:0000518E       cefclient.canGoForward
 0002:000007BC       cefclient.cefclient
 0001:0004958C       cefclient.CefWndProc
 0004:00005184       cefclient.editWnd
 0004:00005188       cefclient.editWndOldProc
 0001:0004A66C       cefclient.Finalization
 0004:00005178       cefclient.forwardWnd
 0003:0000105C       cefclient.handl
 0004:0000518C       cefclient.isLoading
 0003:00001068       cefclient.navigateto
 0004:0000517C       cefclient.reloadWnd
 0004:00005180       cefclient.stopWnd
 0001:00049B2C       cefclient.TCustomClient.Create
 0001:00049BB8       cefclient.TCustomClient.GetDisplayHandler
 0001:00049BCC       cefclient.TCustomClient.GetLifeSpanHandler
 0001:00049BE0       cefclient.TCustomClient.GetLoadHandler
 0001:00049C78       cefclient.TCustomDisplay.OnAddressChange
 0001:00049CB8       cefclient.TCustomDisplay.OnTitleChange
 0001:00049BF4       cefclient.TCustomLifeSpan.OnAfterCreated
 0001:00049C20       cefclient.TCustomLoad.OnLoadEnd
 0001:00049C44       cefclient.TCustomLoad.OnLoadStart
 0001:0004A348       cefclient.TExtension.Execute
 0001:00049CE4       cefclient.TScheme.Create
 0001:00049D3C       cefclient.TScheme.Destroy
 0001:0004A220       cefclient.TScheme.GetResponseHeaders
 0001:0004A2BC       cefclient.TScheme.Output
 0001:00049D6C       cefclient.TScheme.ProcessRequest
 0001:0004A294       cefclient.TScheme.ReadResponse
 0004:00005170       cefclient.Window
 0004:00005190       cefclient.wndClass
 0001:00047B04       ceffilescheme..TFileInfo
 0001:00047820       ceffilescheme..TFileScheme
 0001:00047A08       ceffilescheme.Escape
 0001:000481F8       ceffilescheme.FileSortCompare
 0001:00048240       ceffilescheme.HTTPDecode
 0001:00048658       ceffilescheme.OutPut
 0001:00048704       ceffilescheme.OutputUTF8
 0001:00048394       ceffilescheme.ParseFileUrl
 0003:0000102C       ceffilescheme.s
 0001:00047D14       ceffilescheme.TFileInfo.Create
 0001:000480C4       ceffilescheme.TFileInfo.Display
 0001:00048020       ceffilescheme.TFileInfo.DisplayDate
 0001:00047D80       ceffilescheme.TFileInfo.DisplaySize
 0001:00048598       ceffilescheme.TFileScheme.Cancel
 0001:000485A0       ceffilescheme.TFileScheme.Create
 0001:000485EC       ceffilescheme.TFileScheme.Destroy
 0001:00048620       ceffilescheme.TFileScheme.GetResponseHeaders
 0001:000487B0       ceffilescheme.TFileScheme.ProcessRequest
 0001:00048F7C       ceffilescheme.TFileScheme.ReadResponse
 0004:00004FB8       ceflib..85
 0001:0003C524       ceflib..ECefException
 0001:00038CF4       ceflib..TCefBaseOwn
 0001:00038EB0       ceflib..TCefBaseRef
 0001:00039268       ceflib..TCefBrowserRef
 0001:0003A86C       ceflib..TCefClientOwn
 0001:0003ACD4       ceflib..TCefCustomStreamReader
 0001:0003AB44       ceflib..TCefDisplayHandlerOwn
 0001:0003B988       ceflib..TCefDomDocumentRef
 0001:0003BED4       ceflib..TCefDomEventListenerOwn
 0001:0003BD88       ceflib..TCefDomEventRef
 0001:0003BBEC       ceflib..TCefDomNodeRef
 0001:0003B680       ceflib..TCefDomVisitorOwn
 0001:0003C160       ceflib..TCefFastDomEventListener
 0001:0003B758       ceflib..TCefFastDomVisitor
 0001:0003C3DC       ceflib..TCefFastV8Accessor
 0001:000394C4       ceflib..TCefFrameRef
 0001:0003A96C       ceflib..TCefLifeSpanHandlerOwn
 0001:0003AA60       ceflib..TCefLoadHandlerOwn
 0001:00039800       ceflib..TCefPostDataElementRef
 0001:00039638       ceflib..TCefPostDataRef
 0001:00039A10       ceflib..TCefRequestRef
 0001:0003C07C       ceflib..TCefResponseRef
 0001:0003B210       ceflib..TCefSchemeHandlerCallbackRef
 0001:0003B378       ceflib..TCefSchemeHandlerFactoryOwn
 0001:0003AF1C       ceflib..TCefSchemeHandlerOwn
 0001:00039BB0       ceflib..TCefStreamReaderRef
 0001:0003C300       ceflib..TCefV8AccessorOwn
 0001:0003A5B8       ceflib..TCefv8ContextRef
 0001:0003B53C       ceflib..TCefv8HandlerOwn
 0001:0003A784       ceflib..TCefv8HandlerRef
 0001:0003A064       ceflib..TCefv8ValueRef
 0001:0003CAA8       ceflib..TSHSyncGetResponseHeaders
 0001:0003C5F4       ceflib..TSHSyncProcessRequest
 0001:0003C83C       ceflib..TSHSyncReadResponse
 0001:0004183C       ceflib.CefBrowserCreate
 0003:00000FC8       ceflib.CefCache
 0003:00000FE4       ceflib.CefExtraPluginPaths
 0003:00000FE0       ceflib.CefGraphicsImplementation
 0002:00000338       ceflib.ceflib
 0003:00000FC4       ceflib.CefLibrary
 0001:0003FA34       ceflib.CefLoadLib
 0001:0003F9E8       ceflib.CefLoadLibDefault
 0003:00000FD4       ceflib.CefLocale
 0004:00004FB0       ceflib.CefLocalStorageQuota
 0003:00000FD8       ceflib.CefLogFile
 0003:00000FDC       ceflib.CefLogSeverity
 0003:00000FD0       ceflib.CefProductVersion
 0001:00041AFC       ceflib.CefRegisterCustomScheme
 0001:00041B44       ceflib.CefRegisterExtension
 0001:00041A38       ceflib.CefRegisterSchemeHandlerFactory
 0001:0004187C       ceflib.CefRunMessageLoop
 0004:00004FB4       ceflib.CefSessionStorageQuota
 0001:0004188C       ceflib.CefString
 0001:000418EC       ceflib.CefString
 0001:00041910       ceflib.CefStringAlloc
 0001:000419F0       ceflib.CefStringClearAndGet
 0001:00041A0C       ceflib.CefStringFreeAndGet
 0001:00041988       ceflib.CefStringSet
 0001:0003CD2C       ceflib.CefTimeToDateTime
 0001:0003CCB4       ceflib.CefTimeToSystemTime
 0003:00000FCC       ceflib.CefUserAgent
 0004:000050A8       ceflib.cef_add_cross_origin_whitelist_entry
 0001:0003CD9C       ceflib.cef_base_add_ref
 0001:0003CDCC       ceflib.cef_base_get_refct
 0001:0003CDB4       ceflib.cef_base_release
 0004:00005044       ceflib.cef_browser_create
 0004:00005048       ceflib.cef_browser_create_sync
 0004:000050B0       ceflib.cef_clear_cross_origin_whitelist
 0004:000050A4       ceflib.cef_clear_scheme_handler_factories
 0001:0003CF00       ceflib.cef_client_get_display_handler
 0001:0003D260       ceflib.cef_client_get_drag_handler
 0001:0003D0E0       ceflib.cef_client_get_find_handler
 0001:0003CF60       ceflib.cef_client_get_focus_handler
 0001:0003D1A0       ceflib.cef_client_get_jsbinding_handler
 0001:0003D140       ceflib.cef_client_get_jsdialog_handler
 0001:0003CFC0       ceflib.cef_client_get_keyboard_handler
 0001:0003CDE0       ceflib.cef_client_get_life_span_handler
 0001:0003CE40       ceflib.cef_client_get_load_handler
 0001:0003D020       ceflib.cef_client_get_menu_handler
 0001:0003D080       ceflib.cef_client_get_print_handler
 0001:0003D200       ceflib.cef_client_get_render_handler
 0001:0003CEA0       ceflib.cef_client_get_request_handler
 0004:000050C4       ceflib.cef_create_url
 0004:000050B4       ceflib.cef_currently_on
 0004:000050D4       ceflib.cef_delete_cookies
 0004:000050E0       ceflib.cef_delete_storage
 0001:0003D740       ceflib.cef_display_handler_on_address_change
 0001:0003D96C       ceflib.cef_display_handler_on_console_message
 0001:0003D6D4       ceflib.cef_display_handler_on_nav_state_change
 0001:0003D8F0       ceflib.cef_display_handler_on_status_message
 0001:0003D7D4       ceflib.cef_display_handler_on_title_change
 0001:0003D84C       ceflib.cef_display_handler_on_tooltip
 0001:0003E298       ceflib.cef_dom_event_listener_handle_event
 0001:0003E23C       ceflib.cef_dom_visitor_visite
 0004:0000504C       ceflib.cef_do_message_loop_work
 0004:00005054       ceflib.cef_initialize
 0001:0003D4B0       ceflib.cef_life_span_handler_do_close
 0001:0003D394       ceflib.cef_life_span_handler_on_after_created
 0001:0003D3F0       ceflib.cef_life_span_handler_on_before_close
 0001:0003D2C0       ceflib.cef_life_span_handler_on_before_popup
 0001:0003D44C       ceflib.cef_life_span_handler_run_modal
 0001:0003D590       ceflib.cef_load_handler_on_load_end
 0001:0003D610       ceflib.cef_load_handler_on_load_error
 0001:0003D514       ceflib.cef_load_handler_on_load_start
 0004:000050C0       ceflib.cef_parse_url
 0004:000050E8       ceflib.cef_post_data_create
 0004:000050EC       ceflib.cef_post_data_element_create
 0004:000050BC       ceflib.cef_post_delayed_task
 0004:000050B8       ceflib.cef_post_task
 0001:0003DA58       ceflib.cef_read_handler_eof
 0001:0003DA08       ceflib.cef_read_handler_read
 0001:0003DA28       ceflib.cef_read_handler_seek
 0001:0003DA44       ceflib.cef_read_handler_tell
 0004:0000509C       ceflib.cef_register_custom_scheme
 0004:00005098       ceflib.cef_register_extension
 0004:000050A0       ceflib.cef_register_scheme_handler_factory
 0004:000050AC       ceflib.cef_remove_cross_origin_whitelist_entry
 0004:000050E4       ceflib.cef_request_create
 0004:00005050       ceflib.cef_run_message_loop
 0001:0003DCB8       ceflib.cef_scheme_handler_cancel
 0001:0003DA78       ceflib.cef_scheme_handler_factory_create
 0001:0003DEC0       ceflib.cef_scheme_handler_get_response_headers
 0001:0003DE08       ceflib.cef_scheme_handler_get_response_headers_sync
 0001:0003DB2C       ceflib.cef_scheme_handler_process_request
 0001:0003DBCC       ceflib.cef_scheme_handler_process_request_sync
 0001:0003DCCC       ceflib.cef_scheme_handler_read_response
 0001:0003DD3C       ceflib.cef_scheme_handler_read_response_sync
 0004:000050D0       ceflib.cef_set_cookie
 0004:000050DC       ceflib.cef_set_storage
 0004:00005058       ceflib.cef_shutdown
 0004:000050F4       ceflib.cef_stream_reader_create_for_data
 0004:000050F0       ceflib.cef_stream_reader_create_for_file
 0004:000050F8       ceflib.cef_stream_reader_create_for_handler
 0004:000050FC       ceflib.cef_stream_writer_create_for_file
 0004:00005100       ceflib.cef_stream_writer_create_for_handler
 0004:0000501C       ceflib.cef_string_ascii_to_utf16
 0004:00005018       ceflib.cef_string_ascii_to_wide
 0004:00004FD8       ceflib.cef_string_clear
 0004:00005020       ceflib.cef_string_from_ascii
 0004:0000500C       ceflib.cef_string_from_utf16
 0004:00005004       ceflib.cef_string_from_utf8
 0004:00005014       ceflib.cef_string_from_wide
 0004:0000507C       ceflib.cef_string_list_alloc
 0004:00005088       ceflib.cef_string_list_append
 0004:0000508C       ceflib.cef_string_list_clear
 0004:00005094       ceflib.cef_string_list_copy
 0004:00005090       ceflib.cef_string_list_free
 0004:00005080       ceflib.cef_string_list_size
 0004:00005084       ceflib.cef_string_list_value
 0004:0000505C       ceflib.cef_string_map_alloc
 0004:00005070       ceflib.cef_string_map_append
 0004:00005074       ceflib.cef_string_map_clear
 0004:00005064       ceflib.cef_string_map_find
 0004:00005078       ceflib.cef_string_map_free
 0004:00005068       ceflib.cef_string_map_key
 0004:00005060       ceflib.cef_string_map_size
 0004:0000506C       ceflib.cef_string_map_value
 0004:00004FC8       ceflib.cef_string_set
 0004:00005008       ceflib.cef_string_to_utf16
 0004:00005000       ceflib.cef_string_to_utf8
 0004:00005010       ceflib.cef_string_to_wide
 0004:00005030       ceflib.cef_string_userfree_alloc
 0004:00005040       ceflib.cef_string_userfree_free
 0004:0000502C       ceflib.cef_string_userfree_utf16_alloc
 0004:0000503C       ceflib.cef_string_userfree_utf16_free
 0004:00005028       ceflib.cef_string_userfree_utf8_alloc
 0004:00005038       ceflib.cef_string_userfree_utf8_free
 0004:00005024       ceflib.cef_string_userfree_wide_alloc
 0004:00005034       ceflib.cef_string_userfree_wide_free
 0004:00004FD4       ceflib.cef_string_utf16_clear
 0004:00004FE4       ceflib.cef_string_utf16_cmp
 0001:0003CC98       ceflib.cef_string_utf16_copy
 0004:00004FC4       ceflib.cef_string_utf16_set
 0004:00004FFC       ceflib.cef_string_utf16_to_utf8
 0004:00004FF4       ceflib.cef_string_utf16_to_wide
 0004:00004FD0       ceflib.cef_string_utf8_clear
 0004:00004FE0       ceflib.cef_string_utf8_cmp
 0004:00004FC0       ceflib.cef_string_utf8_set
 0004:00004FF8       ceflib.cef_string_utf8_to_utf16
 0004:00004FEC       ceflib.cef_string_utf8_to_wide
 0004:00004FCC       ceflib.cef_string_wide_clear
 0004:00004FDC       ceflib.cef_string_wide_cmp
 0004:00004FBC       ceflib.cef_string_wide_set
 0004:00004FF0       ceflib.cef_string_wide_to_utf16
 0004:00004FE8       ceflib.cef_string_wide_to_utf8
 0004:00005104       ceflib.cef_v8context_get_current_context
 0004:00005108       ceflib.cef_v8context_get_entered_context
 0004:00005130       ceflib.cef_v8value_create_array
 0004:00005114       ceflib.cef_v8value_create_bool
 0004:00005120       ceflib.cef_v8value_create_date
 0004:0000511C       ceflib.cef_v8value_create_double
 0004:00005134       ceflib.cef_v8value_create_function
 0004:00005118       ceflib.cef_v8value_create_int
 0004:00005110       ceflib.cef_v8value_create_null
 0004:00005128       ceflib.cef_v8value_create_object
 0004:0000512C       ceflib.cef_v8value_create_object_with_accessor
 0004:00005124       ceflib.cef_v8value_create_string
 0004:0000510C       ceflib.cef_v8value_create_undefined
 0001:0003E2F4       ceflib.cef_v8_accessor_get
 0001:0003E3F8       ceflib.cef_v8_accessor_put
 0001:0003DF20       ceflib.cef_v8_handler_execute
 0001:0003E0AC       ceflib.cef_v8_handler_execute_function_with_context
 0004:000050C8       ceflib.cef_visit_all_cookies
 0004:000050D8       ceflib.cef_visit_storage
 0004:000050CC       ceflib.cef_visit_url_cookies
 0004:00005138       ceflib.cef_web_urlrequest_create
 0004:0000513C       ceflib.cef_xml_reader_create
 0004:00005140       ceflib.cef_zip_reader_create
 0001:0003CD64       ceflib.DateTimeToCefTime
 0001:00043F44       ceflib.Finalization
 0003:00000FE8       ceflib.LibHandle
 0001:0003CCF4       ceflib.SystemTimeToCefTime
 0001:0003C5EC       ceflib.SystemTimeToTzSpecificLocalTime
 0001:0003E4A8       ceflib.TCefBaseOwn.CreateData
 0001:0003E528       ceflib.TCefBaseOwn.Destroy
 0001:0003E578       ceflib.TCefBaseOwn.Lock
 0001:0003E584       ceflib.TCefBaseOwn.Unlock
 0001:0003E564       ceflib.TCefBaseOwn.Wrap
 0001:0003E590       ceflib.TCefBaseRef.Create
 0001:0003E660       ceflib.TCefBaseRef.Destroy
 0001:0003E694       ceflib.TCefBaseRef.UnWrap
 0001:0003E6DC       ceflib.TCefBaseRef.Wrap
 0001:0003E6F0       ceflib.TCefBrowserRef.CanGoBack
 0001:0003E704       ceflib.TCefBrowserRef.CanGoForward
 0001:0003E718       ceflib.TCefBrowserRef.ClearHistory
 0001:0003E720       ceflib.TCefBrowserRef.CloseBrowser
 0001:0003E728       ceflib.TCefBrowserRef.CloseDevTools
 0001:0003E730       ceflib.TCefBrowserRef.Find
 0001:0003E89C       ceflib.TCefBrowserRef.GetClient
 0001:0003E770       ceflib.TCefBrowserRef.GetFocusedFrame
 0001:0003E790       ceflib.TCefBrowserRef.GetFrame
 0001:0003E7C4       ceflib.TCefBrowserRef.GetFrameNames
 0001:0003E8BC       ceflib.TCefBrowserRef.GetImage
 0001:0003E8F0       ceflib.TCefBrowserRef.GetMainFrame
 0001:0003E910       ceflib.TCefBrowserRef.GetOpenerWindowHandle
 0001:0003E918       ceflib.TCefBrowserRef.GetSize
 0001:0003E948       ceflib.TCefBrowserRef.GetWindowHandle
 0001:0003E950       ceflib.TCefBrowserRef.GetZoomLevel
 0001:0003E964       ceflib.TCefBrowserRef.GoBack
 0001:0003E96C       ceflib.TCefBrowserRef.GoForward
 0001:0003E974       ceflib.TCefBrowserRef.HasDocument
 0001:0003E988       ceflib.TCefBrowserRef.HidePopup
 0001:0003E994       ceflib.TCefBrowserRef.Invalidate
 0001:0003E9A0       ceflib.TCefBrowserRef.IsPopup
 0001:0003E9B4       ceflib.TCefBrowserRef.IsPopupVisible
 0001:0003E9CC       ceflib.TCefBrowserRef.IsWindowRenderingDisabled
 0001:0003E9E0       ceflib.TCefBrowserRef.ParentWindowWillClose
 0001:0003E9E8       ceflib.TCefBrowserRef.Reload
 0001:0003E9F0       ceflib.TCefBrowserRef.ReloadIgnoreCache
 0001:0003E9F8       ceflib.TCefBrowserRef.SendCaptureLostEvent
 0001:0003EA04       ceflib.TCefBrowserRef.SendFocusEvent
 0001:0003EA14       ceflib.TCefBrowserRef.SendKeyEvent
 0001:0003EA3C       ceflib.TCefBrowserRef.SendMouseClickEvent
 0001:0003EA60       ceflib.TCefBrowserRef.SendMouseMoveEvent
 0001:0003EA7C       ceflib.TCefBrowserRef.SendMouseWheelEvent
 0001:0003EA98       ceflib.TCefBrowserRef.SetFocus
 0001:0003EAA4       ceflib.TCefBrowserRef.SetSize
 0001:0003EAC0       ceflib.TCefBrowserRef.SetZoomLevel
 0001:0003EAD4       ceflib.TCefBrowserRef.ShowDevTools
 0001:0003EADC       ceflib.TCefBrowserRef.StopFinding
 0001:0003EAE8       ceflib.TCefBrowserRef.StopLoad
 0001:0003EAF0       ceflib.TCefBrowserRef.UnWrap
 0001:00043C10       ceflib.TCefClientOwn.Create
 0001:00043CB8       ceflib.TCefClientOwn.GetDisplayHandler
 0001:00043CC4       ceflib.TCefClientOwn.GetDragHandler
 0001:00043CD0       ceflib.TCefClientOwn.GetFindHandler
 0001:00043CDC       ceflib.TCefClientOwn.GetFocusHandler
 0001:00043CE8       ceflib.TCefClientOwn.GetJsbindingHandler
 0001:00043CF4       ceflib.TCefClientOwn.GetJsdialogHandler
 0001:00043D00       ceflib.TCefClientOwn.GetKeyboardHandler
 0001:00043D0C       ceflib.TCefClientOwn.GetLifeSpanHandler
 0001:00043D18       ceflib.TCefClientOwn.GetLoadHandler
 0001:00043D24       ceflib.TCefClientOwn.GetMenuHandler
 0001:00043D30       ceflib.TCefClientOwn.GetPrintHandler
 0001:00043D3C       ceflib.TCefClientOwn.GetRenderHandler
 0001:00043D48       ceflib.TCefClientOwn.GetRequestHandler
 0001:0003F0A0       ceflib.TCefCustomStreamReader.Create
 0001:0003F110       ceflib.TCefCustomStreamReader.Create
 0001:0003F164       ceflib.TCefCustomStreamReader.Destroy
 0001:0003F198       ceflib.TCefCustomStreamReader.Eof
 0001:0003F208       ceflib.TCefCustomStreamReader.Read
 0001:0003F270       ceflib.TCefCustomStreamReader.Seek
 0001:0003F2D0       ceflib.TCefCustomStreamReader.Tell
 0001:00043E48       ceflib.TCefDisplayHandlerOwn.Create
 0001:00043EB8       ceflib.TCefDisplayHandlerOwn.OnAddressChange
 0001:00043EC0       ceflib.TCefDisplayHandlerOwn.OnConsoleMessage
 0001:00043ECC       ceflib.TCefDisplayHandlerOwn.OnNavStateChange
 0001:00043ED4       ceflib.TCefDisplayHandlerOwn.OnStatusMessage
 0001:00043EDC       ceflib.TCefDisplayHandlerOwn.OnTitleChange
 0001:00043EE0       ceflib.TCefDisplayHandlerOwn.OnTooltip
 0001:00043164       ceflib.TCefDomDocumentRef.GetBaseUrl
 0001:00043180       ceflib.TCefDomDocumentRef.GetBody
 0001:000431A0       ceflib.TCefDomDocumentRef.GetCompleteUrl
 0001:000431CC       ceflib.TCefDomDocumentRef.GetDocument
 0001:000431EC       ceflib.TCefDomDocumentRef.GetElementById
 0001:00043220       ceflib.TCefDomDocumentRef.GetFocusedNode
 0001:00043240       ceflib.TCefDomDocumentRef.GetHead
 0001:00043260       ceflib.TCefDomDocumentRef.GetSelectionAsMarkup
 0001:0004327C       ceflib.TCefDomDocumentRef.GetSelectionAsText
 0001:00043298       ceflib.TCefDomDocumentRef.GetSelectionEndNode
 0001:000432B8       ceflib.TCefDomDocumentRef.GetSelectionEndOffset
 0001:000432C0       ceflib.TCefDomDocumentRef.GetSelectionStartNode
 0001:000432E0       ceflib.TCefDomDocumentRef.GetSelectionStartOffset
 0001:000432E8       ceflib.TCefDomDocumentRef.GetTitle
 0001:00043304       ceflib.TCefDomDocumentRef.GetType
 0001:0004330C       ceflib.TCefDomDocumentRef.HasSelection
 0001:00043320       ceflib.TCefDomDocumentRef.UnWrap
 0001:0004380C       ceflib.TCefDomEventListenerOwn.Create
 0001:00043854       ceflib.TCefDomEventListenerOwn.HandleEvent
 0001:00043858       ceflib.TCefDomEventRef.CanBubble
 0001:0004386C       ceflib.TCefDomEventRef.CanCancel
 0001:00043880       ceflib.TCefDomEventRef.GetCategory
 0001:00043888       ceflib.TCefDomEventRef.GetCurrentTarget
 0001:000438A8       ceflib.TCefDomEventRef.GetDocument
 0001:000438C8       ceflib.TCefDomEventRef.GetPhase
 0001:000438D0       ceflib.TCefDomEventRef.GetTarget
 0001:000438F0       ceflib.TCefDomEventRef.GetType
 0001:0004390C       ceflib.TCefDomEventRef.UnWrap
 0001:00043368       ceflib.TCefDomNodeRef.AddEventListener
 0001:00043420       ceflib.TCefDomNodeRef.AddEventListenerProc
 0001:000434A8       ceflib.TCefDomNodeRef.GetAsMarkup
 0001:000434C4       ceflib.TCefDomNodeRef.GetDocument
 0001:000434E4       ceflib.TCefDomNodeRef.GetElementAttribute
 0001:00043510       ceflib.TCefDomNodeRef.GetElementAttributes
 0001:0004352C       ceflib.TCefDomNodeRef.GetElementInnerText
 0001:00043548       ceflib.TCefDomNodeRef.GetElementTagName
 0001:00043564       ceflib.TCefDomNodeRef.GetFirstChild
 0001:00043584       ceflib.TCefDomNodeRef.GetLastChild
 0001:000435A4       ceflib.TCefDomNodeRef.GetName
 0001:000435C0       ceflib.TCefDomNodeRef.GetNextSibling
 0001:000435E0       ceflib.TCefDomNodeRef.GetParent
 0001:00043600       ceflib.TCefDomNodeRef.GetPreviousSibling
 0001:00043620       ceflib.TCefDomNodeRef.GetType
 0001:00043628       ceflib.TCefDomNodeRef.GetValue
 0001:00043644       ceflib.TCefDomNodeRef.HasChildren
 0001:00043658       ceflib.TCefDomNodeRef.HasElementAttribute
 0001:00043680       ceflib.TCefDomNodeRef.HasElementAttributes
 0001:00043694       ceflib.TCefDomNodeRef.IsElement
 0001:000436A8       ceflib.TCefDomNodeRef.IsSame
 0001:00043748       ceflib.TCefDomNodeRef.IsText
 0001:0004375C       ceflib.TCefDomNodeRef.SetElementAttribute
 0001:0004379C       ceflib.TCefDomNodeRef.SetValue
 0001:000437C4       ceflib.TCefDomNodeRef.UnWrap
 0001:000430C8       ceflib.TCefDomVisitorOwn.Create
 0001:00043110       ceflib.TCefDomVisitorOwn.visit
 0001:00043954       ceflib.TCefFastDomEventListener.Create
 0001:00043998       ceflib.TCefFastDomEventListener.HandleEvent
 0001:00043114       ceflib.TCefFastDomVisitor.Create
 0001:00043158       ceflib.TCefFastDomVisitor.visit
 0001:00043B5C       ceflib.TCefFastV8Accessor.Create
 0001:00043BA8       ceflib.TCefFastV8Accessor.Get
 0001:00043BEC       ceflib.TCefFastV8Accessor.Put
 0001:0003EB38       ceflib.TCefFrameRef.Copy
 0001:0003EB40       ceflib.TCefFrameRef.Cut
 0001:0003EB48       ceflib.TCefFrameRef.Del
 0001:0003EB50       ceflib.TCefFrameRef.ExecuteJavaScript
 0001:0003EB90       ceflib.TCefFrameRef.GetBrowser
 0001:0003EBB0       ceflib.TCefFrameRef.GetName
 0001:0003EBCC       ceflib.TCefFrameRef.GetSource
 0001:0003EBE8       ceflib.TCefFrameRef.getText
 0001:0003EC04       ceflib.TCefFrameRef.GetUrl
 0001:0003EC20       ceflib.TCefFrameRef.IsFocused
 0001:0003EC34       ceflib.TCefFrameRef.IsMain
 0001:0003EC48       ceflib.TCefFrameRef.LoadFile
 0001:0003ED2C       ceflib.TCefFrameRef.LoadRequest
 0001:0003EDC0       ceflib.TCefFrameRef.LoadStream
 0001:0003EEC0       ceflib.TCefFrameRef.LoadString
 0001:0003EEF8       ceflib.TCefFrameRef.LoadUrl
 0001:0003EF18       ceflib.TCefFrameRef.Paste
 0001:0003EF20       ceflib.TCefFrameRef.Print
 0001:0003EF28       ceflib.TCefFrameRef.Redo
 0001:0003EF30       ceflib.TCefFrameRef.SelectAll
 0001:0003EF38       ceflib.TCefFrameRef.Undo
 0001:0003F058       ceflib.TCefFrameRef.UnWrap
 0001:0003EF40       ceflib.TCefFrameRef.ViewSource
 0001:0003EF48       ceflib.TCefFrameRef.VisitDom
 0001:0003EFDC       ceflib.TCefFrameRef.VisitDomProc
 0001:00043D54       ceflib.TCefLifeSpanHandlerOwn.Create
 0001:00043DD0       ceflib.TCefLifeSpanHandlerOwn.DoClose
 0001:00043DBC       ceflib.TCefLifeSpanHandlerOwn.OnAfterCreated
 0001:00043DC0       ceflib.TCefLifeSpanHandlerOwn.OnBeforeClose
 0001:00043DC4       ceflib.TCefLifeSpanHandlerOwn.OnBeforePopup
 0001:00043DD4       ceflib.TCefLifeSpanHandlerOwn.RunModal
 0001:00043DD8       ceflib.TCefLoadHandlerOwn.Create
 0001:00043E30       ceflib.TCefLoadHandlerOwn.OnLoadEnd
 0001:00043E38       ceflib.TCefLoadHandlerOwn.OnLoadError
 0001:00043E44       ceflib.TCefLoadHandlerOwn.OnLoadStart
 0001:0003F4F0       ceflib.TCefPostDataElementRef.GetBytes
 0001:0003F4FC       ceflib.TCefPostDataElementRef.GetBytesCount
 0001:0003F504       ceflib.TCefPostDataElementRef.GetFile
 0001:0003F520       ceflib.TCefPostDataElementRef.GetType
 0001:0003F528       ceflib.TCefPostDataElementRef.New
 0001:0003F544       ceflib.TCefPostDataElementRef.SetToBytes
 0001:0003F550       ceflib.TCefPostDataElementRef.SetToEmpty
 0001:0003F558       ceflib.TCefPostDataElementRef.SetToFile
 0001:0003F578       ceflib.TCefPostDataElementRef.UnWrap
 0001:0003F324       ceflib.TCefPostDataRef.AddElement
 0001:0003F3BC       ceflib.TCefPostDataRef.GetCount
 0001:0003F3C4       ceflib.TCefPostDataRef.GetElement
 0001:0003F3EC       ceflib.TCefPostDataRef.New
 0001:0003F408       ceflib.TCefPostDataRef.RemoveElement
 0001:0003F4A0       ceflib.TCefPostDataRef.RemoveElements
 0001:0003F4A8       ceflib.TCefPostDataRef.UnWrap
 0001:0003F5C0       ceflib.TCefRequestRef.GetFirstPartyForCookies
 0001:0003F5DC       ceflib.TCefRequestRef.GetFlags
 0001:0003F5E4       ceflib.TCefRequestRef.GetHeaderMap
 0001:0003F600       ceflib.TCefRequestRef.GetMethod
 0001:0003F61C       ceflib.TCefRequestRef.GetPostData
 0001:0003F63C       ceflib.TCefRequestRef.GetUrl
 0001:0003F658       ceflib.TCefRequestRef.New
 0001:0003F674       ceflib.TCefRequestRef.SetFirstPartyForCookies
 0001:0003F694       ceflib.TCefRequestRef.SetFlags
 0001:0003F6A0       ceflib.TCefRequestRef.SetHeaderMap
 0001:0003F6BC       ceflib.TCefRequestRef.SetMethod
 0001:0003F6DC       ceflib.TCefRequestRef.SetPostData
 0001:0003F774       ceflib.TCefRequestRef.SetUrl
 0001:0003F794       ceflib.TCefRequestRef.UnWrap
 0001:000439B4       ceflib.TCefResponseRef.GetHeader
 0001:000439E0       ceflib.TCefResponseRef.GetHeaderMap
 0001:000439FC       ceflib.TCefResponseRef.GetMimeType
 0001:00043A18       ceflib.TCefResponseRef.GetStatus
 0001:00043A20       ceflib.TCefResponseRef.GetStatusText
 0001:00043A3C       ceflib.TCefResponseRef.SetHeaderMap
 0001:00043A58       ceflib.TCefResponseRef.SetMimeType
 0001:00043A78       ceflib.TCefResponseRef.SetStatus
 0001:00043A84       ceflib.TCefResponseRef.SetStatusText
 0001:00043AA4       ceflib.TCefResponseRef.UnWrap
 0001:00043EE4       ceflib.TCefSchemeHandlerCallbackRef.BytesAvailable
 0001:00043EEC       ceflib.TCefSchemeHandlerCallbackRef.Cancel
 0001:00043EF4       ceflib.TCefSchemeHandlerCallbackRef.HeadersAvailable
 0001:00043EFC       ceflib.TCefSchemeHandlerCallbackRef.UnWrap
 0001:00041C10       ceflib.TCefSchemeHandlerFactoryOwn.Create
 0001:00041C6C       ceflib.TCefSchemeHandlerFactoryOwn.New
 0001:00041CB8       ceflib.TCefSchemeHandlerOwn.Cancel
 0001:00041CC0       ceflib.TCefSchemeHandlerOwn.Create
 0001:00041D70       ceflib.TCefSchemeHandlerOwn.GetResponseHeaders
 0001:00041D74       ceflib.TCefSchemeHandlerOwn.ProcessRequest
 0001:00041D80       ceflib.TCefSchemeHandlerOwn.ReadResponse
 0001:0003F7DC       ceflib.TCefStreamReaderRef.CreateForCustomStream
 0001:0003F880       ceflib.TCefStreamReaderRef.CreateForData
 0001:0003F8AC       ceflib.TCefStreamReaderRef.CreateForFile
 0001:0003F8DC       ceflib.TCefStreamReaderRef.CreateForStream
 0001:0003F960       ceflib.TCefStreamReaderRef.Eof
 0001:0003F974       ceflib.TCefStreamReaderRef.Read
 0001:0003F98C       ceflib.TCefStreamReaderRef.Seek
 0001:0003F998       ceflib.TCefStreamReaderRef.Tell
 0001:0003F9A0       ceflib.TCefStreamReaderRef.UnWrap
 0001:00043AEC       ceflib.TCefV8AccessorOwn.Create
 0001:00043B3C       ceflib.TCefV8AccessorOwn.Get
 0001:00043B50       ceflib.TCefV8AccessorOwn.Put
 0001:00042FC0       ceflib.TCefv8ContextRef.Current
 0001:00042FDC       ceflib.TCefv8ContextRef.Enter
 0001:00042FF0       ceflib.TCefv8ContextRef.Entered
 0001:0004300C       ceflib.TCefv8ContextRef.Exit
 0001:00043020       ceflib.TCefv8ContextRef.GetBrowser
 0001:00043040       ceflib.TCefv8ContextRef.GetFrame
 0001:00043060       ceflib.TCefv8ContextRef.GetGlobal
 0001:00043080       ceflib.TCefv8ContextRef.UnWrap
 0001:00042F58       ceflib.TCefv8HandlerOwn.Create
 0001:00042FA8       ceflib.TCefv8HandlerOwn.Execute
 0001:00042FB4       ceflib.TCefv8HandlerOwn.ExecuteFunctionWithContext
 0001:00042B4C       ceflib.TCefv8HandlerRef.Execute
 0001:00042D38       ceflib.TCefv8HandlerRef.ExecuteFunctionWithContext
 0001:00042F10       ceflib.TCefv8HandlerRef.UnWrap
 0001:00041D8C       ceflib.TCefv8ValueRef.CreateArray
 0001:00041DA8       ceflib.TCefv8ValueRef.CreateBool
 0001:00041DCC       ceflib.TCefv8ValueRef.CreateDate
 0001:00041E04       ceflib.TCefv8ValueRef.CreateDouble
 0001:00041E30       ceflib.TCefv8ValueRef.CreateFunction
 0001:00041EEC       ceflib.TCefv8ValueRef.CreateInt
 0001:00041F0C       ceflib.TCefv8ValueRef.CreateNull
 0001:00041F28       ceflib.TCefv8ValueRef.CreateObject
 0001:00041FCC       ceflib.TCefv8ValueRef.CreateObjectWithAccessor
 0001:000420AC       ceflib.TCefv8ValueRef.CreateObjectWithAccessorProc
 0001:00042138       ceflib.TCefv8ValueRef.CreateString
 0001:00042168       ceflib.TCefv8ValueRef.CreateUndefined
 0001:00042184       ceflib.TCefv8ValueRef.DeleteValueByIndex
 0001:0004219C       ceflib.TCefv8ValueRef.DeleteValueByKey
 0001:000421C4       ceflib.TCefv8ValueRef.ExecuteFunction
 0001:00042378       ceflib.TCefv8ValueRef.ExecuteFunctionWithContext
 0001:00042574       ceflib.TCefv8ValueRef.GetArrayLength
 0001:0004257C       ceflib.TCefv8ValueRef.GetBoolValue
 0001:00042590       ceflib.TCefv8ValueRef.GetDateValue
 0001:000425BC       ceflib.TCefv8ValueRef.GetDoubleValue
 0001:000425D0       ceflib.TCefv8ValueRef.GetFunctionHandler
 0001:000425F4       ceflib.TCefv8ValueRef.GetFunctionName
 0001:00042610       ceflib.TCefv8ValueRef.GetIntValue
 0001:00042618       ceflib.TCefv8ValueRef.GetKeys
 0001:000426F4       ceflib.TCefv8ValueRef.GetStringValue
 0001:00042710       ceflib.TCefv8ValueRef.GetUserData
 0001:00042730       ceflib.TCefv8ValueRef.GetValueByIndex
 0001:00042758       ceflib.TCefv8ValueRef.GetValueByKey
 0001:0004278C       ceflib.TCefv8ValueRef.HasValueByIndex
 0001:000427A4       ceflib.TCefv8ValueRef.HasValueByKey
 0001:000427CC       ceflib.TCefv8ValueRef.IsArray
 0001:000427E0       ceflib.TCefv8ValueRef.IsBool
 0001:000427F4       ceflib.TCefv8ValueRef.IsDate
 0001:00042808       ceflib.TCefv8ValueRef.IsDouble
 0001:0004281C       ceflib.TCefv8ValueRef.IsFunction
 0001:00042830       ceflib.TCefv8ValueRef.IsInt
 0001:00042844       ceflib.TCefv8ValueRef.IsNull
 0001:00042858       ceflib.TCefv8ValueRef.IsObject
 0001:0004286C       ceflib.TCefv8ValueRef.IsSame
 0001:0004290C       ceflib.TCefv8ValueRef.IsString
 0001:00042920       ceflib.TCefv8ValueRef.IsUndefined
 0001:00042934       ceflib.TCefv8ValueRef.SetValueByAccessor
 0001:0004296C       ceflib.TCefv8ValueRef.SetValueByIndex
 0001:00042A14       ceflib.TCefv8ValueRef.SetValueByKey
 0001:00042ACC       ceflib.TCefv8ValueRef.UnWrap
 0001:0003CC48       ceflib.TSHSyncGetResponseHeaders.Create
 0001:0003CC34       ceflib.TSHSyncGetResponseHeaders.Execute
 0001:0003C7E0       ceflib.TSHSyncProcessRequest.Create
 0001:0003C7C4       ceflib.TSHSyncProcessRequest.Execute
 0001:0003CA50       ceflib.TSHSyncReadResponse.Create
 0001:0003CA30       ceflib.TSHSyncReadResponse.Execute
 0001:0003C5E4       ceflib.TzSpecificLocalTimeToSystemTime
 0004:00002C54       Character.CategoryTable
 0004:00002C4C       Character.CatIndexPrimary
 0004:00002C50       Character.CatIndexSecondary
 0004:00002C48       Character.DataTable
 0003:00000A20       Character.Latin1Categories
 0004:00002C60       Character.NumericValueTable
 0004:00002C58       Character.NumIndexPrimary
 0004:00002C5C       Character.NumIndexSecondary
 0001:00009910       Character.TCharacter.CheckLetter
 0001:0000991C       Character.TCharacter.CheckLetterOrDigit
 0001:00009A38       Character.TCharacter.Initialize
 0001:00009A2C       Character.TCharacter.IsAscii
 0001:0000992C       Character.TCharacter.IsLatin1
 0001:00009938       Character.TCharacter.IsLetter
 0001:000099C4       Character.TCharacter.IsLetterOrDigit
 0004:00004F54       Classes..66
 0001:00020C34       Classes..EClassNotFound
 0001:00020F40       Classes..EComponentError
 0001:0002093C       Classes..EFCreateError
 0001:00020A70       Classes..EFilerError
 0001:00020840       Classes..EFileStreamError
 0001:000209D8       Classes..EFOpenError
 0001:00020CD0       Classes..EInvalidImage
 0001:00020E08       Classes..EListError
 0001:00020B08       Classes..EReadError
 0001:00020D6C       Classes..EResNotFound
 0001:000207A4       Classes..EStreamError
 0001:00020E9C       Classes..EStringListError
 0001:00027470       Classes..EThread
 0001:00020B9C       Classes..EWriteError
 0001:00028D98       Classes..TBasicAction
 0001:00028B7C       Classes..TBasicActionLink
 0001:00024D70       Classes..TClassFinder
 0001:0002226C       Classes..TCollection
 0001:000220C8       Classes..TCollectionEnumerator
 0001:00021E5C       Classes..TCollectionItem
 0001:00028234       Classes..TComponent
 0001:00036DC8       Classes..TComponent.FindComponent$ActRec
 0001:00027E5C       Classes..TComponentEnumerator
 0001:00024668       Classes..TCustomMemoryStream
 0001:00025144       Classes..TFiler
 0001:00024484       Classes..TFileStream
 0001:0002426C       Classes..THandleStream
 0001:00021318       Classes..TList
 0001:0002B2DC       Classes..TList.Sort$ActRec
 0001:00021144       Classes..TListEnumerator
 0001:000248B0       Classes..TMemoryStream
 0001:00021CE4       Classes..TPersistent
 0001:0002F390       Classes..TPropFixup
 0001:0002F5BC       Classes..TPropIntfFixup
 0001:00025B5C       Classes..TReader
 0001:000291A4       Classes..TRegGroup
 0001:00029604       Classes..TRegGroups
 0001:00024AF8       Classes..TResourceStream
 0001:00023C60       Classes..TStream
 0001:000235E4       Classes..TStringList
 0001:0002296C       Classes..TStrings
 0001:000227C4       Classes..TStringsEnumerator
 0001:00027664       Classes..TThread
 0001:00021A2C       Classes..TThreadList
 0001:00026A64       Classes..TWriter
 0001:0002F8E8       Classes.AddFinished
 0001:0002F920       Classes.AddNotFinished
 0001:0003058C       Classes.AddSubComponentsToLoaded
 0001:00033B28       Classes.AncestorIsValid
 0001:000305C8       Classes.CheckSubComponents
 0001:00035680       Classes.CheckSynchronize
 0002:0000024C       Classes.Classes
 0001:0002A794       Classes.ClassNotFound
 0001:0003786C       Classes.CleanupInstFreeList
 0001:0002AABC       Classes.CollectionsEqual
 0001:000306A8       Classes.ComponentCreated
 0001:000325C8       Classes.CopyBinary
 0001:00032538       Classes.CopyBytes
 0001:000324EC       Classes.CopyList
 0001:00032464       Classes.CopySetBody
 0001:00030728       Classes.CreateComponent
 0003:00000F64       Classes.CreateVCLComObjectProc
 0001:000355A8       Classes.DoneThreadSynchronization
 0001:0002C6CC       Classes.DoWrite
 0003:00000F74       Classes.Dummy32bitResHeader
 0001:0003793C       Classes.EFileStreamError.Create
 0001:0002F1C8       Classes.Error
 0001:0002A238       Classes.Error
 0004:00004F80       Classes.ExternalThreads
 0003:00000F70       Classes.FilerSignature
 0001:000379EC       Classes.Finalization
 0001:00033218       Classes.FindAncestor
 0001:0002A86C       Classes.FindClass
 0001:000308D8       Classes.FindExistingComponent
 0001:0002A9EC       Classes.FindGlobalComponent
 0004:00004F60       Classes.FindGlobalComponentProcs
 0001:0002A970       Classes.FindIdentToInt
 0001:0002A8F4       Classes.FindIntToIdent
 0001:00033F9C       Classes.FindMethodName
 0001:0002F7F0       Classes.FindNestedComponent
 0001:00031954       Classes.FindUniqueName
 0001:000355C0       Classes.FreeExternalThreads
 0001:000377EC       Classes.FreeIntConstList
 0001:0002A800       Classes.GetClass
 0001:00034690       Classes.GetComponentValue
 0001:0002BB28       Classes.GetDesigner
 0001:0002A788       Classes.GetFieldClassTable
 0001:000378A8       Classes.GetFreeInstBlockItemCount
 0004:00004F64       Classes.GlobalFixupList
 0001:0002F968       Classes.GlobalFixupReferences
 0005:00000010       Classes.GlobalLists
 0005:0000000C       Classes.GlobalLoaded
 0004:00004F48       Classes.GlobalNameSpace
 0001:000310E8       Classes.HandleException
 0001:00035574       Classes.InitThreadSynchronization
 0004:00004F84       Classes.InstBlockList
 0004:00004F88       Classes.InstFreeList
 0004:00004F58       Classes.IntConstList
 0001:00033D1C       Classes.IsDefault
 0001:00033B98       Classes.IsDefaultFloatProp
 0001:00033BF4       Classes.IsDefaultInt64Prop
 0001:00033EC0       Classes.IsDefaultInterfaceProp
 0001:00033FF4       Classes.IsDefaultMethodProp
 0001:00033D74       Classes.IsDefaultObjectProp
 0001:00033B40       Classes.IsDefaultOrdProp
 0001:0003412C       Classes.IsDefaultPropertyValue
 0001:00033C4C       Classes.IsDefaultStrProp
 0001:00033DF4       Classes.IsDefaultValue
 0001:00034094       Classes.IsDefaultVariantProp
 0001:0002AA2C       Classes.IsUniqueGlobalComponentName
 0004:00004F4C       Classes.IsUniqueGlobalComponentNameProc
 0001:00037864       Classes.ModuleUnload
 0003:00000F94       Classes.NilMethod
 0001:0002BBCC       Classes.NotifyDesigner
 0001:00033CDC       Classes.ObjectAncestorMatch
 0001:00034678       Classes.OwnedBy
 0003:00000FA0       Classes.Priorities
 0001:0002FCA8       Classes.PropertyNotFound
 0001:000311B8       Classes.PropPathError
 0001:0002FC9C       Classes.PropValueError
 0001:0002B1A4       Classes.QuickSort
 0001:0002E380       Classes.RaiseException
 0001:00032AB0       Classes.ReadCustomVariant
 0001:0002FC84       Classes.ReadError
 0001:000306C8       Classes.Recover
 0004:00004F5C       Classes.RegGroups
 0001:000378D8       Classes.ReleaseObjectInstanceBlocks
 0001:0002FB3C       Classes.RemoveFixupReferences
 0001:0002FBF0       Classes.RemoveFixups
 0001:0002FFEC       Classes.RemoveGlobalFixup
 0001:0003564C       Classes.ResetSyncEvent
 0001:0002C838       Classes.ReturnAddr
 0001:0002AD20       Classes.ReturnAddr
 0001:00030838       Classes.SetCompName
 0001:0002FCD4       Classes.SetElementValue
 0001:00031530       Classes.SetInterfaceReference
 0001:0003144C       Classes.SetIntIdent
 0001:00031494       Classes.SetObjectIdent
 0001:00030640       Classes.SetSubComponentState
 0001:000314D4       Classes.SetVariantReference
 0001:00035674       Classes.SignalSyncEvent
 0001:00032220       Classes.SkipBinary
 0001:00032250       Classes.SkipCollection
 0001:000321F4       Classes.SkipList
 0001:0002E16C       Classes.StringListCompareStrings
 0004:00004F50       Classes.SyncEvent
 0003:00000F9C       Classes.SyncList
 0001:00037760       Classes.TBasicAction.Change
 0001:000375EC       Classes.TBasicAction.Create
 0001:00037630       Classes.TBasicAction.Destroy
 0001:000376CC       Classes.TBasicAction.Execute
 0001:0003769C       Classes.TBasicAction.ExecuteTarget
 0001:00037698       Classes.TBasicAction.HandlesTarget
 0001:000376A0       Classes.TBasicAction.Notification
 0001:00037774       Classes.TBasicAction.RegisterChanges
 0001:000377C0       Classes.TBasicAction.SetActionComponent
 0001:00037704       Classes.TBasicAction.SetOnExecute
 0001:00037780       Classes.TBasicAction.UnRegisterChanges
 0001:000376E8       Classes.TBasicAction.Update
 0001:000376C8       Classes.TBasicAction.UpdateTarget
 0001:0003753C       Classes.TBasicActionLink.AssignClient
 0001:00037574       Classes.TBasicActionLink.Change
 0001:000374F8       Classes.TBasicActionLink.Create
 0001:00037540       Classes.TBasicActionLink.Destroy
 0001:0003758C       Classes.TBasicActionLink.Execute
 0001:000375D4       Classes.TBasicActionLink.IsOnExecuteLinked
 0001:000375A8       Classes.TBasicActionLink.SetAction
 0001:000375D8       Classes.TBasicActionLink.SetOnExecute
 0001:000375E0       Classes.TBasicActionLink.Update
 0001:0002A4F4       Classes.TClassFinder.Create
 0001:0002A634       Classes.TClassFinder.Destroy
 0001:0002A664       Classes.TClassFinder.GetClass
 0001:0002A700       Classes.TClassFinder.GetClasses
 0001:0002BEFC       Classes.TCollection.Add
 0001:0002C418       Classes.TCollection.Added
 0001:0002BF1C       Classes.TCollection.Assign
 0001:0002BFC4       Classes.TCollection.BeginUpdate
 0001:0002BFC8       Classes.TCollection.Changed
 0001:0002BFD8       Classes.TCollection.Clear
 0001:0002BE64       Classes.TCollection.Create
 0001:0002C3DC       Classes.TCollection.Delete
 0001:0002C41C       Classes.TCollection.Deleting
 0001:0002BEB0       Classes.TCollection.Destroy
 0001:0002C040       Classes.TCollection.EndUpdate
 0001:0002C04C       Classes.TCollection.FindItemID
 0001:0002C080       Classes.TCollection.GetAttr
 0001:0002C07C       Classes.TCollection.GetAttrCount
 0001:0002C0A0       Classes.TCollection.GetCapacity
 0001:0002C0C8       Classes.TCollection.GetCount
 0001:0002C090       Classes.TCollection.GetEnumerator
 0001:0002C0D0       Classes.TCollection.GetItem
 0001:0002C0A8       Classes.TCollection.GetItemAttr
 0001:0002C0E4       Classes.TCollection.GetNamePath
 0001:0002C198       Classes.TCollection.GetPropName
 0001:0002C2EC       Classes.TCollection.Insert
 0001:0002C308       Classes.TCollection.InsertItem
 0001:0002C420       Classes.TCollection.Notify
 0001:0002C40C       Classes.TCollection.Owner
 0001:0002C370       Classes.TCollection.RemoveItem
 0001:0002C3C4       Classes.TCollection.SetCapacity
 0001:0002C3D4       Classes.TCollection.SetItemName
 0001:0002C3D8       Classes.TCollection.Update
 0001:0002BDF8       Classes.TCollectionEnumerator.Create
 0001:0002BE3C       Classes.TCollectionEnumerator.GetCurrent
 0001:0002BE48       Classes.TCollectionEnumerator.MoveNext
 0001:0002BC98       Classes.TCollectionItem.Changed
 0001:0002BC30       Classes.TCollectionItem.Create
 0001:0002BC68       Classes.TCollectionItem.Destroy
 0001:0002BCD4       Classes.TCollectionItem.GetDisplayName
 0001:0002BCBC       Classes.TCollectionItem.GetIndex
 0001:0002BCE8       Classes.TCollectionItem.GetNamePath
 0001:0002BD94       Classes.TCollectionItem.GetOwner
 0001:0002BD98       Classes.TCollectionItem.SetCollection
 0001:0002BDC0       Classes.TCollectionItem.SetDisplayName
 0001:0002BDC8       Classes.TCollectionItem.SetIndex
 0001:00036FF0       Classes.TComponent.AddSortedComponent
 0001:0003680C       Classes.TComponent.BeforeDestruction
 0001:000370A4       Classes.TComponent.ChangeName
 0001:00036778       Classes.TComponent.Create
 0001:00036BB8       Classes.TComponent.DefineProperties
 0001:000367C4       Classes.TComponent.Destroy
 0001:00036A3C       Classes.TComponent.DestroyComponents
 0001:00036AA8       Classes.TComponent.Destroying
 0001:00037200       Classes.TComponent.ExecuteAction
 0001:00036E8C       Classes.TComponent.FindComponent
 0001:00036E80       Classes.TComponent.FindComponent$ActRec.$0$Body
 0001:00036F78       Classes.TComponent.FindSortedComponent
 0001:00036858       Classes.TComponent.FreeNotification
 0001:00037334       Classes.TComponent.FreeOnRelease
 0001:00036C5C       Classes.TComponent.GetChildOwner
 0001:00036C60       Classes.TComponent.GetChildParent
 0001:00036C54       Classes.TComponent.GetChildren
 0001:00037264       Classes.TComponent.GetComObject
 0001:000370F8       Classes.TComponent.GetComponent
 0001:00037124       Classes.TComponent.GetComponentCount
 0001:000370DC       Classes.TComponent.GetComponentIndex
 0001:00036C64       Classes.TComponent.GetEnumerator
 0001:00036C74       Classes.TComponent.GetNamePath
 0001:00036C88       Classes.TComponent.GetOwner
 0001:00036C90       Classes.TComponent.GetParentComponent
 0001:00036C50       Classes.TComponent.HasParent
 0001:000368EC       Classes.TComponent.Insert
 0001:000369A0       Classes.TComponent.InsertComponent
 0001:000373CC       Classes.TComponent.IntfGetComponent
 0001:000373D0       Classes.TComponent.IsImplementorOf
 0001:00036CB0       Classes.TComponent.Loaded
 0001:00036B58       Classes.TComponent.Notification
 0001:00036CBC       Classes.TComponent.PaletteCreated
 0001:0003734C       Classes.TComponent.QueryInterface
 0001:000368AC       Classes.TComponent.ReadLeft
 0001:00036CC0       Classes.TComponent.ReadState
 0001:000368C0       Classes.TComponent.ReadTop
 0001:00037450       Classes.TComponent.ReferenceInterface
 0001:00036928       Classes.TComponent.Remove
 0001:00036A04       Classes.TComponent.RemoveComponent
 0001:00036B3C       Classes.TComponent.RemoveFreeNotification
 0001:00036818       Classes.TComponent.RemoveFreeNotifications
 0001:00036AE4       Classes.TComponent.RemoveNotification
 0001:0003731C       Classes.TComponent.SafeCallException
 0001:00036C8C       Classes.TComponent.SetChildOrder
 0001:00037134       Classes.TComponent.SetComponentIndex
 0001:00037188       Classes.TComponent.SetDesigning
 0001:00037014       Classes.TComponent.SetName
 0001:00036C94       Classes.TComponent.SetParentComponent
 0001:000371D8       Classes.TComponent.SetReference
 0001:00037250       Classes.TComponent.SetSubComponent
 0001:00037228       Classes.TComponent.UpdateAction
 0001:00036CA4       Classes.TComponent.Updated
 0001:00037344       Classes.TComponent.UpdateRegistry
 0001:00036C98       Classes.TComponent.Updating
 0001:00036D58       Classes.TComponent.ValidateContainer
 0001:00036D6C       Classes.TComponent.ValidateInsert
 0001:00036CD0       Classes.TComponent.ValidateRename
 0001:000368D4       Classes.TComponent.WriteLeft
 0001:00036CC8       Classes.TComponent.WriteState
 0001:000368E0       Classes.TComponent.WriteTop
 0001:0003738C       Classes.TComponent._AddRef
 0001:000373AC       Classes.TComponent._Release
 0001:0003670C       Classes.TComponentEnumerator.Create
 0001:00036750       Classes.TComponentEnumerator.GetCurrent
 0001:0003675C       Classes.TComponentEnumerator.MoveNext
 0001:0002EE5C       Classes.TCustomMemoryStream.Read
 0001:0002EED0       Classes.TCustomMemoryStream.SaveToFile
 0001:0002EEB8       Classes.TCustomMemoryStream.SaveToStream
 0001:0002EE94       Classes.TCustomMemoryStream.Seek
 0001:0002EE54       Classes.TCustomMemoryStream.SetPointer
 0001:0002F31C       Classes.TFiler.Create
 0001:000254FC       Classes.TFiler.DefineBinaryProperty
 0001:000254F4       Classes.TFiler.DefineProperty
 0001:0002F364       Classes.TFiler.Destroy
 0001:00025504       Classes.TFiler.FlushBuffer
 0001:0002F38C       Classes.TFiler.SetRoot
 0001:0002EC68       Classes.TFileStream.Create
 0001:0002ECAC       Classes.TFileStream.Create
 0001:0002EE20       Classes.TFileStream.Destroy
 0001:0002EBA4       Classes.THandleStream.Create
 0001:0002EBE0       Classes.THandleStream.Read
 0001:0002EC00       Classes.THandleStream.Seek
 0001:0002EC2C       Classes.THandleStream.SetSize
 0001:0002EC40       Classes.THandleStream.SetSize
 0001:0002EBF0       Classes.THandleStream.Write
 0004:00004F68       Classes.ThreadLock
 0001:00035874       Classes.ThreadProc
 0001:0002AC60       Classes.TList.Add
 0001:0002B49C       Classes.TList.Assign
 0001:0002ACA0       Classes.TList.Clear
 0001:0002ACB8       Classes.TList.Delete
 0001:0002AC40       Classes.TList.Destroy
 0001:0002AD5C       Classes.TList.Error
 0001:0002AD24       Classes.TList.Error
 0001:0002ADB0       Classes.TList.Exchange
 0001:0002AE00       Classes.TList.Expand
 0001:0002B440       Classes.TList.Extract
 0001:0002B448       Classes.TList.ExtractItem
 0001:0002AE18       Classes.TList.First
 0001:0002AE20       Classes.TList.Get
 0001:0002AE44       Classes.TList.GetEnumerator
 0001:0002AE54       Classes.TList.Grow
 0001:0002AE88       Classes.TList.IndexOf
 0001:0002AEAC       Classes.TList.IndexOfItem
 0001:0002AED8       Classes.TList.Insert
 0001:0002AF50       Classes.TList.Last
 0001:0002AF74       Classes.TList.Move
 0001:0002B498       Classes.TList.Notify
 0001:0002B050       Classes.TList.Pack
 0001:0002AFCC       Classes.TList.Put
 0001:0002B028       Classes.TList.Remove
 0001:0002B030       Classes.TList.RemoveItem
 0001:0002B0C4       Classes.TList.SetCapacity
 0001:0002B100       Classes.TList.SetCount
 0001:0002B3A0       Classes.TList.Sort
 0001:0002B394       Classes.TList.Sort$ActRec.$0$Body
 0001:0002B420       Classes.TList.SortList
 0001:0002ABD8       Classes.TListEnumerator.Create
 0001:0002AC1C       Classes.TListEnumerator.GetCurrent
 0001:0002AC28       Classes.TListEnumerator.MoveNext
 0001:0002EF54       Classes.TMemoryStream.Clear
 0001:0002EF28       Classes.TMemoryStream.Destroy
 0001:0002EFA4       Classes.TMemoryStream.LoadFromFile
 0001:0002EF6C       Classes.TMemoryStream.LoadFromStream
 0001:0002F04C       Classes.TMemoryStream.Realloc
 0001:0002EFF8       Classes.TMemoryStream.SetCapacity
 0001:0002F020       Classes.TMemoryStream.SetSize
 0001:0002F0CC       Classes.TMemoryStream.Write
 0001:0002B9B0       Classes.TPersistent.Assign
 0001:0002B9C4       Classes.TPersistent.AssignError
 0001:0002BA80       Classes.TPersistent.AssignTo
 0001:0002BA88       Classes.TPersistent.DefineProperties
 0001:0002B984       Classes.TPersistent.Destroy
 0001:0002BA8C       Classes.TPersistent.GetNamePath
 0001:0002BB24       Classes.TPersistent.GetOwner
 0001:0002F6A4       Classes.TPropFixup.Create
 0001:0002F6FC       Classes.TPropFixup.MakeGlobalReference
 0001:0002F75C       Classes.TPropFixup.ResolveReference
 0001:0002F76C       Classes.TPropIntfFixup.ResolveReference
 0001:0002FD28       Classes.TReader.BeginReferences
 0001:0002FD90       Classes.TReader.CheckValue
 0001:00032620       Classes.TReader.CopyValue
 0001:0002FDF0       Classes.TReader.DefineBinaryProperty
 0001:0002FDB4       Classes.TReader.DefineProperty
 0001:0002FCEC       Classes.TReader.Destroy
 0001:00030074       Classes.TReader.DoFixupReferences
 0001:0002FED8       Classes.TReader.EndOfList
 0001:0002FEEC       Classes.TReader.EndReferences
 0001:0002FF08       Classes.TReader.Error
 0001:000328FC       Classes.TReader.FindAncestorComponent
 0001:000329F4       Classes.TReader.FindComponentClass
 0001:0002FF9C       Classes.TReader.FindMethod
 0001:0002FF2C       Classes.TReader.FindMethodInstance
 0001:000301B8       Classes.TReader.FixupReferences
 0001:000301F0       Classes.TReader.FlushBuffer
 0001:00030214       Classes.TReader.FreeFixups
 0001:00030250       Classes.TReader.GetFieldClass
 0001:000302E4       Classes.TReader.GetPosition
 0001:000302FC       Classes.TReader.NextValue
 0001:0003030C       Classes.TReader.PropertyError
 0001:00030320       Classes.TReader.Read
 0001:000303A8       Classes.TReader.ReadBoolean
 0001:0003036C       Classes.TReader.ReadBuffer
 0001:000303BC       Classes.TReader.ReadChar
 0001:000304B0       Classes.TReader.ReadCollection
 0001:0003097C       Classes.TReader.ReadComponent
 0001:00031CF0       Classes.TReader.ReadComponents
 0001:00030DBC       Classes.TReader.ReadCurrency
 0001:00030BBC       Classes.TReader.ReadData
 0001:00030C2C       Classes.TReader.ReadDataInner
 0001:00030E0C       Classes.TReader.ReadDate
 0001:00030D34       Classes.TReader.ReadDouble
 0001:00030CFC       Classes.TReader.ReadFloat
 0001:00030E50       Classes.TReader.ReadIdent
 0001:00031054       Classes.TReader.ReadInt64
 0001:00030FE8       Classes.TReader.ReadInteger
 0001:00031098       Classes.TReader.ReadListBegin
 0001:000310A0       Classes.TReader.ReadListEnd
 0001:000310A8       Classes.TReader.ReadPrefix
 0001:000311D4       Classes.TReader.ReadProperty
 0001:000315F0       Classes.TReader.ReadPropValue
 0001:000319BC       Classes.TReader.ReadRootComponent
 0001:00031DE0       Classes.TReader.ReadSet
 0001:00031E9C       Classes.TReader.ReadSignature
 0001:00030D78       Classes.TReader.ReadSingle
 0001:00031EC0       Classes.TReader.ReadStr
 0001:00031F50       Classes.TReader.ReadString
 0001:00032178       Classes.TReader.ReadValue
 0001:00032C78       Classes.TReader.ReadVariant
 0001:00030450       Classes.TReader.ReadWideChar
 0001:00032038       Classes.TReader.ReadWideString
 0001:000329B4       Classes.TReader.ReferenceName
 0001:000329CC       Classes.TReader.SetName
 0001:0003218C       Classes.TReader.SetPosition
 0001:00032A68       Classes.TReader.SkipBytes
 0001:00032850       Classes.TReader.SkipComponent
 0001:00032808       Classes.TReader.SkipProperty
 0001:000321AC       Classes.TReader.SkipSetBody
 0001:000322B4       Classes.TReader.SkipValue
 0001:00029AE0       Classes.TRegGroup.AddClass
 0001:00029AEC       Classes.TRegGroup.BestClass
 0001:00029B4C       Classes.TRegGroup.BestGroup
 0001:00029BBC       Classes.TRegGroup.Create
 0001:00029C18       Classes.TRegGroup.Destroy
 0001:00029C58       Classes.TRegGroup.GetClass
 0001:00029CA8       Classes.TRegGroup.GetClasses
 0001:00029CF0       Classes.TRegGroup.IndexOfClass
 0001:00029D68       Classes.TRegGroup.InGroup
 0001:00029DAC       Classes.TRegGroup.RegisterClass
 0001:00029E60       Classes.TRegGroup.RegisterClassAlias
 0001:00029E98       Classes.TRegGroup.Registered
 0001:00029EB0       Classes.TRegGroup.UnregisterClass
 0001:00029F10       Classes.TRegGroup.UnregisterModuleClasses
 0001:0002A050       Classes.TRegGroups.Activate
 0001:0002A09C       Classes.TRegGroups.AddClass
 0001:0002A0BC       Classes.TRegGroups.Create
 0001:0002A130       Classes.TRegGroups.Destroy
 0001:0002A190       Classes.TRegGroups.FindGroup
 0001:0002A1D4       Classes.TRegGroups.GetClass
 0001:0002A218       Classes.TRegGroups.GroupedWith
 0001:0002A2BC       Classes.TRegGroups.GroupWith
 0001:0002A390       Classes.TRegGroups.Lock
 0001:0002A39C       Classes.TRegGroups.RegisterClass
 0001:0002A3B4       Classes.TRegGroups.RegisterClassAlias
 0001:0002A3D4       Classes.TRegGroups.Registered
 0001:0002A418       Classes.TRegGroups.StartGroup
 0001:0002A468       Classes.TRegGroups.Unlock
 0001:0002A474       Classes.TRegGroups.UnregisterClass
 0001:0002A4A4       Classes.TRegGroups.UnregisterModuleClasses
 0001:0002F11C       Classes.TResourceStream.Create
 0001:0002F174       Classes.TResourceStream.CreateFromID
 0001:0002F2D4       Classes.TResourceStream.Destroy
 0001:0002F268       Classes.TResourceStream.Initialize
 0001:0002F304       Classes.TResourceStream.Write
 0001:0002E558       Classes.TStream.CopyFrom
 0001:0002E9C0       Classes.TStream.FixupResourceHeader
 0001:0002E294       Classes.TStream.GetPosition
 0001:0002E2C8       Classes.TStream.GetSize
 0001:0002425C       Classes.TStream.Read
 0001:0002E4E8       Classes.TStream.ReadBuffer
 0001:0002E64C       Classes.TStream.ReadComponent
 0001:0002E710       Classes.TStream.ReadComponentRes
 0001:0002EAB8       Classes.TStream.ReadResHeader
 0001:0002E3F4       Classes.TStream.Seek
 0001:0002E478       Classes.TStream.Seek
 0001:0002E2B4       Classes.TStream.SetPosition
 0001:0002E32C       Classes.TStream.SetSize
 0001:0002E314       Classes.TStream.SetSize
 0001:0002E318       Classes.TStream.SetSize64
 0001:00024264       Classes.TStream.Write
 0001:0002E520       Classes.TStream.WriteBuffer
 0001:0002E6AC       Classes.TStream.WriteComponent
 0001:0002E72C       Classes.TStream.WriteComponentRes
 0001:0002E6B4       Classes.TStream.WriteDescendent
 0001:0002EA84       Classes.TStream.WriteDescendentRes
 0001:0002E734       Classes.TStream.WriteResourceHeader
 0001:0002DB7C       Classes.TStringList.Add
 0001:0002DB8C       Classes.TStringList.AddObject
 0001:0002DBF0       Classes.TStringList.Changed
 0001:0002DC0C       Classes.TStringList.Changing
 0001:0002DC28       Classes.TStringList.Clear
 0001:0002E1D4       Classes.TStringList.CompareStrings
 0001:0002E228       Classes.TStringList.Create
 0001:0002E1F0       Classes.TStringList.Create
 0001:0002E19C       Classes.TStringList.CustomSort
 0001:0002DC90       Classes.TStringList.Delete
 0001:0002DAF8       Classes.TStringList.Destroy
 0001:0002DD10       Classes.TStringList.Exchange
 0001:0002DD6C       Classes.TStringList.ExchangeItems
 0001:0002DD90       Classes.TStringList.Find
 0001:0002DE14       Classes.TStringList.Get
 0001:0002DE44       Classes.TStringList.GetCapacity
 0001:0002DE48       Classes.TStringList.GetCount
 0001:0002DE4C       Classes.TStringList.GetObject
 0001:0002DE70       Classes.TStringList.Grow
 0001:0002DEA4       Classes.TStringList.IndexOf
 0001:0002DEE0       Classes.TStringList.Insert
 0001:0002DF44       Classes.TStringList.InsertItem
 0001:0002DEF0       Classes.TStringList.InsertObject
 0001:0002DFC0       Classes.TStringList.Put
 0001:0002E018       Classes.TStringList.PutObject
 0001:0002E054       Classes.TStringList.QuickSort
 0001:0002E0EC       Classes.TStringList.SetCapacity
 0001:0002E26C       Classes.TStringList.SetCaseSensitive
 0001:0002E12C       Classes.TStringList.SetSorted
 0001:0002E14C       Classes.TStringList.SetUpdateState
 0001:0002E18C       Classes.TStringList.Sort
 0001:0002C4EC       Classes.TStrings.Add
 0001:0002C510       Classes.TStrings.AddObject
 0001:0002C540       Classes.TStrings.AddStrings
 0001:0002C534       Classes.TStrings.Append
 0001:0002C5F8       Classes.TStrings.Assign
 0001:0002C6B4       Classes.TStrings.BeginUpdate
 0001:000234E4       Classes.TStrings.Clear
 0001:0002DAB0       Classes.TStrings.CompareStrings
 0001:0002C724       Classes.TStrings.DefineProperties
 0001:000234EC       Classes.TStrings.Delete
 0001:0002C4BC       Classes.TStrings.Destroy
 0001:0002C77C       Classes.TStrings.EndUpdate
 0001:0002C790       Classes.TStrings.Equals
 0001:0002C874       Classes.TStrings.Error
 0001:0002C83C       Classes.TStrings.Error
 0001:0002C8CC       Classes.TStrings.Exchange
 0001:0002C9B8       Classes.TStrings.GetCapacity
 0001:0002C9C0       Classes.TStrings.GetCommaText
 0001:0002CA58       Classes.TStrings.GetDelimitedText
 0001:0002D99C       Classes.TStrings.GetDelimiter
 0001:0002CCC8       Classes.TStrings.GetEnumerator
 0001:0002D9B8       Classes.TStrings.GetLineBreak
 0001:0002DABC       Classes.TStrings.GetNameValueSeparator
 0001:0002CCD8       Classes.TStrings.GetObject
 0001:0002D9F4       Classes.TStrings.GetQuoteChar
 0001:0002DA10       Classes.TStrings.GetStrictDelimiter
 0001:0002CCDC       Classes.TStrings.GetText
 0001:0002CD30       Classes.TStrings.GetTextStr
 0001:0002CEC8       Classes.TStrings.IndexOf
 0001:0002CF54       Classes.TStrings.IndexOfName
 0001:0002D028       Classes.TStrings.IndexOfObject
 0001:000234F4       Classes.TStrings.Insert
 0001:0002D05C       Classes.TStrings.InsertObject
 0001:0002D0E0       Classes.TStrings.LoadFromFile
 0001:0002D08C       Classes.TStrings.LoadFromFile
 0001:0002D13C       Classes.TStrings.LoadFromStream
 0001:0002D148       Classes.TStrings.LoadFromStream
 0001:0002D23C       Classes.TStrings.Move
 0001:0002D2EC       Classes.TStrings.Put
 0001:0002D31C       Classes.TStrings.PutObject
 0001:0002D320       Classes.TStrings.ReadData
 0001:0002D3D0       Classes.TStrings.SaveToFile
 0001:0002D3E0       Classes.TStrings.SaveToFile
 0001:0002D450       Classes.TStrings.SaveToStream
 0001:0002D440       Classes.TStrings.SaveToStream
 0001:0002D508       Classes.TStrings.SetCapacity
 0001:0002D50C       Classes.TStrings.SetCommaText
 0001:0002D7EC       Classes.TStrings.SetDelimitedText
 0001:0002DA28       Classes.TStrings.SetDelimiter
 0001:0002DA48       Classes.TStrings.SetLineBreak
 0001:0002DAD8       Classes.TStrings.SetNameValueSeparator
 0001:0002DA74       Classes.TStrings.SetQuoteChar
 0001:0002DA94       Classes.TStrings.SetStrictDelimiter
 0001:0002D534       Classes.TStrings.SetStringsAdapter
 0001:0002D568       Classes.TStrings.SetText
 0001:0002D5B8       Classes.TStrings.SetTextStr
 0001:0002D764       Classes.TStrings.SetUpdateState
 0001:0002D768       Classes.TStrings.WriteData
 0001:0002C444       Classes.TStringsEnumerator.Create
 0001:0002C488       Classes.TStringsEnumerator.GetCurrent
 0001:0002C4A0       Classes.TStringsEnumerator.MoveNext
 0004:00004F44       Classes.TThread.$ClassInitFlag
 0001:00035AC8       Classes.TThread.AfterConstruction
 0001:00035B70       Classes.TThread.CallOnTerminate
 0001:00035B58       Classes.TThread.CheckThreadError
 0001:00035ADC       Classes.TThread.CheckThreadError
 0001:00035928       Classes.TThread.Create
 0002:0000023C       Classes.TThread.Create@
 0001:00035A2C       Classes.TThread.Destroy
 0001:00035AA0       Classes.TThread.Destroy@
 0001:00035B84       Classes.TThread.DoTerminate
 0005:00000008       Classes.TThread.FCurrentThread
 0001:00035B98       Classes.TThread.GetPriority
 0001:00035BD4       Classes.TThread.InternalStart
 0001:0003666C       Classes.TThread.NameThreadForDebugging
 0001:00035E00       Classes.TThread.Queue
 0001:00036268       Classes.TThread.Queue
 0001:00035D34       Classes.TThread.Queue
 0001:00035CAC       Classes.TThread.Queue
 0001:000364A0       Classes.TThread.RemoveQueuedEvents
 0001:000363FC       Classes.TThread.RemoveQueuedEvents
 0001:00035EA0       Classes.TThread.RemoveQueuedEvents
 0001:00036560       Classes.TThread.Resume
 0001:00035C80       Classes.TThread.SetPriority
 0001:000364B4       Classes.TThread.SetSuspended
 0001:000364CC       Classes.TThread.SpinWait
 0001:000364E8       Classes.TThread.Start
 0001:00035F64       Classes.TThread.StaticQueue
 0001:000363E8       Classes.TThread.StaticSynchronize
 0001:000364F0       Classes.TThread.Suspend
 0001:00035F78       Classes.TThread.Synchronize
 0001:0003634C       Classes.TThread.Synchronize
 0001:000361D8       Classes.TThread.Synchronize
 0001:0003613C       Classes.TThread.Synchronize
 0001:00036170       Classes.TThread.Synchronize
 0001:00036588       Classes.TThread.Terminate
 0001:000365AC       Classes.TThread.WaitFor
 0001:0002B838       Classes.TThreadList.Add
 0001:0002B8C0       Classes.TThreadList.Clear
 0001:0002B768       Classes.TThreadList.Create
 0001:0002B7BC       Classes.TThreadList.Destroy
 0001:0002B908       Classes.TThreadList.LockList
 0001:0002B91C       Classes.TThreadList.Remove
 0001:0002B924       Classes.TThreadList.RemoveItem
 0001:0002B978       Classes.TThreadList.UnlockList
 0001:00032EC4       Classes.TWriter.AddAncestor
 0001:00032EF8       Classes.TWriter.DefineBinaryProperty
 0001:00032ED0       Classes.TWriter.DefineProperty
 0001:00032E98       Classes.TWriter.Destroy
 0001:00032F34       Classes.TWriter.FindMethodName
 0001:00032F7C       Classes.TWriter.FlushBuffer
 0001:00035550       Classes.TWriter.GetLookupInfo
 0001:00032F24       Classes.TWriter.GetPosition
 0001:00032F84       Classes.TWriter.SetPosition
 0001:00032FC0       Classes.TWriter.SetRoot
 0001:00032FD8       Classes.TWriter.Write
 0001:00033024       Classes.TWriter.WriteBinary
 0001:000330C4       Classes.TWriter.WriteBoolean
 0001:000330AC       Classes.TWriter.WriteBuffer
 0001:000330D8       Classes.TWriter.WriteChar
 0001:00033178       Classes.TWriter.WriteCollection
 0001:00033268       Classes.TWriter.WriteComponent
 0001:00033810       Classes.TWriter.WriteCurrency
 0001:000333BC       Classes.TWriter.WriteData
 0001:00033834       Classes.TWriter.WriteDate
 0001:0003377C       Classes.TWriter.WriteDescendent
 0001:000337EC       Classes.TWriter.WriteDouble
 0001:000337A4       Classes.TWriter.WriteFloat
 0001:00033858       Classes.TWriter.WriteIdent
 0001:000339B0       Classes.TWriter.WriteInteger
 0001:0003393C       Classes.TWriter.WriteInteger
 0001:00033A08       Classes.TWriter.WriteListBegin
 0001:00033A10       Classes.TWriter.WriteListEnd
 0001:00035214       Classes.TWriter.WriteMinStr
 0001:00033A18       Classes.TWriter.WritePrefix
 0001:00033A60       Classes.TWriter.WriteProperties
 0001:00034BB8       Classes.TWriter.WriteProperty
 0001:000350EC       Classes.TWriter.WritePropName
 0001:00035140       Classes.TWriter.WriteRootComponent
 0001:00035148       Classes.TWriter.WriteSignature
 0001:000337C8       Classes.TWriter.WriteSingle
 0001:00035158       Classes.TWriter.WriteStr
 0001:00035348       Classes.TWriter.WriteString
 0001:00035460       Classes.TWriter.WriteUTF8Str
 0001:0003553C       Classes.TWriter.WriteValue
 0001:00034D0C       Classes.TWriter.WriteVariant
 0001:00033128       Classes.TWriter.WriteWideChar
 0001:00035534       Classes.TWriter.WriteWideString
 0001:0002A88C       Classes.UnRegisterModuleClasses
 0001:00035658       Classes.WaitForSyncEvent
 0003:00000F68       Classes.WakeMainThread
 0001:0002AA50       Classes.WriteCollection
 0001:000343E8       Classes.WriteCollectionProp
 0001:00034584       Classes.WriteFloatProp
 0001:000345C4       Classes.WriteInt64Prop
 0001:000349E8       Classes.WriteInterfaceProp
 0001:0003437C       Classes.WriteIntProp
 0001:00034AC4       Classes.WriteMethodProp
 0001:000347D4       Classes.WriteObjectProp
 0001:0003448C       Classes.WriteOrdProp
 0001:00034290       Classes.WritePropPath
 0001:000342E8       Classes.WriteSet
 0001:00034600       Classes.WriteStrProp
 0001:00034B54       Classes.WriteVariantProp
 0001:000471F4       Contnrs..TObjectList
 0001:00047660       Contnrs.TObjectList.Add
 0001:000476A4       Contnrs.TObjectList.Create
 0001:00047668       Contnrs.TObjectList.Create
 0001:000476E8       Contnrs.TObjectList.Extract
 0001:000476FC       Contnrs.TObjectList.ExtractItem
 0001:00047714       Contnrs.TObjectList.FindInstanceOf
 0001:0004779C       Contnrs.TObjectList.First
 0001:000477AC       Contnrs.TObjectList.GetItem
 0001:000477C0       Contnrs.TObjectList.IndexOf
 0001:000477C8       Contnrs.TObjectList.IndexOfItem
 0001:000477D0       Contnrs.TObjectList.Insert
 0001:000477D8       Contnrs.TObjectList.Last
 0001:000477E4       Contnrs.TObjectList.Notify
 0001:00047810       Contnrs.TObjectList.Remove
 0001:00047818       Contnrs.TObjectList.RemoveItem
 0004:00005168       IniFiles..7
 0001:00044100       IniFiles.Finalization
 0002:000007AC       IniFiles.IniFiles
 0003:00000FFC       IniFiles.TCustomIniFile.SectionNameSeparator
 0003:00001000       IniFiles.Values
 0004:00005164       IOUtils..1
 0001:00044038       IOUtils.Finalization
 0002:000007A4       IOUtils.IOUtils
 0004:00005160       IOUtils.TPath.$ClassInitFlag
 0002:0000034C       IOUtils.TPath.Create@
 0001:00044030       IOUtils.TPath.Destroy@
 0004:00005144       IOUtils.TPath.FAltDirectorySeparatorChar
 0003:00000FEC       IOUtils.TPath.FCCurrentDir
 0003:00000FF4       IOUtils.TPath.FCExtendedPrefix
 0003:00000FF8       IOUtils.TPath.FCExtendedUNCPrefix
 0003:00000FF0       IOUtils.TPath.FCParentDir
 0004:00005146       IOUtils.TPath.FDirectorySeparatorChar
 0004:0000514C       IOUtils.TPath.FExtensionSeparatorChar
 0004:0000515C       IOUtils.TPath.FFileNameWildCardChars
 0004:00005154       IOUtils.TPath.FInvalidFileNameChars
 0004:00005150       IOUtils.TPath.FInvalidPathChars
 0004:00005148       IOUtils.TPath.FPathSeparator
 0004:00005158       IOUtils.TPath.FPathWildcardChars
 0004:0000514A       IOUtils.TPath.FVolumeSeparatorChar
 0004:0000516C       Registry..5
 0001:00044150       Registry..ERegistryException
 0001:00044344       Registry..TRegistry
 0001:000453F8       Registry.BinaryToHexString
 0001:00046E28       Registry.CopyKeys
 0001:00046CF0       Registry.CopyValues
 0001:000453D0       Registry.DataTypeToRegData
 0001:00047198       Registry.Finalization
 0001:0004532C       Registry.IsRelative
 0003:00001008       Registry.KeyNames
 0001:00046BD0       Registry.MoveValue
 0001:00045300       Registry.ReadError
 0001:000453A0       Registry.RegDataToDataType
 0002:000007B4       Registry.Registry
 0001:0004565C       Registry.TRegistry.ChangeKey
 0001:000455F4       Registry.TRegistry.CheckResult
 0001:00045600       Registry.TRegistry.CloseKey
 0001:0004558C       Registry.TRegistry.Create
 0001:00045548       Registry.TRegistry.Create
 0001:00045698       Registry.TRegistry.CreateKey
 0001:00045A94       Registry.TRegistry.DeleteKey
 0001:00045C20       Registry.TRegistry.DeleteValue
 0001:000455C8       Registry.TRegistry.Destroy
 0001:00045680       Registry.TRegistry.GetBaseKey
 0001:00046690       Registry.TRegistry.GetData
 0001:0004625C       Registry.TRegistry.GetDataAsString
 0001:00045FEC       Registry.TRegistry.GetDataInfo
 0001:00046040       Registry.TRegistry.GetDataSize
 0001:00046068       Registry.TRegistry.GetDataType
 0001:00046740       Registry.TRegistry.GetKey
 0001:00045C44       Registry.TRegistry.GetKeyInfo
 0001:00045CB0       Registry.TRegistry.GetKeyNames
 0001:00045D78       Registry.TRegistry.GetLastErrorMsg
 0001:00045EEC       Registry.TRegistry.GetRootKeyName
 0001:00045F24       Registry.TRegistry.GetValueNames
 0001:0004670C       Registry.TRegistry.HasSubKeys
 0001:00046ABC       Registry.TRegistry.KeyExists
 0001:00046814       Registry.TRegistry.LoadKey
 0001:00047084       Registry.TRegistry.MoveKey
 0001:00045778       Registry.TRegistry.OpenKey
 0001:000458AC       Registry.TRegistry.OpenKeyReadOnly
 0001:0004661C       Registry.TRegistry.PutData
 0001:000465B8       Registry.TRegistry.ReadBinaryData
 0001:00046464       Registry.TRegistry.ReadBool
 0001:000464D8       Registry.TRegistry.ReadCurrency
 0001:00046568       Registry.TRegistry.ReadDate
 0001:00046520       Registry.TRegistry.ReadDateTime
 0001:00046490       Registry.TRegistry.ReadFloat
 0001:00046428       Registry.TRegistry.ReadInteger
 0001:000461A8       Registry.TRegistry.ReadString
 0001:00046590       Registry.TRegistry.ReadTime
 0001:000467D8       Registry.TRegistry.RegistryConnect
 0001:00046B34       Registry.TRegistry.RenameValue
 0001:000469A0       Registry.TRegistry.ReplaceKey
 0001:00046928       Registry.TRegistry.RestoreKey
 0001:00046A44       Registry.TRegistry.SaveKey
 0001:00045694       Registry.TRegistry.SetCurrentKey
 0001:00045630       Registry.TRegistry.SetRootKey
 0001:000468A4       Registry.TRegistry.UnLoadKey
 0001:00046730       Registry.TRegistry.ValueExists
 0001:000465A4       Registry.TRegistry.WriteBinaryData
 0001:00046458       Registry.TRegistry.WriteBool
 0001:000464C4       Registry.TRegistry.WriteCurrency
 0001:00046554       Registry.TRegistry.WriteDate
 0001:0004650C       Registry.TRegistry.WriteDateTime
 0001:0004611C       Registry.TRegistry.WriteExpandString
 0001:0004647C       Registry.TRegistry.WriteFloat
 0001:00046414       Registry.TRegistry.WriteInteger
 0001:00046090       Registry.TRegistry.WriteString
 0001:0004657C       Registry.TRegistry.WriteTime
 0003:00001024       Registry.Values
 0004:00004FA0       Rtti..23
 0001:000383E0       Rtti.Finalization
 0003:00000FBC       Rtti.Kind
 0004:00004FA4       Rtti.ModListRemovals
 0001:00038390       Rtti.OnUnloadModule
 0004:00004FAC       Rtti.PoolLock
 0002:000002EC       Rtti.Rtti
 0004:00004FA8       Rtti.StringEqCmpCI
 0001:00009AE0       StrUtils.PosEx
 0004:00004F8C       SyncObjs..01
 0001:00037BC0       SyncObjs..TCriticalSection
 0001:00037ABC       SyncObjs..TSynchroObject
 0001:00038388       SyncObjs.Finalization
 0001:0003821C       SyncObjs.InitConditionVariableProcs
 0004:00004F90       SyncObjs.InitializeConditionVariableProc
 0001:00037E7C       SyncObjs.InternalInitConditionVariable
 0001:00037EAC       SyncObjs.InternalSleepConditionVariableCS
 0001:00037E9C       SyncObjs.InternalWakeAllConditionVariable
 0001:00037E8C       SyncObjs.InternalWakeConditionVariable
 0004:00004F94       SyncObjs.SleepConditionVariableCSProc
 0002:000002DC       SyncObjs.SyncObjs
 0001:00037E40       SyncObjs.TCriticalSection.Acquire
 0001:00037DD0       SyncObjs.TCriticalSection.Create
 0001:00037E10       SyncObjs.TCriticalSection.Destroy
 0001:00037E6C       SyncObjs.TCriticalSection.Enter
 0001:00037E74       SyncObjs.TCriticalSection.Leave
 0001:00037E4C       SyncObjs.TCriticalSection.Release
 0001:00037E58       SyncObjs.TCriticalSection.TryEnter
 0001:00037EC8       SyncObjs.TInternalConditionVariable.DequeueWaiter
 0001:00037F20       SyncObjs.TInternalConditionVariable.DequeueWaiterNoLock
 0001:00037F3C       SyncObjs.TInternalConditionVariable.LockQueue
 0001:00037FA0       SyncObjs.TInternalConditionVariable.QueueWaiter
 0001:00038008       SyncObjs.TInternalConditionVariable.RemoveWaiter
 0001:00038094       SyncObjs.TInternalConditionVariable.SleepCriticalSection
 0001:0003818C       SyncObjs.TInternalConditionVariable.UnlockQueue
 0001:00038194       SyncObjs.TInternalConditionVariable.Wake
 0001:000381A8       SyncObjs.TInternalConditionVariable.WakeAll
 0001:00037DC8       SyncObjs.TSynchroObject.Acquire
 0001:00037DCC       SyncObjs.TSynchroObject.Release
 0004:00004F9C       SyncObjs.WakeAllConditionVariableProc
 0004:00004F98       SyncObjs.WakeConditionVariableProc
 0001:00008AF0       SysInit.@GetTls
 0001:00008B3C       SysInit.@InitExe
 0001:00008A98       SysInit.AllocTlsBuffer
 0001:00008A78       SysInit.GetModuleHandle
 0001:00008AA4       SysInit.GetTlsSize
 0004:00002C38       SysInit.HInstance
 0001:00008B30       SysInit.InitializeModule
 0001:00008AAC       SysInit.InitThreadTLS
 0001:00008A80       SysInit.LocalAlloc
 0003:000009F8       SysInit.Module
 0004:00002C35       SysInit.ModuleIsCpp
 0004:00002C34       SysInit.ModuleIsLib
 0003:000009F4       SysInit.PtrToNil
 0004:00002C3C       SysInit.tlsBuffer
 0001:00008A88       SysInit.TlsGetValue
 0003:000009F0       SysInit.TlsIndex
 0005:00000014       SysInit.TlsLast
 0001:00008A90       SysInit.TlsSetValue
 0003:000009E4       System...
 0001:00008628       System...
 0004:00002C1C       System...
 0004:000008D8       System..8
 0001:00000C74       System..TInterfacedObject
 0001:0000040C       System..TObject
 0001:00003474       System.@AbstractError
 0001:0000410C       System.@AfterConstruction
 0001:00004D6C       System.@Assert
 0001:0000353C       System.@AStrCmp
 0001:0000415C       System.@BeforeDestruction
 0001:00003A74       System.@BoundErr
 0001:00003E24       System.@CallDynaInst
 0001:000040B4       System.@ClassCreate
 0001:00004104       System.@ClassDestroy
 0001:000034E4       System.@Close
 0001:000064E8       System.@CopyArray
 0001:000063A8       System.@CopyRecord
 0001:00006624       System.@DispCallByIDError
 0001:00006614       System.@Dispose
 0001:0000471C       System.@DoneExcept
 0001:00006C00       System.@DynArrayAddRef
 0001:00006BD8       System.@DynArrayAsg
 0001:00006B9C       System.@DynArrayClear
 0001:000069D0       System.@DynArrayHigh
 0001:000069C8       System.@DynArrayLength
 0001:00006B90       System.@DynArraySetLength
 0001:00005000       System.@EnsureUnicodeString
 0001:00004804       System.@ExceptionHandler
 0001:000035AC       System.@FillChar
 0001:00006384       System.@Finalize
 0001:00006274       System.@FinalizeArray
 0001:00006224       System.@FinalizeRecord
 0001:00003A68       System.@FpuInit
 0001:000031AC       System.@FreeMem
 0001:00003190       System.@GetMem
 0001:00004D54       System.@Halt
 0001:00004C48       System.@Halt0
 0001:000042C4       System.@HandleAnyException
 0001:00004578       System.@HandleFinally
 0001:00004620       System.@HandleFinallyInternal
 0001:000043F0       System.@HandleOnException
 0001:000089DC       System.@InitDelayHelp
 0001:00006218       System.@Initialize
 0001:00006180       System.@InitializeArray
 0001:0000614C       System.@InitializeRecord
 0001:00004B04       System.@InitImports
 0001:00004AC0       System.@InitResStringImports
 0001:00005020       System.@InternalLStrFromUStr
 0001:00004FF0       System.@InternalUStrFromLStr
 0001:00008040       System.@IntfAddRef
 0001:00008010       System.@IntfCast
 0001:00007FCC       System.@IntfClear
 0001:00007FE4       System.@IntfCopy
 0001:00003A7C       System.@IntOver
 0001:00003DD0       System.@IsClass
 0001:0000519C       System.@LStrAddRef
 0001:00004E64       System.@LStrArrayClr
 0001:00004E94       System.@LStrAsg
 0001:00004E40       System.@LStrClr
 0001:000050B4       System.@LStrFromPChar
 0001:00004F3C       System.@LStrFromPCharLen
 0001:000050E8       System.@LStrFromPWChar
 0001:00005030       System.@LStrFromPWCharLen
 0001:00005128       System.@LStrFromString
 0001:00005840       System.@LStrFromUStr
 0001:00005138       System.@LStrFromWStr
 0001:0000522C       System.@LStrSetLength
 0001:000051AC       System.@LStrToPChar
 0001:00005150       System.@LStrToString
 0001:00008600       System.@memcpy
 0001:00008614       System.@memset
 0001:00006600       System.@New
 0001:00004EF0       System.@NewAnsiString
 0001:00005ED0       System.@NewUnicodeString
 0001:000052CC       System.@NewWideString
 0001:00005174       System.@PCharLen
 0001:00003784       System.@Pow10
 0001:000046C8       System.@RaiseAgain
 0001:00004658       System.@RaiseExcept
 0001:000031C4       System.@ReallocMem
 0001:00003468       System.@ROUND
 0001:00004D60       System.@RunError
 0001:0000374C       System.@SetElem
 0001:00003770       System.@SetUnion
 0001:000089EB       System.@ShutdownDelayHelp
 0001:000049C0       System.@StartExe
 0001:000014D4       System.@strlen
 0001:0000474C       System.@TryFinallyExit
 0001:00005224       System.@UniqueStringA
 0001:000055FC       System.@UStrAddRef
 0001:0000560C       System.@UStrArrayClr
 0001:00005614       System.@UStrAsg
 0001:00005A04       System.@UStrCat
 0001:00005AC4       System.@UStrCat3
 0001:00005BA8       System.@UStrCatN
 0001:00005604       System.@UStrClr
 0001:00005D30       System.@UStrCopy
 0001:00005E00       System.@UStrDelete
 0001:00005CC8       System.@UStrEqual
 0001:00005818       System.@UStrFromLStr
 0001:00005790       System.@UStrFromPChar
 0001:00005740       System.@UStrFromPCharLen
 0001:000057C0       System.@UStrFromPWChar
 0001:00005750       System.@UStrFromPWCharLen
 0001:000057FC       System.@UStrFromWArray
 0001:00005780       System.@UStrFromWChar
 0001:00005864       System.@UStrFromWStr
 0001:00005668       System.@UStrLAsg
 0001:00005960       System.@UStrLen
 0001:0000596C       System.@UStrSetLength
 0001:000056A0       System.@UStrToPWChar
 0001:000058A0       System.@UStrToString
 0001:00006650       System.@ValInt64
 0001:00003648       System.@ValLong
 0001:0000625C       System.@VarClr
 0001:00006390       System.@VarCopy
 0001:0000530C       System.@WStrArrayClr
 0001:00005330       System.@WStrAsg
 0001:000052F4       System.@WStrClr
 0001:000054D0       System.@WStrCmp
 0001:0000555C       System.@WStrCopy
 0001:00005554       System.@WStrEqual
 0001:00005494       System.@WStrFromLStr
 0001:00005428       System.@WStrFromPChar
 0001:000053F4       System.@WStrFromPCharLen
 0001:00005458       System.@WStrFromPWChar
 0001:00005404       System.@WStrFromPWCharLen
 0001:00005878       System.@WStrFromUStr
 0001:000055A8       System.@WStrSetLength
 0001:000054C0       System.@WStrToPWChar
 0001:0000870E       System.@_delayLoadHelper
 0001:00008972       System.@_FUnloadDelayLoadedDLL
 0001:000032D8       System.@_IOTest
 0001:0000662C       System.@_llmul
 0003:000009E8       System.@__pfnDliFailureHook
 0003:000009EC       System.@__pfnDliNotifyHook
 0004:00000030       System.AbstractErrorProc
 0001:00003234       System.AcquireExceptionObject
 0001:00007E5C       System.AddModuleUnloadProc
 0001:00007E6C       System.AddModuleUnloadProc
 0001:00001A30       System.AllocateLargeBlock
 0001:00003178       System.AllocMem
 0001:00001970       System.AllocNewSequentialFeedMediumPool
 0004:000008DC       System.AllocSize2SmallBlockTypeIndX4
 0003:0000006C       System.AnsiStringBlockMessage
 0001:00002720       System.AppendClassNameToBuffer
 0001:00002708       System.AppendStringToBuffer
 0004:00000028       System.AssertErrorProc
 0001:00004DC4       System.BeginThread
 0001:00001904       System.BinMediumSequentialFeedRemainder
 0001:00002F28       System.BuildBlockTypeLookupTable
 0003:00000064       System.BytesMessage
 0004:00002B6C       System.CachedLangID
 0004:00002B70       System.CachedLanguageNames
 0001:000025EC       System.CardinalToStrBuf
 0001:00004FA0       System.CharFromWChar
 0001:00004F74       System.CharFromWChar
 0001:0000141C       System.CharNext
 0001:000072FC       System.CheckDifferentLanguageList
 0001:00004240       System.CheckJmp
 0001:00002984       System.CheckSmallBlockPoolForLeaks
 0001:000013CC       System.CloseHandle
 0004:00000044       System.CmdLine
 0004:00000040       System.CmdShow
 0001:0000142C       System.CompareString
 0001:00001424       System.CompareStringW
 0001:00007074       System.ConvertResToUILanguages
 0001:000069D8       System.CopyArray
 0003:00000054       System.Copyright
 0004:00000050       System.CPUCount
 0001:00001434       System.CreateThread
 0004:00002B54       System.CrSec
 0003:00000028       System.DebugHook
 0003:00000024       System.Default8087CW
 0004:000008C8       System.DefaultSystemCodePage
 0004:000008CC       System.DefaultUnicodeCodePage
 0001:00006C0C       System.DelayLoadResourceModule
 0001:000013EC       System.DeleteCriticalSection
 0004:00000000       System.DispCallByIDProc
 0004:00002B14       System.DLLThreadContext
 0001:000069F0       System.DynArrayClear
 0001:000069F8       System.DynArraySetLength
 0003:000007C8       System.EmptyStringW
 0001:00004E24       System.EndThread
 0001:00004FD8       System.EnsureAnsiString
 0001:00004FE8       System.EnsureUnicodeString
 0001:000013DC       System.EnterCriticalSection
 0001:00007E28       System.EnumResourceModules
 0001:00007E30       System.EnumResourceModules
 0003:00000790       System.errCaption
 0001:000032CC       System.Error
 0003:00000004       System.ErrorAddr
 0001:00003280       System.ErrorAt
 0004:00000008       System.ErrorProc
 0004:000005F4       System.ErrOutput
 0004:0000000C       System.ExceptClsProc
 0004:00000020       System.ExceptionAcquired
 0004:00000024       System.ExceptionClass
 0001:00003214       System.ExceptObject
 0004:00000010       System.ExceptObjProc
 0004:00000004       System.ExceptProc
 0003:00000000       System.ExitCode
 0001:00004B8C       System.ExitDll
 0004:00000048       System.ExitProc
 0001:00001444       System.ExitProcess
 0004:0000002C       System.ExitProcessProc
 0001:0000143C       System.ExitThread
 0004:00002AD8       System.ExpectedMemoryLeaks
 0004:00002ADC       System.ExpectedMemoryLeaksListLocked
 0003:0000000C       System.FileMode
 0001:00008A04       System.Finalization
 0001:000069E8       System.FinalizeArray
 0001:00006FA8       System.FinalizeLocaleDate
 0001:00003124       System.FinalizeMemoryManager
 0001:000048EC       System.FinalizeUnits
 0001:000075A8       System.FindBS
 0001:00001454       System.FindClose
 0001:00003DF4       System.FindDynaMethod
 0001:0000145C       System.FindFirstFile
 0001:00006C54       System.FindResourceHInstance
 0001:000034D8       System.Flush
 0001:0000377C       System.FPower10
 0001:00003094       System.FreeAllMemory
 0001:00001A94       System.FreeLargeBlock
 0001:00001464       System.FreeLibrary
 0001:00003460       System.Get8087CW
 0001:00008588       System.GetACP
 0001:0000154C       System.GetCmdShow
 0001:0000146C       System.GetCommandLine
 0001:00008590       System.GetCPUCount
 0001:00001524       System.GetCurrentThreadId
 0001:000025B0       System.GetFirstAndLastSmallBlockInPool
 0001:00002570       System.GetFirstMediumBlockInPool
 0001:00001474       System.GetLastError
 0001:0000147C       System.GetLocaleInfo
 0001:000077C8       System.GetLocaleOverride
 0001:0000148C       System.GetModuleFileName
 0001:00001494       System.GetModuleHandle
 0001:00002850       System.GetObjectClass
 0001:00007364       System.GetPreferredLangForNewOS
 0001:00007164       System.GetPreferredLangForOldOS
 0001:0000149C       System.GetProcAddress
 0001:00007C78       System.GetResourceModuleName
 0001:000014A4       System.GetStartupInfo
 0001:000013F4       System.GetStdHandle
 0001:000014AC       System.GetSystemDefaultUILanguage
 0001:00001544       System.GetSystemInfo
 0004:00002B44       System.GetThreadPreferredUILanguages
 0004:00002B4C       System.GetThreadUILanguage
 0001:0000153C       System.GetTickCount
 0001:00007484       System.GetUILanguages
 0001:00001484       System.GetUserDefaultUILanguage
 0001:0000152C       System.GetVersion
 0003:000009E0       System.hexdig
 0003:000007B8       System.hexDigits
 0004:00002AE4       System.InitContext
 0001:000013D4       System.InitializeCriticalSection
 0001:00006EB8       System.InitializeLocaleData
 0001:00002F6C       System.InitializeMemoryManager
 0001:00004954       System.InitUnits
 0005:00000004       System.InOutRes
 0004:00000054       System.Input
 0001:000018A4       System.InsertMediumBlockIntoBin
 0001:000013C0       System.InterlockedDecrement
 0001:000013B4       System.InterlockedIncrement
 0001:00003490       System.InternalFlush
 0001:000027D0       System.InternalIsValidClass
 0001:000051C4       System.InternalUniqueString
 0001:00005E74       System.InternalUniqueStringU
 0001:000056AC       System.InternalUStrFromPCharLen
 0001:00005358       System.InternalWStrFromPCharLen
 0001:00003C40       System.InvokeImplGetter
 0001:00003308       System.IOResult
 0004:0000004C       System.IsConsole
 0004:0000003C       System.IsLibrary
 0004:0000004D       System.IsMultiThread
 0001:000014B4       System.IsValidLocale
 0001:00002754       System.IsValidVMTAddress
 0003:0000002C       System.JITEnable
 0004:00002AC8       System.LargeBlocksCircularList
 0004:00002AC4       System.LargeBlocksLocked
 0003:00000060       System.LargeLeakDetail
 0001:00006FD4       System.LastHyphenPos
 0004:00000A38       System.LastSequentiallyFedMediumBlock
 0003:00000074       System.LeakMessageFooter
 0003:00000058       System.LeakMessageHeader
 0003:00000078       System.LeakMessageTitle
 0001:000013E4       System.LeaveCriticalSection
 0003:0000003C       System.LibModuleList
 0001:00007C1C       System.Load3LettersModule
 0001:00007B6C       System.LoadLanguageList
 0001:000085F0       System.LoadLibraryA
 0001:000014BC       System.LoadLibraryEx
 0001:00007A68       System.LoadResourceModule
 0001:0000851C       System.LoadResString
 0001:00004A08       System.LoadResStringA
 0001:00004AAC       System.LoadResStringU
 0001:00004A5C       System.LoadResStringW
 0001:000014C4       System.LoadString
 0001:000085E0       System.LocalAlloc
 0003:000007D8       System.LocaleTable
 0001:000085E8       System.LocalFree
 0001:000016D8       System.LockCmpxchg
 0001:00002878       System.LockExpectedMemoryLeaksList
 0001:000019E8       System.LockLargeBlocks
 0001:000085F8       System.lstrcmpiA
 0001:000014CC       System.lstrcpyn
 0004:00000034       System.MainInstance
 0004:00000038       System.MainThreadID
 0001:00004B28       System.MakeErrorMessage
 0004:00002AE0       System.MappingObjectHandle
 0001:00004764       System.MapToRunError
 0004:00000A44       System.MediumBlockBinBitmaps
 0004:00000A40       System.MediumBlockBinGroupBitmap
 0004:00000AC4       System.MediumBlockBins
 0004:00000A24       System.MediumBlockPoolsCircularList
 0004:00000A34       System.MediumBlocksLocked
 0004:00000A3C       System.MediumSequentialFeedBytesLeft
 0003:0000075C       System.MemoryManager
 0001:0000144C       System.MessageBoxA
 0004:00000A22       System.MinimumBlockAlignment
 0003:00000040       System.ModuleUnloadList
 0004:000008C4       System.MonitorSupport
 0001:00003328       System.Move
 0001:000016E0       System.Move12
 0001:000016F4       System.Move20
 0001:00001714       System.Move28
 0001:00001740       System.Move36
 0001:00001760       System.Move44
 0001:00001784       System.Move52
 0001:000017B0       System.Move60
 0001:000017E0       System.Move68
 0001:00001818       System.MoveX16L4
 0001:00001848       System.MoveX8L4
 0001:000014DC       System.MultiByteToWideChar
 0004:000008D5       System.NeverSleepOnMMThreadContention
 0001:0000254C       System.NextMediumBlock
 0003:00000030       System.NoErrMsg
 0001:0000422C       System.NotifyAnyExcept
 0001:00004200       System.NotifyExcept
 0001:00004260       System.NotifyExceptFinally
 0001:00007EF0       System.NotifyModuleUnload
 0001:000041DC       System.NotifyNonDelphiException
 0001:00004218       System.NotifyOnExcept
 0001:000041C0       System.NotifyReRaise
 0001:00004288       System.NotifyTerminate
 0001:000042A4       System.NotifyUnhandled
 0003:00000044       System.ObjCastGUID
 0004:00000324       System.Output
 0001:00005F14       System.Pos
 0001:00001534       System.QueryPerformanceCounter
 0001:000013FC       System.RaiseException
 0004:00000014       System.RaiseExceptionProc
 0004:0000001C       System.RaiseExceptObjProc
 0001:00003268       System.RaiseList
 0005:00000000       System.RaiseListPtr
 0001:00003428       System.Randomize
 0003:00000008       System.RandSeed
 0001:00001B38       System.ReallocateLargeBlock
 0001:000014E4       System.RegCloseKey
 0001:00007F4C       System.RegisterModule
 0001:000014EC       System.RegOpenKeyEx
 0001:000014F4       System.RegQueryValueEx
 0003:00000774       System.reMap
 0001:00001864       System.RemoveMediumFreeBlock
 0001:00007E64       System.RemoveModuleUnloadProc
 0001:00007E8C       System.RemoveModuleUnloadProc
 0004:000008D4       System.ReportMemoryLeaksOnShutdown
 0001:00007B34       System.ResouceDLLExists
 0001:00001404       System.RtlUnwind
 0004:00000018       System.RTLUnwindProc
 0003:00000798       System.runErrMsg
 0001:00003274       System.RunErrorAt
 0001:00002B44       System.ScanForMemoryLeaks
 0001:00003450       System.Set8087CW
 0001:00005F60       System.SetCodePage
 0001:000048A4       System.SetExceptionHandler
 0001:000032F8       System.SetInOutRes
 0004:00002B48       System.SetThreadPreferredUILanguages
 0001:000085A4       System.SetUtf8CompareLocale
 0001:00001588       System.Sleep
 0003:0000007C       System.SmallBlockTypes
 0003:0000005C       System.SmallLeakDetail
 0001:00002518       System.SysAllocMem
 0001:0000150C       System.SysAllocStringLen
 0001:00002008       System.SysFreeMem
 0001:0000151C       System.SysFreeString
 0001:00001C84       System.SysGetMem
 0001:00002200       System.SysReallocMem
 0001:00001514       System.SysReAllocStringLen
 0001:000028EC       System.SysRegisterExpectedMemoryLeak
 0002:00000000       System.System
 0003:00000038       System.SystemThreadEndProc
 0003:00000034       System.SystemThreadFuncProc
 0001:0000292C       System.SysUnregisterExpectedMemoryLeak
 0004:0000004E       System.Test8086
 0001:00007320       System.ThreadUILanguages
 0001:00004D8C       System.ThreadWrapper
 0001:0000804C       System.TInterfacedObject.AfterConstruction
 0001:00008058       System.TInterfacedObject.BeforeDestruction
 0001:00008068       System.TInterfacedObject.NewInstance
 0001:00008078       System.TInterfacedObject.QueryInterface
 0001:000080A0       System.TInterfacedObject._AddRef
 0001:000080B4       System.TInterfacedObject._Release
 0001:00004184       System.TMonitor.Destroy
 0001:0000416C       System.TMonitor.Destroy
 0001:000041B0       System.TMonitor.GetFieldAddress
 0001:00003E78       System.TObject.AfterConstruction
 0001:00003E7C       System.TObject.BeforeDestruction
 0001:00003E50       System.TObject.ClassInfo
 0001:00003A8C       System.TObject.ClassName
 0001:00003AA4       System.TObject.ClassNameIs
 0001:00003B40       System.TObject.ClassParent
 0001:00003A84       System.TObject.ClassType
 0001:00003C18       System.TObject.CleanupInstance
 0001:00003B84       System.TObject.Create
 0001:00003E74       System.TObject.DefaultHandler
 0001:00003BA4       System.TObject.Destroy
 0001:00003E80       System.TObject.Dispatch
 0001:00003C70       System.TObject.Equals
 0001:0000408C       System.TObject.FieldAddress
 0001:00004018       System.TObject.FieldAddress
 0001:00003BB4       System.TObject.Free
 0001:00003B68       System.TObject.FreeInstance
 0001:00003C78       System.TObject.GetHashCode
 0001:00003C7C       System.TObject.GetInterface
 0001:00003D4C       System.TObject.GetInterfaceEntry
 0001:00003D90       System.TObject.GetInterfaceTable
 0001:00003E3C       System.TObject.InheritsFrom
 0001:00003BC0       System.TObject.InitInstance
 0001:00003B7C       System.TObject.InstanceSize
 0001:00003F34       System.TObject.MethodAddress
 0001:00003FA4       System.TObject.MethodAddress
 0001:00003FCC       System.TObject.MethodName
 0001:00003B4C       System.TObject.NewInstance
 0001:00003E58       System.TObject.SafeCallException
 0001:00003E60       System.TObject.ToString
 0001:00003D98       System.TObject.UnitName
 0001:000075CC       System.ToLongPath
 0001:0000140C       System.UnhandledExceptionFilter
 0003:00000070       System.UnicodeStringBlockMessage
 0001:000080DC       System.UnicodeToUtf8
 0001:0000521C       System.UniqueString
 0001:00005EC8       System.UniqueString
 0003:00000068       System.UnknownClassNameMsg
 0001:00007F5C       System.UnregisterModule
 0001:000048C4       System.UnsetExceptionHandler
 0004:00002B50       System.UseThreadUILanguageAPI
 0001:00003EA8       System.UTF8Compare
 0004:000008D0       System.UTF8CompareLocale
 0001:000081F0       System.UTF8Encode
 0001:00008310       System.UTF8EncodeToShortString
 0001:00003F20       System.UTF8ShortStringToString
 0001:00008508       System.UTF8ToString
 0001:0000816C       System.Utf8ToUnicode
 0001:0000839C       System.UTF8ToUnicodeString
 0001:00008474       System.UTF8ToUnicodeString
 0003:00000014       System.VarAddRefProc
 0003:00000010       System.VarClearProc
 0003:00000018       System.VarCopyProc
 0003:0000001C       System.VarToLStrProc
 0003:00000020       System.VarToWStrProc
 0001:00001578       System.VirtualAlloc
 0001:00001580       System.VirtualFree
 0001:00001504       System.VirtualQuery
 0001:00004FBC       System.WCharFromChar
 0001:000014FC       System.WideCharToMultiByte
 0001:00004BB8       System.WriteErrorMessage
 0001:00001414       System.WriteFile
 0001:000052C4       System.WStrError
 0001:000052E4       System.WStrSet
 0004:00002DA4       SysUtils..76
 0001:0000B260       SysUtils..EAbstractError
 0001:0000AEB0       SysUtils..EAccessViolation
 0001:0000B1BC       SysUtils..EAssertionFailed
 0001:0000B08C       SysUtils..EControlC
 0001:0000AE14       SysUtils..EConvertError
 0001:0000A818       SysUtils..EDivByZero
 0001:0000BD04       SysUtils..EEncodingError
 0001:0000A624       SysUtils..EExternal
 0001:0000A6DC       SysUtils..EExternalException
 0001:0000A3DC       SysUtils..EHeapException
 0001:0000A56C       SysUtils..EInOutError
 0001:0000A784       SysUtils..EIntError
 0001:0000B300       SysUtils..EIntfCastError
 0001:0000A948       SysUtils..EIntOverflow
 0001:0000AD78       SysUtils..EInvalidCast
 0001:0000AA7C       SysUtils..EInvalidOp
 0001:0000ACD8       SysUtils..EInvalidPointer
 0001:0000A9E4       SysUtils..EMathError
 0001:0000B4F8       SysUtils..EMonitor
 0001:0000B58C       SysUtils..EMonitorLockException
 0001:0000B638       SysUtils..ENoMonitorSupportException
 0001:0000B3A0       SysUtils..EOSError
 0001:0000A4D0       SysUtils..EOutOfMemory
 0001:0000ABAC       SysUtils..EOverflow
 0001:0000AF54       SysUtils..EPrivilege
 0001:0000A8B0       SysUtils..ERangeError
 0001:0000B450       SysUtils..ESafecallException
 0001:0000AFEC       SysUtils..EStackOverflow
 0001:0000AC40       SysUtils..EUnderflow
 0001:0000B120       SysUtils..EVariantError
 0001:00009E14       SysUtils..Exception
 0001:0000AB14       SysUtils..EZeroDivide
 0001:0000CEF0       SysUtils..TBigEndianUnicodeEncoding
 0001:0000BDA4       SysUtils..TEncoding
 0001:0000C72C       SysUtils..TMBCSEncoding
 0001:0000B9FC       SysUtils..TMultiReadExclusiveWriteSynchronizer
 0001:0000B7D8       SysUtils..TThreadLocalCounter
 0001:0000CD30       SysUtils..TUnicodeEncoding
 0001:0000C9F0       SysUtils..TUTF7Encoding
 0001:0000CB70       SysUtils..TUTF8Encoding
 0001:00012D2C       SysUtils.AbstractErrorHandler
 0003:00000BA4       SysUtils.AccessMode
 0001:0000D4E8       SysUtils.AnsiCompareStr
 0001:0000D5B4       SysUtils.AnsiCompareText
 0001:0000D8E0       SysUtils.AnsiExtractQuotedStr
 0001:00013CC0       SysUtils.AnsiPos
 0001:0000D740       SysUtils.AnsiQuotedStr
 0001:00013DA0       SysUtils.AnsiStrPos
 0001:00013DA8       SysUtils.AnsiStrRScan
 0001:00013DB0       SysUtils.AnsiStrScan
 0001:0000D458       SysUtils.AnsiUpperCase
 0001:0000FEBC       SysUtils.AppendChars
 0001:00010324       SysUtils.AppendFormat
 0001:0000FF74       SysUtils.AppendNumber
 0001:0000FF00       SysUtils.AppendString
 0001:00012D10       SysUtils.AssertErrorHandler
 0001:0000E738       SysUtils.BackfillGetDiskFreeSpaceEx
 0001:0000E0FC       SysUtils.BoolToStr
 0001:000136F8       SysUtils.ByteToCharIndex
 0001:00013610       SysUtils.ByteToCharLen
 0001:0001345C       SysUtils.ByteType
 0001:00013A80       SysUtils.CharLength
 0001:00013900       SysUtils.CharToByteIndex
 0001:00013A18       SysUtils.CharToByteLen
 0001:00013820       SysUtils.CharToElementIndex
 0001:00013908       SysUtils.CharToElementLen
 0001:00013388       SysUtils.CleanEventList
 0001:00013358       SysUtils.CleanStack
 0001:00014E00       SysUtils.ClearHashTables
 0001:0000D2A4       SysUtils.CompareMem
 0001:0000D1E4       SysUtils.CompareStr
 0001:0000D338       SysUtils.CompareText
 0001:0000E004       SysUtils.CompareWith
 0001:00014FE0       SysUtils.ContainsPreamble
 0001:00011FA4       SysUtils.ConvertAddr
 0001:0001006C       SysUtils.ConvertEraString
 0001:0000D018       SysUtils.ConvertError
 0001:0000D030       SysUtils.ConvertErrorFmt
 0001:000101F8       SysUtils.ConvertYearString
 0001:00013700       SysUtils.CountChars
 0001:00012C54       SysUtils.CreateAssertException
 0001:00012DE4       SysUtils.CreateAVObject
 0001:000129FC       SysUtils.CreateInOutError
 0003:00000B9C       SysUtils.cSimpleBoolStrs
 0004:00002C7E       SysUtils.CurrencyDecimals
 0004:00002C78       SysUtils.CurrencyFormat
 0004:00002C74       SysUtils.CurrencyString
 0001:0000FEA8       SysUtils.CurrentYear
 0001:0000F894       SysUtils.CurrToStr
 0001:0000DBC8       SysUtils.CvtInt
 0001:0000DDB4       SysUtils.CvtInt64
 0001:0000DCD0       SysUtils.CvtInt64W
 0001:0000DC14       SysUtils.CvtIntW
 0003:00000BF0       SysUtils.CWNear
 0004:00002C80       SysUtils.DateSeparator
 0001:00010B18       SysUtils.DateTimeToString
 0001:0000FDD0       SysUtils.DateTimeToSystemTime
 0001:0000F9DC       SysUtils.DateTimeToTimeStamp
 0001:0000FE80       SysUtils.DayOfWeek
 0003:00000BEC       SysUtils.DCon10
 0004:00002C7C       SysUtils.DecimalSeparator
 0001:0000FDB0       SysUtils.DecodeDate
 0001:0000FC64       SysUtils.DecodeDateFully
 0001:0000FAD0       SysUtils.DecodeTime
 0003:00000DF8       SysUtils.DefaultFallbackLanguages
 0003:00000C80       SysUtils.DefLongDayNames
 0003:00000C34       SysUtils.DefLongMonthNames
 0003:00000C64       SysUtils.DefShortDayNames
 0003:00000C04       SysUtils.DefShortMonthNames
 0001:0000E39C       SysUtils.DirectoryExists
 0001:0000CFFC       SysUtils.DivMod
 0001:0001314C       SysUtils.DoneExceptions
 0001:000133B4       SysUtils.DoneMonitorSupport
 0001:000129A0       SysUtils.EHeapException.FreeInstance
 0001:000129AC       SysUtils.EHeapException.RaisingException
 0001:00013618       SysUtils.ElementToCharIndex
 0001:0001356C       SysUtils.ElementToCharLen
 0003:00000B28       SysUtils.EmptyAnsiStr
 0003:00000B20       SysUtils.EmptyStr
 0003:00000B24       SysUtils.EmptyWideStr
 0001:0000FC34       SysUtils.EncodeDate
 0001:0000FA90       SysUtils.EncodeTime
 0001:00011B7C       SysUtils.EnumEraNames
 0001:00011BB8       SysUtils.EnumEraYearOffsets
 0001:0000E190       SysUtils.EnumStringModules
 0004:00002D48       SysUtils.EraNames
 0001:00010FE4       SysUtils.EraToYear
 0004:00002D64       SysUtils.EraYearOffsets
 0001:00012BFC       SysUtils.ErrorHandler
 0003:00000C9C       SysUtils.ErrorMap
 0004:00002EB0       SysUtils.EventCache
 0004:00002EB4       SysUtils.EventItemHolders
 0001:000130AC       SysUtils.ExceptHandler
 0004:00002C64       SysUtils.Exception.$ClassInitFlag
 0004:00002C70       SysUtils.Exception.CleanUpStackInfoProc
 0001:000122E4       SysUtils.Exception.Create
 0002:000000CC       SysUtils.Exception.Create@
 0001:00012320       SysUtils.Exception.CreateFmt
 0001:000125C4       SysUtils.Exception.CreateFmtHelp
 0001:0001257C       SysUtils.Exception.CreateHelp
 0001:00012418       SysUtils.Exception.CreateRes
 0001:000123A0       SysUtils.Exception.CreateRes
 0001:000124E8       SysUtils.Exception.CreateResFmt
 0001:00012454       SysUtils.Exception.CreateResFmt
 0001:000127B0       SysUtils.Exception.CreateResFmtHelp
 0001:00012714       SysUtils.Exception.CreateResFmtHelp
 0001:0001264C       SysUtils.Exception.CreateResHelp
 0001:000126CC       SysUtils.Exception.CreateResHelp
 0001:0001284C       SysUtils.Exception.Destroy
 0001:000131CC       SysUtils.Exception.Destroy@
 0001:00012890       SysUtils.Exception.GetBaseException
 0004:00002C68       SysUtils.Exception.GetExceptionStackInfoProc
 0004:00002C6C       SysUtils.Exception.GetStackInfoStringProc
 0001:0001289C       SysUtils.Exception.GetStackTrace
 0001:000128C8       SysUtils.Exception.RaiseOuterException
 0001:000128F0       SysUtils.Exception.RaisingException
 0001:0001291C       SysUtils.Exception.SetInnerException
 0001:00012944       SysUtils.Exception.SetStackInfo
 0001:000128DC       SysUtils.Exception.ThrowOuterException
 0001:00012948       SysUtils.Exception.ToString
 0001:00011FB0       SysUtils.ExceptionErrorMessage
 0003:00000D20       SysUtils.ExceptMap
 0003:00000CD4       SysUtils.ExceptTypes
 0001:0000E6A4       SysUtils.ExpandFileName
 0001:0000E5F0       SysUtils.ExtractFileExt
 0001:0000E5B0       SysUtils.ExtractFileName
 0004:00002D84       SysUtils.FalseBoolStrs
 0003:00000BE0       SysUtils.FCon1E18
 0001:0000E2B0       SysUtils.FileCreate
 0001:0000E258       SysUtils.FileOpen
 0001:0000E2F4       SysUtils.FileRead
 0001:0000E34C       SysUtils.FileSeek
 0001:0000E320       SysUtils.FileWrite
 0001:00016408       SysUtils.Finalization
 0001:0000E4B8       SysUtils.FindClose
 0001:0000E444       SysUtils.FindFirst
 0001:0000E3C0       SysUtils.FindMatchingFile
 0001:0000E494       SysUtils.FindNext
 0001:0000E1CC       SysUtils.FindStringResource
 0001:0000F4C0       SysUtils.FloatToDecimal
 0001:0000F864       SysUtils.FloatToStr
 0001:0000F1C0       SysUtils.FloatToText
 0003:00000BF4       SysUtils.FMSecsPerDay
 0001:0000EB20       SysUtils.FmtStr
 0001:0000EB0C       SysUtils.Format
 0003:00000BFC       SysUtils.Format
 0001:0000EAAC       SysUtils.FormatBuf
 0001:0000EA64       SysUtils.FormatError
 0003:00000BD8       SysUtils.FormatErrorStrs
 0001:00014D34       SysUtils.FreeAndNil
 0001:00013280       SysUtils.FreeSyncObj
 0001:00014850       SysUtils.FreeTerminateProcs
 0001:000132E8       SysUtils.FreeWaitObj
 0001:0000FFC0       SysUtils.GetCount
 0001:0000FFF4       SysUtils.GetDate
 0001:00010E34       SysUtils.GetDateOrder
 0003:00000B98       SysUtils.GetDiskFreeSpaceEx
 0001:00011C30       SysUtils.GetEraNamesAndYearOffsets
 0001:00010F90       SysUtils.GetEraYearOffset
 0001:00012DC4       SysUtils.GetExceptionClass
 0001:00012FB0       SysUtils.GetExceptionObject
 0001:00013ECC       SysUtils.GetFormatSettings
 0001:000119EC       SysUtils.GetLocaleChar
 0001:000119A0       SysUtils.GetLocaleStr
 0001:00011A58       SysUtils.GetMonthDayNames
 0001:0001002C       SysUtils.GetTime
 0001:00014644       SysUtils.HashName
 0001:000145B0       SysUtils.HashNameMBCS
 0003:00000B94       SysUtils.HexDisplayPrefix
 0003:00000BF8       SysUtils.IMSecsPerDay
 0001:00013C70       SysUtils.IncludeTrailingPathDelimiter
 0001:00014874       SysUtils.InitDriveSpacePtr
 0001:000130BC       SysUtils.InitExceptions
 0001:00013DB8       SysUtils.InitLeadBytes
 0001:0001334C       SysUtils.InitMonitorSupport
 0001:000133EC       SysUtils.InitPlatformId
 0001:00013E14       SysUtils.InitSysLocale
 0001:000148FC       SysUtils.InterlockedDecrement
 0001:00014908       SysUtils.InterlockedExchange
 0001:00014910       SysUtils.InterlockedExchangeAdd
 0001:000148F0       SysUtils.InterlockedIncrement
 0001:0000DEA8       SysUtils.IntToHex
 0001:0000DC74       SysUtils.IntToStr
 0001:0000DE80       SysUtils.IntToStr
 0004:00002DAC       SysUtils.InvalidPointer
 0001:0000FB2C       SysUtils.IsLeapYear
 0001:00013BB0       SysUtils.IsPathDelimiter
 0001:0000DA1C       SysUtils.IsValidIdent
 0004:00004EA0       SysUtils.LanguageArray
 0001:0000E4D4       SysUtils.LastDelimiter
 0003:00000B74       SysUtils.LeadBytes
 0004:00002D46       SysUtils.ListSeparator
 0001:0000E244       SysUtils.LoadStr
 0001:00011A18       SysUtils.LocalGetLocaleStr
 0004:00002C88       SysUtils.LongDateFormat
 0004:00002D1C       SysUtils.LongDayNames
 0004:00002CD0       SysUtils.LongMonthNames
 0004:00002C9C       SysUtils.LongTimeFormat
 0001:0000D16C       SysUtils.LowerCase
 0001:0000D11C       SysUtils.LowerCaseFromAnsiString
 0001:00012D44       SysUtils.MapException
 0001:0001467C       SysUtils.ModuleUnloaded
 0003:00000DE0       SysUtils.MonitorSupport
 0003:00000B44       SysUtils.MonthDays
 0004:00002C79       SysUtils.NegCurrFormat
 0001:0001321C       SysUtils.NewSyncObj
 0001:000132A8       SysUtils.NewWaitObj
 0001:00013B14       SysUtils.NextCharIndex
 0004:00002DA8       SysUtils.OutOfMemory
 0001:000131FC       SysUtils.Pop
 0001:000131DC       SysUtils.Push
 0001:0000F15C       SysUtils.PutExponent
 0001:00012D00       SysUtils.RaiseAssertException
 0001:00013088       SysUtils.RaiseExceptObject
 0001:000147A8       SysUtils.RaiseLastOSError
 0001:0001479C       SysUtils.RaiseLastOSError
 0001:0000D434       SysUtils.SameText
 0001:00010B74       SysUtils.ScanBlanks
 0001:00010D88       SysUtils.ScanChar
 0001:00011040       SysUtils.ScanDate
 0001:00010BE0       SysUtils.ScanNumber
 0001:00010CA8       SysUtils.ScanString
 0001:000113F8       SysUtils.ScanTime
 0001:00010ECC       SysUtils.ScanToNumber
 0003:00000BC4       SysUtils.ShareMode
 0003:00000BB0       SysUtils.ShareMode
 0004:00002C84       SysUtils.ShortDateFormat
 0004:00002D00       SysUtils.ShortDayNames
 0004:00002CA0       SysUtils.ShortMonthNames
 0004:00002C98       SysUtils.ShortTimeFormat
 0001:000121A0       SysUtils.ShowException
 0001:00014794       SysUtils.Sleep
 0001:00013A20       SysUtils.StrCharLength
 0001:0000E7FC       SysUtils.StrEnd
 0001:000142B8       SysUtils.StringReplace
 0001:0000E864       SysUtils.StrLComp
 0001:0000E828       SysUtils.StrLCopy
 0001:0000E7AC       SysUtils.StrLen
 0001:0000E7DC       SysUtils.StrLen
 0001:0000EAC8       SysUtils.StrLFmt
 0001:0000E8B0       SysUtils.StrLIComp
 0001:0000E818       SysUtils.StrMove
 0001:0000EA38       SysUtils.StrNew
 0001:00013A50       SysUtils.StrNextChar
 0001:0000E968       SysUtils.StrPos
 0001:0000E9C0       SysUtils.StrPosLen
 0001:0000E938       SysUtils.StrRScan
 0001:0000E91C       SysUtils.StrScan
 0001:0000DED0       SysUtils.StrToInt
 0001:0000DF0C       SysUtils.StrToIntDef
 0001:00014D44       SysUtils.Supports
 0001:00014D68       SysUtils.Supports
 0004:00002DB0       SysUtils.SyncEventCache
 0001:00011950       SysUtils.SysErrorMessage
 0004:00002D38       SysUtils.SysLocale
 0001:0000FE10       SysUtils.SystemTimeToDateTime
 0002:000000DC       SysUtils.SysUtils
 0001:00015FE0       SysUtils.TBigEndianUnicodeEncoding.GetBytes
 0001:00016014       SysUtils.TBigEndianUnicodeEncoding.GetChars
 0001:00016050       SysUtils.TBigEndianUnicodeEncoding.GetPreamble
 0004:00002DA0       SysUtils.TEncoding.$ClassInitFlag
 0001:00014E30       SysUtils.TEncoding.Convert
 0001:00014EA4       SysUtils.TEncoding.Convert
 0002:000000C4       SysUtils.TEncoding.Create@
 0001:00014F20       SysUtils.TEncoding.Destroy@
 0004:00002D88       SysUtils.TEncoding.FASCIIEncoding
 0004:00002D8C       SysUtils.TEncoding.FBigEndianUnicodeEncoding
 0004:00002D90       SysUtils.TEncoding.FDefaultEncoding
 0001:00014F34       SysUtils.TEncoding.FreeEncodings
 0004:00002D94       SysUtils.TEncoding.FUnicodeEncoding
 0004:00002D98       SysUtils.TEncoding.FUTF7Encoding
 0004:00002D9C       SysUtils.TEncoding.FUTF8Encoding
 0001:00014FA4       SysUtils.TEncoding.GetBigEndianUnicode
 0001:0001503C       SysUtils.TEncoding.GetBufferEncoding
 0001:00015290       SysUtils.TEncoding.GetByteCount
 0001:0001520C       SysUtils.TEncoding.GetByteCount
 0001:00015160       SysUtils.TEncoding.GetByteCount
 0001:00015144       SysUtils.TEncoding.GetByteCount
 0001:00015394       SysUtils.TEncoding.GetBytes
 0001:00015548       SysUtils.TEncoding.GetBytes
 0001:000155EC       SysUtils.TEncoding.GetBytes
 0001:000153DC       SysUtils.TEncoding.GetBytes
 0001:000157AC       SysUtils.TEncoding.GetCharCount
 0001:00015790       SysUtils.TEncoding.GetCharCount
 0001:0001599C       SysUtils.TEncoding.GetChars
 0001:00015878       SysUtils.TEncoding.GetChars
 0001:0001589C       SysUtils.TEncoding.GetChars
 0001:00015AF0       SysUtils.TEncoding.GetDefault
 0001:00015B30       SysUtils.TEncoding.GetEncoding
 0001:0000C714       SysUtils.TEncoding.GetMaxByteCount
 0001:0000C71C       SysUtils.TEncoding.GetMaxCharCount
 0001:0000C724       SysUtils.TEncoding.GetPreamble
 0001:00015B64       SysUtils.TEncoding.GetString
 0001:00015B40       SysUtils.TEncoding.GetString
 0001:00015BD4       SysUtils.TEncoding.GetUnicode
 0001:00015C10       SysUtils.TEncoding.GetUTF8
 0001:00015C4C       SysUtils.TEncoding.IsStandardEncoding
 0003:00000DF4       SysUtils.TerminateProcList
 0001:0000F800       SysUtils.TextToFloat
 0001:0000F6EC       SysUtils.TextToFloat
 0004:00002C7A       SysUtils.ThousandSeparator
 0004:00002C90       SysUtils.TimeAMString
 0004:00002C94       SysUtils.TimePMString
 0004:00002C8C       SysUtils.TimeSeparator
 0001:00015CC4       SysUtils.TMBCSEncoding.Create
 0001:00015D0C       SysUtils.TMBCSEncoding.Create
 0001:00015C84       SysUtils.TMBCSEncoding.Create
 0001:00015D88       SysUtils.TMBCSEncoding.GetByteCount
 0001:00015DA0       SysUtils.TMBCSEncoding.GetBytes
 0001:00015DC4       SysUtils.TMBCSEncoding.GetCharCount
 0001:00015DD8       SysUtils.TMBCSEncoding.GetChars
 0001:00015DF8       SysUtils.TMBCSEncoding.GetMaxByteCount
 0001:00015E00       SysUtils.TMBCSEncoding.GetMaxCharCount
 0001:00015E04       SysUtils.TMBCSEncoding.GetPreamble
 0001:00014C5C       SysUtils.TMultiReadExclusiveWriteSynchronizer.BeginRead
 0001:00014B60       SysUtils.TMultiReadExclusiveWriteSynchronizer.BeginWrite
 0001:00014B1C       SysUtils.TMultiReadExclusiveWriteSynchronizer.BlockReaders
 0001:00014A60       SysUtils.TMultiReadExclusiveWriteSynchronizer.Create
 0001:00014AD4       SysUtils.TMultiReadExclusiveWriteSynchronizer.Destroy
 0001:00014CCC       SysUtils.TMultiReadExclusiveWriteSynchronizer.EndRead
 0001:00014C0C       SysUtils.TMultiReadExclusiveWriteSynchronizer.EndWrite
 0001:00014B34       SysUtils.TMultiReadExclusiveWriteSynchronizer.UnblockOneWriter
 0001:00014B28       SysUtils.TMultiReadExclusiveWriteSynchronizer.UnblockReaders
 0001:00014B40       SysUtils.TMultiReadExclusiveWriteSynchronizer.WaitForReadSignal
 0001:00014B50       SysUtils.TMultiReadExclusiveWriteSynchronizer.WaitForWriteSignal
 0001:00011CE4       SysUtils.TranslateDateFormat
 0001:0000D680       SysUtils.Trim
 0004:00002D80       SysUtils.TrueBoolStrs
 0001:0000FB68       SysUtils.TryEncodeDate
 0001:0000FA20       SysUtils.TryEncodeTime
 0001:0000E054       SysUtils.TryStrToBool
 0001:0000F9C0       SysUtils.TryStrToCurr
 0001:00011600       SysUtils.TryStrToDate
 0001:00011720       SysUtils.TryStrToDateTime
 0001:0000F950       SysUtils.TryStrToFloat
 0001:0000F8C4       SysUtils.TryStrToFloat
 0001:0000F8E0       SysUtils.TryStrToFloat
 0001:0000DF24       SysUtils.TryStrToInt
 0001:0000DF44       SysUtils.TryStrToInt64
 0001:00011690       SysUtils.TryStrToTime
 0001:00014A04       SysUtils.TThreadLocalCounter.Close
 0001:00014A0C       SysUtils.TThreadLocalCounter.Delete
 0001:00014918       SysUtils.TThreadLocalCounter.Destroy
 0001:00014970       SysUtils.TThreadLocalCounter.HashIndex
 0001:0001498C       SysUtils.TThreadLocalCounter.Open
 0001:00014A1C       SysUtils.TThreadLocalCounter.Recycle
 0001:00015F24       SysUtils.TUnicodeEncoding.Create
 0001:00015F50       SysUtils.TUnicodeEncoding.GetByteCount
 0001:00015F58       SysUtils.TUnicodeEncoding.GetBytes
 0001:00015F74       SysUtils.TUnicodeEncoding.GetCharCount
 0001:00015F80       SysUtils.TUnicodeEncoding.GetChars
 0001:00015FA0       SysUtils.TUnicodeEncoding.GetMaxByteCount
 0001:00015FA8       SysUtils.TUnicodeEncoding.GetMaxCharCount
 0001:00015FB8       SysUtils.TUnicodeEncoding.GetPreamble
 0001:00015E20       SysUtils.TUTF7Encoding.Create
 0001:00015E5C       SysUtils.TUTF7Encoding.GetByteCount
 0001:00015E64       SysUtils.TUTF7Encoding.GetBytes
 0001:00015E7C       SysUtils.TUTF7Encoding.GetCharCount
 0001:00015E84       SysUtils.TUTF7Encoding.GetChars
 0001:00015E9C       SysUtils.TUTF7Encoding.GetMaxByteCount
 0001:00015EA4       SysUtils.TUTF7Encoding.GetMaxCharCount
 0001:00015EA8       SysUtils.TUTF8Encoding.Create
 0001:00015EE8       SysUtils.TUTF8Encoding.GetMaxByteCount
 0001:00015EF0       SysUtils.TUTF8Encoding.GetMaxCharCount
 0001:00015EF4       SysUtils.TUTF8Encoding.GetPreamble
 0003:00000B40       SysUtils.TwoDigitYearCenturyWindow
 0001:0000DC94       SysUtils.UIntToStr
 0004:00003EAC       SysUtils.UnitHashBuckets
 0001:0000D0A4       SysUtils.UpperCase
 0001:0000D054       SysUtils.UpperCaseFromAnsiString
 0004:00002EB8       SysUtils.ValidatedUnitHashBuckets
 0001:0000DF64       SysUtils.VerifyBoolStrArray
 0001:00013314       SysUtils.WaitAndOrSignalObj
 0001:0000ED5C       SysUtils.WideFloatToText
 0001:0000ED78       SysUtils.WideFormatBuf
 0001:0000ECB8       SysUtils.WideFormatError
 0001:0000ED38       SysUtils.WideFormatVarToStr
 0001:0000EA20       SysUtils.WideStrAlloc
 0003:00000B38       SysUtils.Win32BuildNumber
 0001:00014840       SysUtils.Win32Check
 0003:00000B3C       SysUtils.Win32CSDVersion
 0003:00000B30       SysUtils.Win32MajorVersion
 0003:00000B34       SysUtils.Win32MinorVersion
 0003:00000B2C       SysUtils.Win32Platform
 0004:00004F40       TypInfo..5
 0001:0001F930       TypInfo.AssignLongStr
 0001:00020468       TypInfo.AssignVariant
 0003:00000F58       TypInfo.BooleanIdents
 0003:00000F60       TypInfo.DotSep
 0001:000206CC       TypInfo.Finalization
 0001:0001FB30       TypInfo.GetAnsiStrProp
 0001:0001F1E4       TypInfo.GetEnumName
 0001:0001F350       TypInfo.GetEnumNameValue
 0001:0001F3C8       TypInfo.GetEnumValue
 0001:00020158       TypInfo.GetFloatProp
 0001:00020574       TypInfo.GetInt64Prop
 0001:000205D8       TypInfo.GetInterfaceProp
 0001:0001F948       TypInfo.GetLongStrProp
 0001:000204FC       TypInfo.GetMethodProp
 0001:0001F5FC       TypInfo.GetOrdProp
 0001:0001F524       TypInfo.GetPropInfo
 0001:0001F578       TypInfo.GetPropInfos
 0001:0001F188       TypInfo.GetPropName
 0001:0001F6CC       TypInfo.GetSetElementName
 0001:0001F760       TypInfo.GetSetElementValue
 0001:0001F834       TypInfo.GetShortStrProp
 0001:0001F8CC       TypInfo.GetShortStrPropAsLongStr
 0001:0001F1D8       TypInfo.GetTypeData
 0001:0001FDC8       TypInfo.GetUnicodeStrProp
 0001:0001FA7C       TypInfo.GetUnicodeStrPropAsLongStr
 0001:0002047C       TypInfo.GetVariantProp
 0001:0001FBB8       TypInfo.GetWideStrProp
 0001:0001F9C8       TypInfo.GetWideStrPropAsLongStr
 0001:0001F470       TypInfo.InternalGetPropInfo
 0001:0001F5CC       TypInfo.IsStoredProp
 0001:0001FB7C       TypInfo.SetAnsiStrProp
 0001:00020270       TypInfo.SetFloatProp
 0001:0002059C       TypInfo.SetInt64Prop
 0001:00020658       TypInfo.SetInterfaceProp
 0001:0001F988       TypInfo.SetLongStrProp
 0001:0002053C       TypInfo.SetMethodProp
 0001:0001F670       TypInfo.SetOrdProp
 0001:0001FEE0       TypInfo.SetRawByteStrProp
 0001:0001F878       TypInfo.SetShortStrProp
 0001:0001F8FC       TypInfo.SetShortStrPropAsLongStr
 0001:00020034       TypInfo.SetUnicodeStrProp
 0001:0001FAD8       TypInfo.SetUnicodeStrPropAsLongStr
 0001:000204BC       TypInfo.SetVariantProp
 0001:0001FCCC       TypInfo.SetWideStrProp
 0001:0001FA24       TypInfo.SetWideStrPropAsLongStr
 0002:00000234       TypInfo.TypInfo
 0001:0001F2DC       TypInfo.UTF8SameText
 0004:00004F20       Variants..81
 0001:000177FC       Variants..EVariantArrayCreateError
 0001:00017748       Variants..EVariantArrayLockedError
 0001:0001769C       Variants..EVariantBadIndexError
 0001:000175EC       Variants..EVariantBadVarTypeError
 0001:00017AC0       Variants..EVariantDispatchError
 0001:0001753C       Variants..EVariantInvalidArgError
 0001:00017B6C       Variants..EVariantInvalidNullOpError
 0001:00017334       Variants..EVariantInvalidOpError
 0001:000178B0       Variants..EVariantNotImplError
 0001:0001795C       Variants..EVariantOutOfMemoryError
 0001:00017490       Variants..EVariantOverflowError
 0001:000173E4       Variants..EVariantTypeCastError
 0001:00017A10       Variants..EVariantUnexpectedError
 0001:00016E24       Variants..TCustomVariantType
 0001:000181C4       Variants.@DispInvokeError
 0001:0001E1A0       Variants.@VarAddRef
 0001:00018B48       Variants.@VarCast
 0001:000184C8       Variants.@VarClear
 0001:000184DC       Variants.@VarClr
 0001:0001EE88       Variants.@VarCmpEQ
 0001:00018830       Variants.@VarCopy
 0001:0001D698       Variants.@VarFromBool
 0001:0001D4F8       Variants.@VarFromByte
 0001:0001D6E8       Variants.@VarFromCurr
 0001:0001D640       Variants.@VarFromCurrency
 0001:0001D66C       Variants.@VarFromDate
 0001:0001D7B8       Variants.@VarFromDisp
 0001:0001D614       Variants.@VarFromDouble
 0001:0001D49C       Variants.@VarFromInt
 0001:0001D5C4       Variants.@VarFromInt64
 0001:0001D4D8       Variants.@VarFromInteger
 0001:0001D78C       Variants.@VarFromIntf
 0001:0001D538       Variants.@VarFromLongWord
 0001:0001D6FC       Variants.@VarFromLStr
 0001:0001D6C0       Variants.@VarFromReal
 0001:0001D584       Variants.@VarFromShortInt
 0001:0001D5F0       Variants.@VarFromSingle
 0001:0001D5A4       Variants.@VarFromSmallInt
 0001:0001D6D4       Variants.@VarFromTDateTime
 0001:0001D558       Variants.@VarFromUInt64
 0001:0001D760       Variants.@VarFromUStr
 0001:0001D518       Variants.@VarFromWord
 0001:0001D728       Variants.@VarFromWStr
 0001:00018218       Variants.@VarNull
 0001:0001A5B0       Variants.@VarToBool
 0001:0001A214       Variants.@VarToBoolean
 0001:00019498       Variants.@VarToByte
 0001:0001B590       Variants.@VarToCurrency
 0001:0001AF94       Variants.@VarToDate
 0001:0001D3F0       Variants.@VarToDisp
 0001:0001A77C       Variants.@VarToDouble
 0001:00019A6C       Variants.@VarToInt64
 0001:00018F34       Variants.@VarToInteger
 0001:0001D324       Variants.@VarToIntf
 0001:0001971C       Variants.@VarToLongWord
 0001:0001BCC8       Variants.@VarToLStr
 0001:0001AB6C       Variants.@VarToReal
 0001:000193E4       Variants.@VarToShortInt
 0001:0001AB88       Variants.@VarToSingle
 0001:00019544       Variants.@VarToSmallInt
 0001:00019EFC       Variants.@VarToUInt64
 0001:0001CCA4       Variants.@VarToUStr
 0001:00019640       Variants.@VarToWord
 0001:0001C57C       Variants.@VarToWStr
 0001:0001D2AC       Variants.AnyToIntf
 0003:00000E1C       Variants.BaseTypeMap
 0003:00000E18       Variants.BooleanToStringRule
 0001:0001BA5C       Variants.BoolToWStrViaOS
 0003:00000E4C       Variants.CBooleanToRelationship
 0004:00004F18       Variants.ChangeAnyProc
 0001:0001D7E4       Variants.CheckType
 0003:00000E34       Variants.CInvalidCustomVariantType
 0004:00004F14       Variants.ClearAnyProc
 0001:0001E78C       Variants.ClearVariantTypeList
 0003:00000E58       Variants.CmpTypeMap
 0003:00000E38       Variants.CRangeToType
 0003:00000F44       Variants.CRelationshipToBoolean
 0003:00000EE8       Variants.CText
 0001:0001DACC       Variants.CurrCompare
 0001:0001B9EC       Variants.CurrToWStrViaOS
 0001:0001DAA0       Variants.DateCompare
 0001:0001BA24       Variants.DateToWStrViaOS
 0001:0001D8E8       Variants.EmptyCompare
 0004:00004F00       Variants.EmptyParam
 0001:0001EE98       Variants.Finalization
 0001:0001ECF0       Variants.FindCustomVariantType
 0001:0001EDAC       Variants.FindCustomVariantType
 0001:0001E5D0       Variants.FindVarData
 0001:0001E6F0       Variants.GetVarDataArrayInfo
 0001:00018140       Variants.HandleConversionException
 0001:0001822C       Variants.InBounds
 0001:000184E4       Variants.InBounds
 0001:0001825C       Variants.Increment
 0001:00018514       Variants.Increment
 0001:0001DA04       Variants.Int64Compare
 0001:0001D9F0       Variants.IntCompare
 0003:00000F40       Variants.LNextVarType
 0004:00004F24       Variants.LVarTypes
 0004:00004F28       Variants.LVarTypeSync
 0001:0001EE80       Variants.Null
 0003:00000E10       Variants.NullAsStringValue
 0001:0001D8FC       Variants.NullCompare
 0003:00000E04       Variants.NullEqualityRule
 0003:00000E08       Variants.NullMagnitudeRule
 0003:00000E0C       Variants.NullStrictConvert
 0003:00000E14       Variants.PackVarCreation
 0001:0001DA74       Variants.RealCompare
 0004:00004F1C       Variants.RefAnyProc
 0001:0001E6E4       Variants.SetClearVarToEmptyParam
 0001:0001E6CC       Variants.SetVarAsError
 0001:0001DAFC       Variants.StringCompare
 0001:0001E7F8       Variants.TCustomVariantType.BinaryOp
 0001:0001E804       Variants.TCustomVariantType.Cast
 0001:0001E83C       Variants.TCustomVariantType.CastTo
 0001:0001E8C8       Variants.TCustomVariantType.CastToOle
 0001:00017324       Variants.TCustomVariantType.Clear
 0001:0001E884       Variants.TCustomVariantType.Compare
 0001:0001E890       Variants.TCustomVariantType.CompareOp
 0001:0001732C       Variants.TCustomVariantType.Copy
 0001:0001E948       Variants.TCustomVariantType.Create
 0001:0001E904       Variants.TCustomVariantType.Create
 0001:0001EBC4       Variants.TCustomVariantType.Destroy
 0001:0001ECA4       Variants.TCustomVariantType.DispInvoke
 0001:0001EC50       Variants.TCustomVariantType.IsClear
 0001:0001EC54       Variants.TCustomVariantType.LeftPromotion
 0001:0001EC68       Variants.TCustomVariantType.OlePromotion
 0001:0001ECC8       Variants.TCustomVariantType.QueryInterface
 0001:0001EC70       Variants.TCustomVariantType.RaiseCastError
 0001:0001EC80       Variants.TCustomVariantType.RaiseDispError
 0001:0001EC78       Variants.TCustomVariantType.RaiseInvalidOp
 0001:0001EC88       Variants.TCustomVariantType.RightPromotion
 0001:0001EC9C       Variants.TCustomVariantType.UnaryOp
 0001:0001ECB0       Variants.TCustomVariantType._AddRef
 0001:0001ECBC       Variants.TCustomVariantType._Release
 0001:00017EAC       Variants.TranslateResult
 0001:0001DA40       Variants.UInt64Compare
 0001:000182B8       Variants.VarArrayClear
 0001:00018570       Variants.VarArrayCopyForEach
 0001:00017E58       Variants.VarArrayCreateError
 0001:00018874       Variants.VarCastAsAny
 0001:000189C4       Variants.VarCastAsDispatch
 0001:00018A10       Variants.VarCastAsInterface
 0001:000188E0       Variants.VarCastAsOleStr
 0001:0001892C       Variants.VarCastAsString
 0001:00018978       Variants.VarCastAsUString
 0001:00017C24       Variants.VarCastError
 0001:00017C78       Variants.VarCastError
 0001:00018ADC       Variants.VarCastRare
 0001:00018A5C       Variants.VarCastViaOS
 0001:00018434       Variants.VarClearDeep
 0001:0001E138       Variants.VarCompare
 0001:0001D810       Variants.VarCompareAny
 0001:0001DD14       Variants.VarCompareRare
 0001:0001DB68       Variants.VarCompareSimple
 0001:0001873C       Variants.VarCopyCopyProc
 0001:00018744       Variants.VarCopyDeep
 0004:00004F10       Variants.VarDispProc
 0002:00000188       Variants.Variants
 0001:00017D68       Variants.VarInvalidNullOp
 0001:00017D14       Variants.VarInvalidOp
 0001:0001E734       Variants.VarIsArray
 0001:0001E73C       Variants.VarIsArray
 0001:0001E5E0       Variants.VarIsClear
 0001:00017DBC       Variants.VarOverflowError
 0001:0001810C       Variants.VarResultCheck
 0001:00018100       Variants.VarResultCheck
 0001:0001E654       Variants.VarSameValue
 0001:0001A164       Variants.VarToBoolAny
 0001:0001A060       Variants.VarToBoolAsString
 0001:0001A1C8       Variants.VarToBoolCustom
 0001:0001A124       Variants.VarToBoolViaOS
 0001:0001B4E0       Variants.VarToCurrencyAny
 0001:0001B434       Variants.VarToCurrencyAsDouble
 0001:0001B378       Variants.VarToCurrencyAsString
 0001:0001B544       Variants.VarToCurrencyCustom
 0001:0001B494       Variants.VarToCurrencyViaOS
 0001:0001AEE4       Variants.VarToDateAny
 0001:0001AE38       Variants.VarToDateAsDouble
 0001:0001AD4C       Variants.VarToDateAsString
 0001:0001AF48       Variants.VarToDateCustom
 0001:0001AE98       Variants.VarToDateViaOS
 0001:0001A6CC       Variants.VarToDoubleAny
 0001:0001A5BC       Variants.VarToDoubleAsString
 0001:0001A730       Variants.VarToDoubleCustom
 0001:0001A680       Variants.VarToDoubleViaOS
 0001:000199B4       Variants.VarToInt64Any
 0001:000198B4       Variants.VarToInt64AsString
 0001:00019A20       Variants.VarToInt64Custom
 0001:00019808       Variants.VarToInt64ViaOS
 0001:00018E8C       Variants.VarToIntAny
 0001:00018D9C       Variants.VarToIntAsString
 0001:00018EF0       Variants.VarToIntCustom
 0001:00018E50       Variants.VarToIntViaOS
 0001:0001BBDC       Variants.VarToLStrAny
 0001:0001BC40       Variants.VarToLStrCustom
 0001:0001BB24       Variants.VarToLStrViaOS
 0001:0001CB78       Variants.VarToUStrAny
 0001:0001CBDC       Variants.VarToUStrCustom
 0001:0001C43C       Variants.VarToWStrAny
 0001:0001C4A0       Variants.VarToWStrCustom
 0001:0001C370       Variants.VarToWStrViaOS
 0001:0001E41C       Variants.VarTypeAsText
 0004:00004EFC       VarUtils..5
 0001:00016840       VarUtils.BackupVarBoolFromStr
 0001:000169A4       VarUtils.BackupVarBStrFromBool
 0001:000168C0       VarUtils.BackupVarBStrFromCy
 0001:00016930       VarUtils.BackupVarBStrFromDate
 0001:000167D4       VarUtils.BackupVarCyFromStr
 0001:00016768       VarUtils.BackupVarDateFromStr
 0001:00016624       VarUtils.BackupVarI4FromStr
 0001:000165D0       VarUtils.BackupVariantChangeTypeEx
 0001:00016690       VarUtils.BackupVarR4FromStr
 0001:000166FC       VarUtils.BackupVarR8FromStr
 0001:0001660C       VarUtils.BiUnimplemented
 0001:00016618       VarUtils.CmpUnimplemented
 0003:00000DFC       VarUtils.CResult
 0001:00016D7C       VarUtils.Finalization
 0001:00016A38       VarUtils.FindProc
 0001:00016A64       VarUtils.InitializeVarUtils
 0001:00016A18       VarUtils.SafeArrayCreate
 0001:00016A20       VarUtils.SafeArrayGetLBound
 0001:00016A28       VarUtils.SafeArrayGetUBound
 0001:00016A30       VarUtils.SafeArrayPtrOfIndex
 0001:00016600       VarUtils.UniUnimplemented
 0004:00004EB0       VarUtils.VarAdd
 0004:00004EC8       VarUtils.VarAnd
 0004:00004EEC       VarUtils.VarBoolFromStr
 0004:00004EF8       VarUtils.VarBstrFromBool
 0004:00004EF0       VarUtils.VarBstrFromCy
 0004:00004EF4       VarUtils.VarBstrFromDate
 0004:00004ED4       VarUtils.VarCmp
 0004:00004EE8       VarUtils.VarCyFromStr
 0004:00004EE4       VarUtils.VarDateFromStr
 0004:00004EBC       VarUtils.VarDiv
 0004:00004ED8       VarUtils.VarI4FromStr
 0001:000165C8       VarUtils.VariantChangeType
 0004:00004EA4       VarUtils.VariantChangeTypeEx
 0001:000165B8       VarUtils.VariantClear
 0001:000165C0       VarUtils.VariantCopy
 0001:000165B0       VarUtils.VariantInit
 0004:00004EC0       VarUtils.VarIDiv
 0004:00004EC4       VarUtils.VarMod
 0004:00004EB8       VarUtils.VarMul
 0004:00004EA8       VarUtils.VarNeg
 0004:00004EAC       VarUtils.VarNot
 0004:00004ECC       VarUtils.VarOr
 0004:00004EDC       VarUtils.VarR4FromStr
 0004:00004EE0       VarUtils.VarR8FromStr
 0004:00004EB4       VarUtils.VarSub
 0002:00000178       VarUtils.VarUtils
 0004:00004ED0       VarUtils.VarXor
 0004:00002C40       Windows..2
 0001:00009284       Windows.BeginDeferWindowPos
 0001:0000928C       Windows.BeginPaint
 0001:00009294       Windows.CallWindowProc
 0001:0000929C       Windows.CharNext
 0001:000092A4       Windows.CharUpperBuff
 0001:00008FD8       Windows.CloseHandle
 0001:00008FE0       Windows.CompareString
 0001:00008FE8       Windows.CompareStringW
 0001:00008FF0       Windows.CreateEvent
 0001:00008FF8       Windows.CreateFile
 0001:00009374       Windows.CreateWindow
 0001:000093CC       Windows.CreateWindowW
 0001:000092B4       Windows.DeferWindowPos
 0001:000092AC       Windows.DefWindowProc
 0001:00009000       Windows.DeleteCriticalSection
 0001:000092BC       Windows.EnableWindow
 0001:000092C4       Windows.EndDeferWindowPos
 0001:000092CC       Windows.EndPaint
 0001:00009008       Windows.EnterCriticalSection
 0001:00009010       Windows.EnumCalendarInfo
 0001:00009018       Windows.FileTimeToDosDateTime
 0001:00009020       Windows.FileTimeToLocalFileTime
 0001:00009028       Windows.FileTimeToSystemTime
 0001:00009460       Windows.Finalization
 0001:00009030       Windows.FindClose
 0001:00009038       Windows.FindFirstFile
 0001:00009040       Windows.FindNextFile
 0001:00009048       Windows.FindResource
 0001:00009050       Windows.FormatMessage
 0001:00009058       Windows.FreeLibrary
 0001:00009098       Windows.FreeResource
 0001:000092D4       Windows.GetClientRect
 0001:000090A0       Windows.GetCPInfo
 0001:000090A8       Windows.GetCurrentProcess
 0001:000090B0       Windows.GetCurrentThread
 0001:000090B8       Windows.GetCurrentThreadId
 0001:000090C0       Windows.GetDateFormat
 0001:000090C8       Windows.GetDiskFreeSpace
 0001:000090D0       Windows.GetExitCodeThread
 0001:000090D8       Windows.GetFileAttributes
 0001:000090E0       Windows.GetFullPathName
 0001:000090E8       Windows.GetLastError
 0001:000090F8       Windows.GetLocaleInfo
 0001:000090F0       Windows.GetLocalTime
 0001:00009100       Windows.GetModuleFileName
 0001:00009108       Windows.GetModuleHandle
 0001:00009110       Windows.GetProcAddress
 0001:00009118       Windows.GetProcAddress
 0001:0000918C       Windows.GetStdHandle
 0001:000092DC       Windows.GetSystemMetrics
 0001:00009194       Windows.GetThreadLocale
 0001:0000919C       Windows.GetThreadPriority
 0001:000091A4       Windows.GetVersionEx
 0001:000092E4       Windows.GetWindowLong
 0004:00002C44       Windows.HtmlHelpModule
 0001:000091AC       Windows.InitializeCriticalSection
 0001:00009424       Windows.InitVersionInfo
 0001:00009060       Windows.InterlockedCompareExchange
 0001:00009068       Windows.InterlockedCompareExchangePointer
 0001:00009080       Windows.InterlockedExchange
 0001:00009088       Windows.InterlockedExchangeAdd
 0001:00009090       Windows.InterlockedIncrement
 0001:000091DC       Windows.IsDebuggerPresent
 0001:000091B4       Windows.LeaveCriticalSection
 0001:000092EC       Windows.LoadCursor
 0001:000092F4       Windows.LoadIcon
 0001:000091BC       Windows.LoadLibrary
 0001:000091C4       Windows.LoadResource
 0001:000092FC       Windows.LoadString
 0001:000091CC       Windows.LockResource
 0001:00009304       Windows.MessageBox
 0001:0000930C       Windows.MsgWaitForMultipleObjects
 0001:000091D4       Windows.MultiByteToWideChar
 0001:00009314       Windows.PeekMessage
 0001:0000931C       Windows.PostMessage
 0001:00009324       Windows.PostQuitMessage
 0001:000091E4       Windows.RaiseException
 0001:000091EC       Windows.ReadFile
 0001:00008F50       Windows.RegCloseKey
 0001:00008F58       Windows.RegConnectRegistry
 0001:00008F60       Windows.RegCreateKeyEx
 0001:00008F68       Windows.RegDeleteKey
 0001:00008F70       Windows.RegDeleteValue
 0001:00008F78       Windows.RegEnumKeyEx
 0001:00008F80       Windows.RegEnumValue
 0001:00008F88       Windows.RegFlushKey
 0001:0000932C       Windows.RegisterClass
 0001:00008F90       Windows.RegLoadKey
 0001:00008F98       Windows.RegOpenKeyEx
 0001:00008FA0       Windows.RegQueryInfoKey
 0001:00008FA8       Windows.RegQueryValueEx
 0001:00008FB0       Windows.RegReplaceKey
 0001:00008FB8       Windows.RegRestoreKey
 0001:00008FC0       Windows.RegSaveKey
 0001:00008FC8       Windows.RegSetValueEx
 0001:00008FD0       Windows.RegUnLoadKey
 0001:000091F4       Windows.ResetEvent
 0001:000091FC       Windows.ResumeThread
 0001:00009334       Windows.SendMessageW
 0001:00009204       Windows.SetEndOfFile
 0001:0000920C       Windows.SetEvent
 0001:00009214       Windows.SetFilePointer
 0001:0000921C       Windows.SetLastError
 0001:00009224       Windows.SetThreadPriority
 0001:0000933C       Windows.SetTimer
 0001:00009344       Windows.SetWindowLong
 0001:0000934C       Windows.SetWindowTextW
 0001:00009354       Windows.ShowWindow
 0001:0000922C       Windows.SignalObjectAndWait
 0001:00009234       Windows.SizeofResource
 0001:0000923C       Windows.SuspendThread
 0001:00009244       Windows.SwitchToThread
 0001:0000924C       Windows.TryEnterCriticalSection
 0001:0000935C       Windows.UpdateWindow
 0001:00009254       Windows.VirtualFree
 0001:0000925C       Windows.VirtualQuery
 0001:00009264       Windows.VirtualQueryEx
 0001:0000926C       Windows.WaitForSingleObject
 0001:00009274       Windows.WideCharToMultiByte
 0003:00000A14       Windows.Win32MajorVersion
 0003:00000A18       Windows.Win32MinorVersion
 0003:00000A1C       Windows.Win32Platform
 0002:000000AC       Windows.Windows
 0001:0000927C       Windows.WriteFile
 0001:00009364       Windows._CreateWindowEx
 0001:0000936C       Windows._CreateWindowExW


  Address             Publics by Value

 0001:0000040C       System..TObject
 0001:00000C74       System..TInterfacedObject
 0001:000013B4       System.InterlockedIncrement
 0001:000013C0       System.InterlockedDecrement
 0001:000013CC       System.CloseHandle
 0001:000013D4       System.InitializeCriticalSection
 0001:000013DC       System.EnterCriticalSection
 0001:000013E4       System.LeaveCriticalSection
 0001:000013EC       System.DeleteCriticalSection
 0001:000013F4       System.GetStdHandle
 0001:000013FC       System.RaiseException
 0001:00001404       System.RtlUnwind
 0001:0000140C       System.UnhandledExceptionFilter
 0001:00001414       System.WriteFile
 0001:0000141C       System.CharNext
 0001:00001424       System.CompareStringW
 0001:0000142C       System.CompareString
 0001:00001434       System.CreateThread
 0001:0000143C       System.ExitThread
 0001:00001444       System.ExitProcess
 0001:0000144C       System.MessageBoxA
 0001:00001454       System.FindClose
 0001:0000145C       System.FindFirstFile
 0001:00001464       System.FreeLibrary
 0001:0000146C       System.GetCommandLine
 0001:00001474       System.GetLastError
 0001:0000147C       System.GetLocaleInfo
 0001:00001484       System.GetUserDefaultUILanguage
 0001:0000148C       System.GetModuleFileName
 0001:00001494       System.GetModuleHandle
 0001:0000149C       System.GetProcAddress
 0001:000014A4       System.GetStartupInfo
 0001:000014AC       System.GetSystemDefaultUILanguage
 0001:000014B4       System.IsValidLocale
 0001:000014BC       System.LoadLibraryEx
 0001:000014C4       System.LoadString
 0001:000014CC       System.lstrcpyn
 0001:000014D4       System.@strlen
 0001:000014DC       System.MultiByteToWideChar
 0001:000014E4       System.RegCloseKey
 0001:000014EC       System.RegOpenKeyEx
 0001:000014F4       System.RegQueryValueEx
 0001:000014FC       System.WideCharToMultiByte
 0001:00001504       System.VirtualQuery
 0001:0000150C       System.SysAllocStringLen
 0001:00001514       System.SysReAllocStringLen
 0001:0000151C       System.SysFreeString
 0001:00001524       System.GetCurrentThreadId
 0001:0000152C       System.GetVersion
 0001:00001534       System.QueryPerformanceCounter
 0001:0000153C       System.GetTickCount
 0001:00001544       System.GetSystemInfo
 0001:0000154C       System.GetCmdShow
 0001:00001578       System.VirtualAlloc
 0001:00001580       System.VirtualFree
 0001:00001588       System.Sleep
 0001:000016D8       System.LockCmpxchg
 0001:000016E0       System.Move12
 0001:000016F4       System.Move20
 0001:00001714       System.Move28
 0001:00001740       System.Move36
 0001:00001760       System.Move44
 0001:00001784       System.Move52
 0001:000017B0       System.Move60
 0001:000017E0       System.Move68
 0001:00001818       System.MoveX16L4
 0001:00001848       System.MoveX8L4
 0001:00001864       System.RemoveMediumFreeBlock
 0001:000018A4       System.InsertMediumBlockIntoBin
 0001:00001904       System.BinMediumSequentialFeedRemainder
 0001:00001970       System.AllocNewSequentialFeedMediumPool
 0001:000019E8       System.LockLargeBlocks
 0001:00001A30       System.AllocateLargeBlock
 0001:00001A94       System.FreeLargeBlock
 0001:00001B38       System.ReallocateLargeBlock
 0001:00001C84       System.SysGetMem
 0001:00002008       System.SysFreeMem
 0001:00002200       System.SysReallocMem
 0001:00002518       System.SysAllocMem
 0001:0000254C       System.NextMediumBlock
 0001:00002570       System.GetFirstMediumBlockInPool
 0001:000025B0       System.GetFirstAndLastSmallBlockInPool
 0001:000025EC       System.CardinalToStrBuf
 0001:00002708       System.AppendStringToBuffer
 0001:00002720       System.AppendClassNameToBuffer
 0001:00002754       System.IsValidVMTAddress
 0001:000027D0       System.InternalIsValidClass
 0001:00002850       System.GetObjectClass
 0001:00002878       System.LockExpectedMemoryLeaksList
 0001:000028EC       System.SysRegisterExpectedMemoryLeak
 0001:0000292C       System.SysUnregisterExpectedMemoryLeak
 0001:00002984       System.CheckSmallBlockPoolForLeaks
 0001:00002B44       System.ScanForMemoryLeaks
 0001:00002F28       System.BuildBlockTypeLookupTable
 0001:00002F6C       System.InitializeMemoryManager
 0001:00003094       System.FreeAllMemory
 0001:00003124       System.FinalizeMemoryManager
 0001:00003178       System.AllocMem
 0001:00003190       System.@GetMem
 0001:000031AC       System.@FreeMem
 0001:000031C4       System.@ReallocMem
 0001:00003214       System.ExceptObject
 0001:00003234       System.AcquireExceptionObject
 0001:00003268       System.RaiseList
 0001:00003274       System.RunErrorAt
 0001:00003280       System.ErrorAt
 0001:000032CC       System.Error
 0001:000032D8       System.@_IOTest
 0001:000032F8       System.SetInOutRes
 0001:00003308       System.IOResult
 0001:00003328       System.Move
 0001:00003428       System.Randomize
 0001:00003450       System.Set8087CW
 0001:00003460       System.Get8087CW
 0001:00003468       System.@ROUND
 0001:00003474       System.@AbstractError
 0001:00003490       System.InternalFlush
 0001:000034D8       System.Flush
 0001:000034E4       System.@Close
 0001:0000353C       System.@AStrCmp
 0001:000035AC       System.@FillChar
 0001:00003648       System.@ValLong
 0001:0000374C       System.@SetElem
 0001:00003770       System.@SetUnion
 0001:0000377C       System.FPower10
 0001:00003784       System.@Pow10
 0001:00003A68       System.@FpuInit
 0001:00003A74       System.@BoundErr
 0001:00003A7C       System.@IntOver
 0001:00003A84       System.TObject.ClassType
 0001:00003A8C       System.TObject.ClassName
 0001:00003AA4       System.TObject.ClassNameIs
 0001:00003B40       System.TObject.ClassParent
 0001:00003B4C       System.TObject.NewInstance
 0001:00003B68       System.TObject.FreeInstance
 0001:00003B7C       System.TObject.InstanceSize
 0001:00003B84       System.TObject.Create
 0001:00003BA4       System.TObject.Destroy
 0001:00003BB4       System.TObject.Free
 0001:00003BC0       System.TObject.InitInstance
 0001:00003C18       System.TObject.CleanupInstance
 0001:00003C40       System.InvokeImplGetter
 0001:00003C70       System.TObject.Equals
 0001:00003C78       System.TObject.GetHashCode
 0001:00003C7C       System.TObject.GetInterface
 0001:00003D4C       System.TObject.GetInterfaceEntry
 0001:00003D90       System.TObject.GetInterfaceTable
 0001:00003D98       System.TObject.UnitName
 0001:00003DD0       System.@IsClass
 0001:00003DF4       System.FindDynaMethod
 0001:00003E24       System.@CallDynaInst
 0001:00003E3C       System.TObject.InheritsFrom
 0001:00003E50       System.TObject.ClassInfo
 0001:00003E58       System.TObject.SafeCallException
 0001:00003E60       System.TObject.ToString
 0001:00003E74       System.TObject.DefaultHandler
 0001:00003E78       System.TObject.AfterConstruction
 0001:00003E7C       System.TObject.BeforeDestruction
 0001:00003E80       System.TObject.Dispatch
 0001:00003EA8       System.UTF8Compare
 0001:00003F20       System.UTF8ShortStringToString
 0001:00003F34       System.TObject.MethodAddress
 0001:00003FA4       System.TObject.MethodAddress
 0001:00003FCC       System.TObject.MethodName
 0001:00004018       System.TObject.FieldAddress
 0001:0000408C       System.TObject.FieldAddress
 0001:000040B4       System.@ClassCreate
 0001:00004104       System.@ClassDestroy
 0001:0000410C       System.@AfterConstruction
 0001:0000415C       System.@BeforeDestruction
 0001:0000416C       System.TMonitor.Destroy
 0001:00004184       System.TMonitor.Destroy
 0001:000041B0       System.TMonitor.GetFieldAddress
 0001:000041C0       System.NotifyReRaise
 0001:000041DC       System.NotifyNonDelphiException
 0001:00004200       System.NotifyExcept
 0001:00004218       System.NotifyOnExcept
 0001:0000422C       System.NotifyAnyExcept
 0001:00004240       System.CheckJmp
 0001:00004260       System.NotifyExceptFinally
 0001:00004288       System.NotifyTerminate
 0001:000042A4       System.NotifyUnhandled
 0001:000042C4       System.@HandleAnyException
 0001:000043F0       System.@HandleOnException
 0001:00004578       System.@HandleFinally
 0001:00004620       System.@HandleFinallyInternal
 0001:00004658       System.@RaiseExcept
 0001:000046C8       System.@RaiseAgain
 0001:0000471C       System.@DoneExcept
 0001:0000474C       System.@TryFinallyExit
 0001:00004764       System.MapToRunError
 0001:00004804       System.@ExceptionHandler
 0001:000048A4       System.SetExceptionHandler
 0001:000048C4       System.UnsetExceptionHandler
 0001:000048EC       System.FinalizeUnits
 0001:00004954       System.InitUnits
 0001:000049C0       System.@StartExe
 0001:00004A08       System.LoadResStringA
 0001:00004A5C       System.LoadResStringW
 0001:00004AAC       System.LoadResStringU
 0001:00004AC0       System.@InitResStringImports
 0001:00004B04       System.@InitImports
 0001:00004B28       System.MakeErrorMessage
 0001:00004B8C       System.ExitDll
 0001:00004BB8       System.WriteErrorMessage
 0001:00004C48       System.@Halt0
 0001:00004D54       System.@Halt
 0001:00004D60       System.@RunError
 0001:00004D6C       System.@Assert
 0001:00004D8C       System.ThreadWrapper
 0001:00004DC4       System.BeginThread
 0001:00004E24       System.EndThread
 0001:00004E40       System.@LStrClr
 0001:00004E64       System.@LStrArrayClr
 0001:00004E94       System.@LStrAsg
 0001:00004EF0       System.@NewAnsiString
 0001:00004F3C       System.@LStrFromPCharLen
 0001:00004F74       System.CharFromWChar
 0001:00004FA0       System.CharFromWChar
 0001:00004FBC       System.WCharFromChar
 0001:00004FD8       System.EnsureAnsiString
 0001:00004FE8       System.EnsureUnicodeString
 0001:00004FF0       System.@InternalUStrFromLStr
 0001:00005000       System.@EnsureUnicodeString
 0001:00005020       System.@InternalLStrFromUStr
 0001:00005030       System.@LStrFromPWCharLen
 0001:000050B4       System.@LStrFromPChar
 0001:000050E8       System.@LStrFromPWChar
 0001:00005128       System.@LStrFromString
 0001:00005138       System.@LStrFromWStr
 0001:00005150       System.@LStrToString
 0001:00005174       System.@PCharLen
 0001:0000519C       System.@LStrAddRef
 0001:000051AC       System.@LStrToPChar
 0001:000051C4       System.InternalUniqueString
 0001:0000521C       System.UniqueString
 0001:00005224       System.@UniqueStringA
 0001:0000522C       System.@LStrSetLength
 0001:000052C4       System.WStrError
 0001:000052CC       System.@NewWideString
 0001:000052E4       System.WStrSet
 0001:000052F4       System.@WStrClr
 0001:0000530C       System.@WStrArrayClr
 0001:00005330       System.@WStrAsg
 0001:00005358       System.InternalWStrFromPCharLen
 0001:000053F4       System.@WStrFromPCharLen
 0001:00005404       System.@WStrFromPWCharLen
 0001:00005428       System.@WStrFromPChar
 0001:00005458       System.@WStrFromPWChar
 0001:00005494       System.@WStrFromLStr
 0001:000054C0       System.@WStrToPWChar
 0001:000054D0       System.@WStrCmp
 0001:00005554       System.@WStrEqual
 0001:0000555C       System.@WStrCopy
 0001:000055A8       System.@WStrSetLength
 0001:000055FC       System.@UStrAddRef
 0001:00005604       System.@UStrClr
 0001:0000560C       System.@UStrArrayClr
 0001:00005614       System.@UStrAsg
 0001:00005668       System.@UStrLAsg
 0001:000056A0       System.@UStrToPWChar
 0001:000056AC       System.InternalUStrFromPCharLen
 0001:00005740       System.@UStrFromPCharLen
 0001:00005750       System.@UStrFromPWCharLen
 0001:00005780       System.@UStrFromWChar
 0001:00005790       System.@UStrFromPChar
 0001:000057C0       System.@UStrFromPWChar
 0001:000057FC       System.@UStrFromWArray
 0001:00005818       System.@UStrFromLStr
 0001:00005840       System.@LStrFromUStr
 0001:00005864       System.@UStrFromWStr
 0001:00005878       System.@WStrFromUStr
 0001:000058A0       System.@UStrToString
 0001:00005960       System.@UStrLen
 0001:0000596C       System.@UStrSetLength
 0001:00005A04       System.@UStrCat
 0001:00005AC4       System.@UStrCat3
 0001:00005BA8       System.@UStrCatN
 0001:00005CC8       System.@UStrEqual
 0001:00005D30       System.@UStrCopy
 0001:00005E00       System.@UStrDelete
 0001:00005E74       System.InternalUniqueStringU
 0001:00005EC8       System.UniqueString
 0001:00005ED0       System.@NewUnicodeString
 0001:00005F14       System.Pos
 0001:00005F60       System.SetCodePage
 0001:0000614C       System.@InitializeRecord
 0001:00006180       System.@InitializeArray
 0001:00006218       System.@Initialize
 0001:00006224       System.@FinalizeRecord
 0001:0000625C       System.@VarClr
 0001:00006274       System.@FinalizeArray
 0001:00006384       System.@Finalize
 0001:00006390       System.@VarCopy
 0001:000063A8       System.@CopyRecord
 0001:000064E8       System.@CopyArray
 0001:00006600       System.@New
 0001:00006614       System.@Dispose
 0001:00006624       System.@DispCallByIDError
 0001:0000662C       System.@_llmul
 0001:00006650       System.@ValInt64
 0001:000069C8       System.@DynArrayLength
 0001:000069D0       System.@DynArrayHigh
 0001:000069D8       System.CopyArray
 0001:000069E8       System.FinalizeArray
 0001:000069F0       System.DynArrayClear
 0001:000069F8       System.DynArraySetLength
 0001:00006B90       System.@DynArraySetLength
 0001:00006B9C       System.@DynArrayClear
 0001:00006BD8       System.@DynArrayAsg
 0001:00006C00       System.@DynArrayAddRef
 0001:00006C0C       System.DelayLoadResourceModule
 0001:00006C54       System.FindResourceHInstance
 0001:00006EB8       System.InitializeLocaleData
 0001:00006FA8       System.FinalizeLocaleDate
 0001:00006FD4       System.LastHyphenPos
 0001:00007074       System.ConvertResToUILanguages
 0001:00007164       System.GetPreferredLangForOldOS
 0001:000072FC       System.CheckDifferentLanguageList
 0001:00007320       System.ThreadUILanguages
 0001:00007364       System.GetPreferredLangForNewOS
 0001:00007484       System.GetUILanguages
 0001:000075A8       System.FindBS
 0001:000075CC       System.ToLongPath
 0001:000077C8       System.GetLocaleOverride
 0001:00007A68       System.LoadResourceModule
 0001:00007B34       System.ResouceDLLExists
 0001:00007B6C       System.LoadLanguageList
 0001:00007C1C       System.Load3LettersModule
 0001:00007C78       System.GetResourceModuleName
 0001:00007E28       System.EnumResourceModules
 0001:00007E30       System.EnumResourceModules
 0001:00007E5C       System.AddModuleUnloadProc
 0001:00007E64       System.RemoveModuleUnloadProc
 0001:00007E6C       System.AddModuleUnloadProc
 0001:00007E8C       System.RemoveModuleUnloadProc
 0001:00007EF0       System.NotifyModuleUnload
 0001:00007F4C       System.RegisterModule
 0001:00007F5C       System.UnregisterModule
 0001:00007FCC       System.@IntfClear
 0001:00007FE4       System.@IntfCopy
 0001:00008010       System.@IntfCast
 0001:00008040       System.@IntfAddRef
 0001:0000804C       System.TInterfacedObject.AfterConstruction
 0001:00008058       System.TInterfacedObject.BeforeDestruction
 0001:00008068       System.TInterfacedObject.NewInstance
 0001:00008078       System.TInterfacedObject.QueryInterface
 0001:000080A0       System.TInterfacedObject._AddRef
 0001:000080B4       System.TInterfacedObject._Release
 0001:000080DC       System.UnicodeToUtf8
 0001:0000816C       System.Utf8ToUnicode
 0001:000081F0       System.UTF8Encode
 0001:00008310       System.UTF8EncodeToShortString
 0001:0000839C       System.UTF8ToUnicodeString
 0001:00008474       System.UTF8ToUnicodeString
 0001:00008508       System.UTF8ToString
 0001:0000851C       System.LoadResString
 0001:00008588       System.GetACP
 0001:00008590       System.GetCPUCount
 0001:000085A4       System.SetUtf8CompareLocale
 0001:000085E0       System.LocalAlloc
 0001:000085E8       System.LocalFree
 0001:000085F0       System.LoadLibraryA
 0001:000085F8       System.lstrcmpiA
 0001:00008600       System.@memcpy
 0001:00008614       System.@memset
 0001:00008628       System...
 0001:0000870E       System.@_delayLoadHelper
 0001:00008972       System.@_FUnloadDelayLoadedDLL
 0001:000089DC       System.@InitDelayHelp
 0001:000089EB       System.@ShutdownDelayHelp
 0001:00008A04       System.Finalization
 0001:00008A78       SysInit.GetModuleHandle
 0001:00008A80       SysInit.LocalAlloc
 0001:00008A88       SysInit.TlsGetValue
 0001:00008A90       SysInit.TlsSetValue
 0001:00008A98       SysInit.AllocTlsBuffer
 0001:00008AA4       SysInit.GetTlsSize
 0001:00008AAC       SysInit.InitThreadTLS
 0001:00008AF0       SysInit.@GetTls
 0001:00008B30       SysInit.InitializeModule
 0001:00008B3C       SysInit.@InitExe
 0001:00008F50       Windows.RegCloseKey
 0001:00008F58       Windows.RegConnectRegistry
 0001:00008F60       Windows.RegCreateKeyEx
 0001:00008F68       Windows.RegDeleteKey
 0001:00008F70       Windows.RegDeleteValue
 0001:00008F78       Windows.RegEnumKeyEx
 0001:00008F80       Windows.RegEnumValue
 0001:00008F88       Windows.RegFlushKey
 0001:00008F90       Windows.RegLoadKey
 0001:00008F98       Windows.RegOpenKeyEx
 0001:00008FA0       Windows.RegQueryInfoKey
 0001:00008FA8       Windows.RegQueryValueEx
 0001:00008FB0       Windows.RegReplaceKey
 0001:00008FB8       Windows.RegRestoreKey
 0001:00008FC0       Windows.RegSaveKey
 0001:00008FC8       Windows.RegSetValueEx
 0001:00008FD0       Windows.RegUnLoadKey
 0001:00008FD8       Windows.CloseHandle
 0001:00008FE0       Windows.CompareString
 0001:00008FE8       Windows.CompareStringW
 0001:00008FF0       Windows.CreateEvent
 0001:00008FF8       Windows.CreateFile
 0001:00009000       Windows.DeleteCriticalSection
 0001:00009008       Windows.EnterCriticalSection
 0001:00009010       Windows.EnumCalendarInfo
 0001:00009018       Windows.FileTimeToDosDateTime
 0001:00009020       Windows.FileTimeToLocalFileTime
 0001:00009028       Windows.FileTimeToSystemTime
 0001:00009030       Windows.FindClose
 0001:00009038       Windows.FindFirstFile
 0001:00009040       Windows.FindNextFile
 0001:00009048       Windows.FindResource
 0001:00009050       Windows.FormatMessage
 0001:00009058       Windows.FreeLibrary
 0001:00009060       Windows.InterlockedCompareExchange
 0001:00009068       Windows.InterlockedCompareExchangePointer
 0001:00009080       Windows.InterlockedExchange
 0001:00009088       Windows.InterlockedExchangeAdd
 0001:00009090       Windows.InterlockedIncrement
 0001:00009098       Windows.FreeResource
 0001:000090A0       Windows.GetCPInfo
 0001:000090A8       Windows.GetCurrentProcess
 0001:000090B0       Windows.GetCurrentThread
 0001:000090B8       Windows.GetCurrentThreadId
 0001:000090C0       Windows.GetDateFormat
 0001:000090C8       Windows.GetDiskFreeSpace
 0001:000090D0       Windows.GetExitCodeThread
 0001:000090D8       Windows.GetFileAttributes
 0001:000090E0       Windows.GetFullPathName
 0001:000090E8       Windows.GetLastError
 0001:000090F0       Windows.GetLocalTime
 0001:000090F8       Windows.GetLocaleInfo
 0001:00009100       Windows.GetModuleFileName
 0001:00009108       Windows.GetModuleHandle
 0001:00009110       Windows.GetProcAddress
 0001:00009118       Windows.GetProcAddress
 0001:0000918C       Windows.GetStdHandle
 0001:00009194       Windows.GetThreadLocale
 0001:0000919C       Windows.GetThreadPriority
 0001:000091A4       Windows.GetVersionEx
 0001:000091AC       Windows.InitializeCriticalSection
 0001:000091B4       Windows.LeaveCriticalSection
 0001:000091BC       Windows.LoadLibrary
 0001:000091C4       Windows.LoadResource
 0001:000091CC       Windows.LockResource
 0001:000091D4       Windows.MultiByteToWideChar
 0001:000091DC       Windows.IsDebuggerPresent
 0001:000091E4       Windows.RaiseException
 0001:000091EC       Windows.ReadFile
 0001:000091F4       Windows.ResetEvent
 0001:000091FC       Windows.ResumeThread
 0001:00009204       Windows.SetEndOfFile
 0001:0000920C       Windows.SetEvent
 0001:00009214       Windows.SetFilePointer
 0001:0000921C       Windows.SetLastError
 0001:00009224       Windows.SetThreadPriority
 0001:0000922C       Windows.SignalObjectAndWait
 0001:00009234       Windows.SizeofResource
 0001:0000923C       Windows.SuspendThread
 0001:00009244       Windows.SwitchToThread
 0001:0000924C       Windows.TryEnterCriticalSection
 0001:00009254       Windows.VirtualFree
 0001:0000925C       Windows.VirtualQuery
 0001:00009264       Windows.VirtualQueryEx
 0001:0000926C       Windows.WaitForSingleObject
 0001:00009274       Windows.WideCharToMultiByte
 0001:0000927C       Windows.WriteFile
 0001:00009284       Windows.BeginDeferWindowPos
 0001:0000928C       Windows.BeginPaint
 0001:00009294       Windows.CallWindowProc
 0001:0000929C       Windows.CharNext
 0001:000092A4       Windows.CharUpperBuff
 0001:000092AC       Windows.DefWindowProc
 0001:000092B4       Windows.DeferWindowPos
 0001:000092BC       Windows.EnableWindow
 0001:000092C4       Windows.EndDeferWindowPos
 0001:000092CC       Windows.EndPaint
 0001:000092D4       Windows.GetClientRect
 0001:000092DC       Windows.GetSystemMetrics
 0001:000092E4       Windows.GetWindowLong
 0001:000092EC       Windows.LoadCursor
 0001:000092F4       Windows.LoadIcon
 0001:000092FC       Windows.LoadString
 0001:00009304       Windows.MessageBox
 0001:0000930C       Windows.MsgWaitForMultipleObjects
 0001:00009314       Windows.PeekMessage
 0001:0000931C       Windows.PostMessage
 0001:00009324       Windows.PostQuitMessage
 0001:0000932C       Windows.RegisterClass
 0001:00009334       Windows.SendMessageW
 0001:0000933C       Windows.SetTimer
 0001:00009344       Windows.SetWindowLong
 0001:0000934C       Windows.SetWindowTextW
 0001:00009354       Windows.ShowWindow
 0001:0000935C       Windows.UpdateWindow
 0001:00009364       Windows._CreateWindowEx
 0001:0000936C       Windows._CreateWindowExW
 0001:00009374       Windows.CreateWindow
 0001:000093CC       Windows.CreateWindowW
 0001:00009424       Windows.InitVersionInfo
 0001:00009460       Windows.Finalization
 0001:00009910       Character.TCharacter.CheckLetter
 0001:0000991C       Character.TCharacter.CheckLetterOrDigit
 0001:0000992C       Character.TCharacter.IsLatin1
 0001:00009938       Character.TCharacter.IsLetter
 0001:000099C4       Character.TCharacter.IsLetterOrDigit
 0001:00009A2C       Character.TCharacter.IsAscii
 0001:00009A38       Character.TCharacter.Initialize
 0001:00009AE0       StrUtils.PosEx
 0001:00009E14       SysUtils..Exception
 0001:0000A3DC       SysUtils..EHeapException
 0001:0000A4D0       SysUtils..EOutOfMemory
 0001:0000A56C       SysUtils..EInOutError
 0001:0000A624       SysUtils..EExternal
 0001:0000A6DC       SysUtils..EExternalException
 0001:0000A784       SysUtils..EIntError
 0001:0000A818       SysUtils..EDivByZero
 0001:0000A8B0       SysUtils..ERangeError
 0001:0000A948       SysUtils..EIntOverflow
 0001:0000A9E4       SysUtils..EMathError
 0001:0000AA7C       SysUtils..EInvalidOp
 0001:0000AB14       SysUtils..EZeroDivide
 0001:0000ABAC       SysUtils..EOverflow
 0001:0000AC40       SysUtils..EUnderflow
 0001:0000ACD8       SysUtils..EInvalidPointer
 0001:0000AD78       SysUtils..EInvalidCast
 0001:0000AE14       SysUtils..EConvertError
 0001:0000AEB0       SysUtils..EAccessViolation
 0001:0000AF54       SysUtils..EPrivilege
 0001:0000AFEC       SysUtils..EStackOverflow
 0001:0000B08C       SysUtils..EControlC
 0001:0000B120       SysUtils..EVariantError
 0001:0000B1BC       SysUtils..EAssertionFailed
 0001:0000B260       SysUtils..EAbstractError
 0001:0000B300       SysUtils..EIntfCastError
 0001:0000B3A0       SysUtils..EOSError
 0001:0000B450       SysUtils..ESafecallException
 0001:0000B4F8       SysUtils..EMonitor
 0001:0000B58C       SysUtils..EMonitorLockException
 0001:0000B638       SysUtils..ENoMonitorSupportException
 0001:0000B7D8       SysUtils..TThreadLocalCounter
 0001:0000B9FC       SysUtils..TMultiReadExclusiveWriteSynchronizer
 0001:0000BD04       SysUtils..EEncodingError
 0001:0000BDA4       SysUtils..TEncoding
 0001:0000C714       SysUtils.TEncoding.GetMaxByteCount
 0001:0000C71C       SysUtils.TEncoding.GetMaxCharCount
 0001:0000C724       SysUtils.TEncoding.GetPreamble
 0001:0000C72C       SysUtils..TMBCSEncoding
 0001:0000C9F0       SysUtils..TUTF7Encoding
 0001:0000CB70       SysUtils..TUTF8Encoding
 0001:0000CD30       SysUtils..TUnicodeEncoding
 0001:0000CEF0       SysUtils..TBigEndianUnicodeEncoding
 0001:0000CFFC       SysUtils.DivMod
 0001:0000D018       SysUtils.ConvertError
 0001:0000D030       SysUtils.ConvertErrorFmt
 0001:0000D054       SysUtils.UpperCaseFromAnsiString
 0001:0000D0A4       SysUtils.UpperCase
 0001:0000D11C       SysUtils.LowerCaseFromAnsiString
 0001:0000D16C       SysUtils.LowerCase
 0001:0000D1E4       SysUtils.CompareStr
 0001:0000D2A4       SysUtils.CompareMem
 0001:0000D338       SysUtils.CompareText
 0001:0000D434       SysUtils.SameText
 0001:0000D458       SysUtils.AnsiUpperCase
 0001:0000D4E8       SysUtils.AnsiCompareStr
 0001:0000D5B4       SysUtils.AnsiCompareText
 0001:0000D680       SysUtils.Trim
 0001:0000D740       SysUtils.AnsiQuotedStr
 0001:0000D8E0       SysUtils.AnsiExtractQuotedStr
 0001:0000DA1C       SysUtils.IsValidIdent
 0001:0000DBC8       SysUtils.CvtInt
 0001:0000DC14       SysUtils.CvtIntW
 0001:0000DC74       SysUtils.IntToStr
 0001:0000DC94       SysUtils.UIntToStr
 0001:0000DCD0       SysUtils.CvtInt64W
 0001:0000DDB4       SysUtils.CvtInt64
 0001:0000DE80       SysUtils.IntToStr
 0001:0000DEA8       SysUtils.IntToHex
 0001:0000DED0       SysUtils.StrToInt
 0001:0000DF0C       SysUtils.StrToIntDef
 0001:0000DF24       SysUtils.TryStrToInt
 0001:0000DF44       SysUtils.TryStrToInt64
 0001:0000DF64       SysUtils.VerifyBoolStrArray
 0001:0000E004       SysUtils.CompareWith
 0001:0000E054       SysUtils.TryStrToBool
 0001:0000E0FC       SysUtils.BoolToStr
 0001:0000E190       SysUtils.EnumStringModules
 0001:0000E1CC       SysUtils.FindStringResource
 0001:0000E244       SysUtils.LoadStr
 0001:0000E258       SysUtils.FileOpen
 0001:0000E2B0       SysUtils.FileCreate
 0001:0000E2F4       SysUtils.FileRead
 0001:0000E320       SysUtils.FileWrite
 0001:0000E34C       SysUtils.FileSeek
 0001:0000E39C       SysUtils.DirectoryExists
 0001:0000E3C0       SysUtils.FindMatchingFile
 0001:0000E444       SysUtils.FindFirst
 0001:0000E494       SysUtils.FindNext
 0001:0000E4B8       SysUtils.FindClose
 0001:0000E4D4       SysUtils.LastDelimiter
 0001:0000E5B0       SysUtils.ExtractFileName
 0001:0000E5F0       SysUtils.ExtractFileExt
 0001:0000E6A4       SysUtils.ExpandFileName
 0001:0000E738       SysUtils.BackfillGetDiskFreeSpaceEx
 0001:0000E7AC       SysUtils.StrLen
 0001:0000E7DC       SysUtils.StrLen
 0001:0000E7FC       SysUtils.StrEnd
 0001:0000E818       SysUtils.StrMove
 0001:0000E828       SysUtils.StrLCopy
 0001:0000E864       SysUtils.StrLComp
 0001:0000E8B0       SysUtils.StrLIComp
 0001:0000E91C       SysUtils.StrScan
 0001:0000E938       SysUtils.StrRScan
 0001:0000E968       SysUtils.StrPos
 0001:0000E9C0       SysUtils.StrPosLen
 0001:0000EA20       SysUtils.WideStrAlloc
 0001:0000EA38       SysUtils.StrNew
 0001:0000EA64       SysUtils.FormatError
 0001:0000EAAC       SysUtils.FormatBuf
 0001:0000EAC8       SysUtils.StrLFmt
 0001:0000EB0C       SysUtils.Format
 0001:0000EB20       SysUtils.FmtStr
 0001:0000ECB8       SysUtils.WideFormatError
 0001:0000ED38       SysUtils.WideFormatVarToStr
 0001:0000ED5C       SysUtils.WideFloatToText
 0001:0000ED78       SysUtils.WideFormatBuf
 0001:0000F15C       SysUtils.PutExponent
 0001:0000F1C0       SysUtils.FloatToText
 0001:0000F4C0       SysUtils.FloatToDecimal
 0001:0000F6EC       SysUtils.TextToFloat
 0001:0000F800       SysUtils.TextToFloat
 0001:0000F864       SysUtils.FloatToStr
 0001:0000F894       SysUtils.CurrToStr
 0001:0000F8C4       SysUtils.TryStrToFloat
 0001:0000F8E0       SysUtils.TryStrToFloat
 0001:0000F950       SysUtils.TryStrToFloat
 0001:0000F9C0       SysUtils.TryStrToCurr
 0001:0000F9DC       SysUtils.DateTimeToTimeStamp
 0001:0000FA20       SysUtils.TryEncodeTime
 0001:0000FA90       SysUtils.EncodeTime
 0001:0000FAD0       SysUtils.DecodeTime
 0001:0000FB2C       SysUtils.IsLeapYear
 0001:0000FB68       SysUtils.TryEncodeDate
 0001:0000FC34       SysUtils.EncodeDate
 0001:0000FC64       SysUtils.DecodeDateFully
 0001:0000FDB0       SysUtils.DecodeDate
 0001:0000FDD0       SysUtils.DateTimeToSystemTime
 0001:0000FE10       SysUtils.SystemTimeToDateTime
 0001:0000FE80       SysUtils.DayOfWeek
 0001:0000FEA8       SysUtils.CurrentYear
 0001:0000FEBC       SysUtils.AppendChars
 0001:0000FF00       SysUtils.AppendString
 0001:0000FF74       SysUtils.AppendNumber
 0001:0000FFC0       SysUtils.GetCount
 0001:0000FFF4       SysUtils.GetDate
 0001:0001002C       SysUtils.GetTime
 0001:0001006C       SysUtils.ConvertEraString
 0001:000101F8       SysUtils.ConvertYearString
 0001:00010324       SysUtils.AppendFormat
 0001:00010B18       SysUtils.DateTimeToString
 0001:00010B74       SysUtils.ScanBlanks
 0001:00010BE0       SysUtils.ScanNumber
 0001:00010CA8       SysUtils.ScanString
 0001:00010D88       SysUtils.ScanChar
 0001:00010E34       SysUtils.GetDateOrder
 0001:00010ECC       SysUtils.ScanToNumber
 0001:00010F90       SysUtils.GetEraYearOffset
 0001:00010FE4       SysUtils.EraToYear
 0001:00011040       SysUtils.ScanDate
 0001:000113F8       SysUtils.ScanTime
 0001:00011600       SysUtils.TryStrToDate
 0001:00011690       SysUtils.TryStrToTime
 0001:00011720       SysUtils.TryStrToDateTime
 0001:00011950       SysUtils.SysErrorMessage
 0001:000119A0       SysUtils.GetLocaleStr
 0001:000119EC       SysUtils.GetLocaleChar
 0001:00011A18       SysUtils.LocalGetLocaleStr
 0001:00011A58       SysUtils.GetMonthDayNames
 0001:00011B7C       SysUtils.EnumEraNames
 0001:00011BB8       SysUtils.EnumEraYearOffsets
 0001:00011C30       SysUtils.GetEraNamesAndYearOffsets
 0001:00011CE4       SysUtils.TranslateDateFormat
 0001:00011FA4       SysUtils.ConvertAddr
 0001:00011FB0       SysUtils.ExceptionErrorMessage
 0001:000121A0       SysUtils.ShowException
 0001:000122E4       SysUtils.Exception.Create
 0001:00012320       SysUtils.Exception.CreateFmt
 0001:000123A0       SysUtils.Exception.CreateRes
 0001:00012418       SysUtils.Exception.CreateRes
 0001:00012454       SysUtils.Exception.CreateResFmt
 0001:000124E8       SysUtils.Exception.CreateResFmt
 0001:0001257C       SysUtils.Exception.CreateHelp
 0001:000125C4       SysUtils.Exception.CreateFmtHelp
 0001:0001264C       SysUtils.Exception.CreateResHelp
 0001:000126CC       SysUtils.Exception.CreateResHelp
 0001:00012714       SysUtils.Exception.CreateResFmtHelp
 0001:000127B0       SysUtils.Exception.CreateResFmtHelp
 0001:0001284C       SysUtils.Exception.Destroy
 0001:00012890       SysUtils.Exception.GetBaseException
 0001:0001289C       SysUtils.Exception.GetStackTrace
 0001:000128C8       SysUtils.Exception.RaiseOuterException
 0001:000128DC       SysUtils.Exception.ThrowOuterException
 0001:000128F0       SysUtils.Exception.RaisingException
 0001:0001291C       SysUtils.Exception.SetInnerException
 0001:00012944       SysUtils.Exception.SetStackInfo
 0001:00012948       SysUtils.Exception.ToString
 0001:000129A0       SysUtils.EHeapException.FreeInstance
 0001:000129AC       SysUtils.EHeapException.RaisingException
 0001:000129FC       SysUtils.CreateInOutError
 0001:00012BFC       SysUtils.ErrorHandler
 0001:00012C54       SysUtils.CreateAssertException
 0001:00012D00       SysUtils.RaiseAssertException
 0001:00012D10       SysUtils.AssertErrorHandler
 0001:00012D2C       SysUtils.AbstractErrorHandler
 0001:00012D44       SysUtils.MapException
 0001:00012DC4       SysUtils.GetExceptionClass
 0001:00012DE4       SysUtils.CreateAVObject
 0001:00012FB0       SysUtils.GetExceptionObject
 0001:00013088       SysUtils.RaiseExceptObject
 0001:000130AC       SysUtils.ExceptHandler
 0001:000130BC       SysUtils.InitExceptions
 0001:0001314C       SysUtils.DoneExceptions
 0001:000131CC       SysUtils.Exception.Destroy@
 0001:000131DC       SysUtils.Push
 0001:000131FC       SysUtils.Pop
 0001:0001321C       SysUtils.NewSyncObj
 0001:00013280       SysUtils.FreeSyncObj
 0001:000132A8       SysUtils.NewWaitObj
 0001:000132E8       SysUtils.FreeWaitObj
 0001:00013314       SysUtils.WaitAndOrSignalObj
 0001:0001334C       SysUtils.InitMonitorSupport
 0001:00013358       SysUtils.CleanStack
 0001:00013388       SysUtils.CleanEventList
 0001:000133B4       SysUtils.DoneMonitorSupport
 0001:000133EC       SysUtils.InitPlatformId
 0001:0001345C       SysUtils.ByteType
 0001:0001356C       SysUtils.ElementToCharLen
 0001:00013610       SysUtils.ByteToCharLen
 0001:00013618       SysUtils.ElementToCharIndex
 0001:000136F8       SysUtils.ByteToCharIndex
 0001:00013700       SysUtils.CountChars
 0001:00013820       SysUtils.CharToElementIndex
 0001:00013900       SysUtils.CharToByteIndex
 0001:00013908       SysUtils.CharToElementLen
 0001:00013A18       SysUtils.CharToByteLen
 0001:00013A20       SysUtils.StrCharLength
 0001:00013A50       SysUtils.StrNextChar
 0001:00013A80       SysUtils.CharLength
 0001:00013B14       SysUtils.NextCharIndex
 0001:00013BB0       SysUtils.IsPathDelimiter
 0001:00013C70       SysUtils.IncludeTrailingPathDelimiter
 0001:00013CC0       SysUtils.AnsiPos
 0001:00013DA0       SysUtils.AnsiStrPos
 0001:00013DA8       SysUtils.AnsiStrRScan
 0001:00013DB0       SysUtils.AnsiStrScan
 0001:00013DB8       SysUtils.InitLeadBytes
 0001:00013E14       SysUtils.InitSysLocale
 0001:00013ECC       SysUtils.GetFormatSettings
 0001:000142B8       SysUtils.StringReplace
 0001:000145B0       SysUtils.HashNameMBCS
 0001:00014644       SysUtils.HashName
 0001:0001467C       SysUtils.ModuleUnloaded
 0001:00014794       SysUtils.Sleep
 0001:0001479C       SysUtils.RaiseLastOSError
 0001:000147A8       SysUtils.RaiseLastOSError
 0001:00014840       SysUtils.Win32Check
 0001:00014850       SysUtils.FreeTerminateProcs
 0001:00014874       SysUtils.InitDriveSpacePtr
 0001:000148F0       SysUtils.InterlockedIncrement
 0001:000148FC       SysUtils.InterlockedDecrement
 0001:00014908       SysUtils.InterlockedExchange
 0001:00014910       SysUtils.InterlockedExchangeAdd
 0001:00014918       SysUtils.TThreadLocalCounter.Destroy
 0001:00014970       SysUtils.TThreadLocalCounter.HashIndex
 0001:0001498C       SysUtils.TThreadLocalCounter.Open
 0001:00014A04       SysUtils.TThreadLocalCounter.Close
 0001:00014A0C       SysUtils.TThreadLocalCounter.Delete
 0001:00014A1C       SysUtils.TThreadLocalCounter.Recycle
 0001:00014A60       SysUtils.TMultiReadExclusiveWriteSynchronizer.Create
 0001:00014AD4       SysUtils.TMultiReadExclusiveWriteSynchronizer.Destroy
 0001:00014B1C       SysUtils.TMultiReadExclusiveWriteSynchronizer.BlockReaders
 0001:00014B28       SysUtils.TMultiReadExclusiveWriteSynchronizer.UnblockReaders
 0001:00014B34       SysUtils.TMultiReadExclusiveWriteSynchronizer.UnblockOneWriter
 0001:00014B40       SysUtils.TMultiReadExclusiveWriteSynchronizer.WaitForReadSignal
 0001:00014B50       SysUtils.TMultiReadExclusiveWriteSynchronizer.WaitForWriteSignal
 0001:00014B60       SysUtils.TMultiReadExclusiveWriteSynchronizer.BeginWrite
 0001:00014C0C       SysUtils.TMultiReadExclusiveWriteSynchronizer.EndWrite
 0001:00014C5C       SysUtils.TMultiReadExclusiveWriteSynchronizer.BeginRead
 0001:00014CCC       SysUtils.TMultiReadExclusiveWriteSynchronizer.EndRead
 0001:00014D34       SysUtils.FreeAndNil
 0001:00014D44       SysUtils.Supports
 0001:00014D68       SysUtils.Supports
 0001:00014E00       SysUtils.ClearHashTables
 0001:00014E30       SysUtils.TEncoding.Convert
 0001:00014EA4       SysUtils.TEncoding.Convert
 0001:00014F20       SysUtils.TEncoding.Destroy@
 0001:00014F34       SysUtils.TEncoding.FreeEncodings
 0001:00014FA4       SysUtils.TEncoding.GetBigEndianUnicode
 0001:00014FE0       SysUtils.ContainsPreamble
 0001:0001503C       SysUtils.TEncoding.GetBufferEncoding
 0001:00015144       SysUtils.TEncoding.GetByteCount
 0001:00015160       SysUtils.TEncoding.GetByteCount
 0001:0001520C       SysUtils.TEncoding.GetByteCount
 0001:00015290       SysUtils.TEncoding.GetByteCount
 0001:00015394       SysUtils.TEncoding.GetBytes
 0001:000153DC       SysUtils.TEncoding.GetBytes
 0001:00015548       SysUtils.TEncoding.GetBytes
 0001:000155EC       SysUtils.TEncoding.GetBytes
 0001:00015790       SysUtils.TEncoding.GetCharCount
 0001:000157AC       SysUtils.TEncoding.GetCharCount
 0001:00015878       SysUtils.TEncoding.GetChars
 0001:0001589C       SysUtils.TEncoding.GetChars
 0001:0001599C       SysUtils.TEncoding.GetChars
 0001:00015AF0       SysUtils.TEncoding.GetDefault
 0001:00015B30       SysUtils.TEncoding.GetEncoding
 0001:00015B40       SysUtils.TEncoding.GetString
 0001:00015B64       SysUtils.TEncoding.GetString
 0001:00015BD4       SysUtils.TEncoding.GetUnicode
 0001:00015C10       SysUtils.TEncoding.GetUTF8
 0001:00015C4C       SysUtils.TEncoding.IsStandardEncoding
 0001:00015C84       SysUtils.TMBCSEncoding.Create
 0001:00015CC4       SysUtils.TMBCSEncoding.Create
 0001:00015D0C       SysUtils.TMBCSEncoding.Create
 0001:00015D88       SysUtils.TMBCSEncoding.GetByteCount
 0001:00015DA0       SysUtils.TMBCSEncoding.GetBytes
 0001:00015DC4       SysUtils.TMBCSEncoding.GetCharCount
 0001:00015DD8       SysUtils.TMBCSEncoding.GetChars
 0001:00015DF8       SysUtils.TMBCSEncoding.GetMaxByteCount
 0001:00015E00       SysUtils.TMBCSEncoding.GetMaxCharCount
 0001:00015E04       SysUtils.TMBCSEncoding.GetPreamble
 0001:00015E20       SysUtils.TUTF7Encoding.Create
 0001:00015E5C       SysUtils.TUTF7Encoding.GetByteCount
 0001:00015E64       SysUtils.TUTF7Encoding.GetBytes
 0001:00015E7C       SysUtils.TUTF7Encoding.GetCharCount
 0001:00015E84       SysUtils.TUTF7Encoding.GetChars
 0001:00015E9C       SysUtils.TUTF7Encoding.GetMaxByteCount
 0001:00015EA4       SysUtils.TUTF7Encoding.GetMaxCharCount
 0001:00015EA8       SysUtils.TUTF8Encoding.Create
 0001:00015EE8       SysUtils.TUTF8Encoding.GetMaxByteCount
 0001:00015EF0       SysUtils.TUTF8Encoding.GetMaxCharCount
 0001:00015EF4       SysUtils.TUTF8Encoding.GetPreamble
 0001:00015F24       SysUtils.TUnicodeEncoding.Create
 0001:00015F50       SysUtils.TUnicodeEncoding.GetByteCount
 0001:00015F58       SysUtils.TUnicodeEncoding.GetBytes
 0001:00015F74       SysUtils.TUnicodeEncoding.GetCharCount
 0001:00015F80       SysUtils.TUnicodeEncoding.GetChars
 0001:00015FA0       SysUtils.TUnicodeEncoding.GetMaxByteCount
 0001:00015FA8       SysUtils.TUnicodeEncoding.GetMaxCharCount
 0001:00015FB8       SysUtils.TUnicodeEncoding.GetPreamble
 0001:00015FE0       SysUtils.TBigEndianUnicodeEncoding.GetBytes
 0001:00016014       SysUtils.TBigEndianUnicodeEncoding.GetChars
 0001:00016050       SysUtils.TBigEndianUnicodeEncoding.GetPreamble
 0001:00016408       SysUtils.Finalization
 0001:000165B0       VarUtils.VariantInit
 0001:000165B8       VarUtils.VariantClear
 0001:000165C0       VarUtils.VariantCopy
 0001:000165C8       VarUtils.VariantChangeType
 0001:000165D0       VarUtils.BackupVariantChangeTypeEx
 0001:00016600       VarUtils.UniUnimplemented
 0001:0001660C       VarUtils.BiUnimplemented
 0001:00016618       VarUtils.CmpUnimplemented
 0001:00016624       VarUtils.BackupVarI4FromStr
 0001:00016690       VarUtils.BackupVarR4FromStr
 0001:000166FC       VarUtils.BackupVarR8FromStr
 0001:00016768       VarUtils.BackupVarDateFromStr
 0001:000167D4       VarUtils.BackupVarCyFromStr
 0001:00016840       VarUtils.BackupVarBoolFromStr
 0001:000168C0       VarUtils.BackupVarBStrFromCy
 0001:00016930       VarUtils.BackupVarBStrFromDate
 0001:000169A4       VarUtils.BackupVarBStrFromBool
 0001:00016A18       VarUtils.SafeArrayCreate
 0001:00016A20       VarUtils.SafeArrayGetLBound
 0001:00016A28       VarUtils.SafeArrayGetUBound
 0001:00016A30       VarUtils.SafeArrayPtrOfIndex
 0001:00016A38       VarUtils.FindProc
 0001:00016A64       VarUtils.InitializeVarUtils
 0001:00016D7C       VarUtils.Finalization
 0001:00016E24       Variants..TCustomVariantType
 0001:00017324       Variants.TCustomVariantType.Clear
 0001:0001732C       Variants.TCustomVariantType.Copy
 0001:00017334       Variants..EVariantInvalidOpError
 0001:000173E4       Variants..EVariantTypeCastError
 0001:00017490       Variants..EVariantOverflowError
 0001:0001753C       Variants..EVariantInvalidArgError
 0001:000175EC       Variants..EVariantBadVarTypeError
 0001:0001769C       Variants..EVariantBadIndexError
 0001:00017748       Variants..EVariantArrayLockedError
 0001:000177FC       Variants..EVariantArrayCreateError
 0001:000178B0       Variants..EVariantNotImplError
 0001:0001795C       Variants..EVariantOutOfMemoryError
 0001:00017A10       Variants..EVariantUnexpectedError
 0001:00017AC0       Variants..EVariantDispatchError
 0001:00017B6C       Variants..EVariantInvalidNullOpError
 0001:00017C24       Variants.VarCastError
 0001:00017C78       Variants.VarCastError
 0001:00017D14       Variants.VarInvalidOp
 0001:00017D68       Variants.VarInvalidNullOp
 0001:00017DBC       Variants.VarOverflowError
 0001:00017E58       Variants.VarArrayCreateError
 0001:00017EAC       Variants.TranslateResult
 0001:00018100       Variants.VarResultCheck
 0001:0001810C       Variants.VarResultCheck
 0001:00018140       Variants.HandleConversionException
 0001:000181C4       Variants.@DispInvokeError
 0001:00018218       Variants.@VarNull
 0001:0001822C       Variants.InBounds
 0001:0001825C       Variants.Increment
 0001:000182B8       Variants.VarArrayClear
 0001:00018434       Variants.VarClearDeep
 0001:000184C8       Variants.@VarClear
 0001:000184DC       Variants.@VarClr
 0001:000184E4       Variants.InBounds
 0001:00018514       Variants.Increment
 0001:00018570       Variants.VarArrayCopyForEach
 0001:0001873C       Variants.VarCopyCopyProc
 0001:00018744       Variants.VarCopyDeep
 0001:00018830       Variants.@VarCopy
 0001:00018874       Variants.VarCastAsAny
 0001:000188E0       Variants.VarCastAsOleStr
 0001:0001892C       Variants.VarCastAsString
 0001:00018978       Variants.VarCastAsUString
 0001:000189C4       Variants.VarCastAsDispatch
 0001:00018A10       Variants.VarCastAsInterface
 0001:00018A5C       Variants.VarCastViaOS
 0001:00018ADC       Variants.VarCastRare
 0001:00018B48       Variants.@VarCast
 0001:00018D9C       Variants.VarToIntAsString
 0001:00018E50       Variants.VarToIntViaOS
 0001:00018E8C       Variants.VarToIntAny
 0001:00018EF0       Variants.VarToIntCustom
 0001:00018F34       Variants.@VarToInteger
 0001:000193E4       Variants.@VarToShortInt
 0001:00019498       Variants.@VarToByte
 0001:00019544       Variants.@VarToSmallInt
 0001:00019640       Variants.@VarToWord
 0001:0001971C       Variants.@VarToLongWord
 0001:00019808       Variants.VarToInt64ViaOS
 0001:000198B4       Variants.VarToInt64AsString
 0001:000199B4       Variants.VarToInt64Any
 0001:00019A20       Variants.VarToInt64Custom
 0001:00019A6C       Variants.@VarToInt64
 0001:00019EFC       Variants.@VarToUInt64
 0001:0001A060       Variants.VarToBoolAsString
 0001:0001A124       Variants.VarToBoolViaOS
 0001:0001A164       Variants.VarToBoolAny
 0001:0001A1C8       Variants.VarToBoolCustom
 0001:0001A214       Variants.@VarToBoolean
 0001:0001A5B0       Variants.@VarToBool
 0001:0001A5BC       Variants.VarToDoubleAsString
 0001:0001A680       Variants.VarToDoubleViaOS
 0001:0001A6CC       Variants.VarToDoubleAny
 0001:0001A730       Variants.VarToDoubleCustom
 0001:0001A77C       Variants.@VarToDouble
 0001:0001AB6C       Variants.@VarToReal
 0001:0001AB88       Variants.@VarToSingle
 0001:0001AD4C       Variants.VarToDateAsString
 0001:0001AE38       Variants.VarToDateAsDouble
 0001:0001AE98       Variants.VarToDateViaOS
 0001:0001AEE4       Variants.VarToDateAny
 0001:0001AF48       Variants.VarToDateCustom
 0001:0001AF94       Variants.@VarToDate
 0001:0001B378       Variants.VarToCurrencyAsString
 0001:0001B434       Variants.VarToCurrencyAsDouble
 0001:0001B494       Variants.VarToCurrencyViaOS
 0001:0001B4E0       Variants.VarToCurrencyAny
 0001:0001B544       Variants.VarToCurrencyCustom
 0001:0001B590       Variants.@VarToCurrency
 0001:0001B9EC       Variants.CurrToWStrViaOS
 0001:0001BA24       Variants.DateToWStrViaOS
 0001:0001BA5C       Variants.BoolToWStrViaOS
 0001:0001BB24       Variants.VarToLStrViaOS
 0001:0001BBDC       Variants.VarToLStrAny
 0001:0001BC40       Variants.VarToLStrCustom
 0001:0001BCC8       Variants.@VarToLStr
 0001:0001C370       Variants.VarToWStrViaOS
 0001:0001C43C       Variants.VarToWStrAny
 0001:0001C4A0       Variants.VarToWStrCustom
 0001:0001C57C       Variants.@VarToWStr
 0001:0001CB78       Variants.VarToUStrAny
 0001:0001CBDC       Variants.VarToUStrCustom
 0001:0001CCA4       Variants.@VarToUStr
 0001:0001D2AC       Variants.AnyToIntf
 0001:0001D324       Variants.@VarToIntf
 0001:0001D3F0       Variants.@VarToDisp
 0001:0001D49C       Variants.@VarFromInt
 0001:0001D4D8       Variants.@VarFromInteger
 0001:0001D4F8       Variants.@VarFromByte
 0001:0001D518       Variants.@VarFromWord
 0001:0001D538       Variants.@VarFromLongWord
 0001:0001D558       Variants.@VarFromUInt64
 0001:0001D584       Variants.@VarFromShortInt
 0001:0001D5A4       Variants.@VarFromSmallInt
 0001:0001D5C4       Variants.@VarFromInt64
 0001:0001D5F0       Variants.@VarFromSingle
 0001:0001D614       Variants.@VarFromDouble
 0001:0001D640       Variants.@VarFromCurrency
 0001:0001D66C       Variants.@VarFromDate
 0001:0001D698       Variants.@VarFromBool
 0001:0001D6C0       Variants.@VarFromReal
 0001:0001D6D4       Variants.@VarFromTDateTime
 0001:0001D6E8       Variants.@VarFromCurr
 0001:0001D6FC       Variants.@VarFromLStr
 0001:0001D728       Variants.@VarFromWStr
 0001:0001D760       Variants.@VarFromUStr
 0001:0001D78C       Variants.@VarFromIntf
 0001:0001D7B8       Variants.@VarFromDisp
 0001:0001D7E4       Variants.CheckType
 0001:0001D810       Variants.VarCompareAny
 0001:0001D8E8       Variants.EmptyCompare
 0001:0001D8FC       Variants.NullCompare
 0001:0001D9F0       Variants.IntCompare
 0001:0001DA04       Variants.Int64Compare
 0001:0001DA40       Variants.UInt64Compare
 0001:0001DA74       Variants.RealCompare
 0001:0001DAA0       Variants.DateCompare
 0001:0001DACC       Variants.CurrCompare
 0001:0001DAFC       Variants.StringCompare
 0001:0001DB68       Variants.VarCompareSimple
 0001:0001DD14       Variants.VarCompareRare
 0001:0001E138       Variants.VarCompare
 0001:0001E1A0       Variants.@VarAddRef
 0001:0001E41C       Variants.VarTypeAsText
 0001:0001E5D0       Variants.FindVarData
 0001:0001E5E0       Variants.VarIsClear
 0001:0001E654       Variants.VarSameValue
 0001:0001E6CC       Variants.SetVarAsError
 0001:0001E6E4       Variants.SetClearVarToEmptyParam
 0001:0001E6F0       Variants.GetVarDataArrayInfo
 0001:0001E734       Variants.VarIsArray
 0001:0001E73C       Variants.VarIsArray
 0001:0001E78C       Variants.ClearVariantTypeList
 0001:0001E7F8       Variants.TCustomVariantType.BinaryOp
 0001:0001E804       Variants.TCustomVariantType.Cast
 0001:0001E83C       Variants.TCustomVariantType.CastTo
 0001:0001E884       Variants.TCustomVariantType.Compare
 0001:0001E890       Variants.TCustomVariantType.CompareOp
 0001:0001E8C8       Variants.TCustomVariantType.CastToOle
 0001:0001E904       Variants.TCustomVariantType.Create
 0001:0001E948       Variants.TCustomVariantType.Create
 0001:0001EBC4       Variants.TCustomVariantType.Destroy
 0001:0001EC50       Variants.TCustomVariantType.IsClear
 0001:0001EC54       Variants.TCustomVariantType.LeftPromotion
 0001:0001EC68       Variants.TCustomVariantType.OlePromotion
 0001:0001EC70       Variants.TCustomVariantType.RaiseCastError
 0001:0001EC78       Variants.TCustomVariantType.RaiseInvalidOp
 0001:0001EC80       Variants.TCustomVariantType.RaiseDispError
 0001:0001EC88       Variants.TCustomVariantType.RightPromotion
 0001:0001EC9C       Variants.TCustomVariantType.UnaryOp
 0001:0001ECA4       Variants.TCustomVariantType.DispInvoke
 0001:0001ECB0       Variants.TCustomVariantType._AddRef
 0001:0001ECBC       Variants.TCustomVariantType._Release
 0001:0001ECC8       Variants.TCustomVariantType.QueryInterface
 0001:0001ECF0       Variants.FindCustomVariantType
 0001:0001EDAC       Variants.FindCustomVariantType
 0001:0001EE80       Variants.Null
 0001:0001EE88       Variants.@VarCmpEQ
 0001:0001EE98       Variants.Finalization
 0001:0001F188       TypInfo.GetPropName
 0001:0001F1D8       TypInfo.GetTypeData
 0001:0001F1E4       TypInfo.GetEnumName
 0001:0001F2DC       TypInfo.UTF8SameText
 0001:0001F350       TypInfo.GetEnumNameValue
 0001:0001F3C8       TypInfo.GetEnumValue
 0001:0001F470       TypInfo.InternalGetPropInfo
 0001:0001F524       TypInfo.GetPropInfo
 0001:0001F578       TypInfo.GetPropInfos
 0001:0001F5CC       TypInfo.IsStoredProp
 0001:0001F5FC       TypInfo.GetOrdProp
 0001:0001F670       TypInfo.SetOrdProp
 0001:0001F6CC       TypInfo.GetSetElementName
 0001:0001F760       TypInfo.GetSetElementValue
 0001:0001F834       TypInfo.GetShortStrProp
 0001:0001F878       TypInfo.SetShortStrProp
 0001:0001F8CC       TypInfo.GetShortStrPropAsLongStr
 0001:0001F8FC       TypInfo.SetShortStrPropAsLongStr
 0001:0001F930       TypInfo.AssignLongStr
 0001:0001F948       TypInfo.GetLongStrProp
 0001:0001F988       TypInfo.SetLongStrProp
 0001:0001F9C8       TypInfo.GetWideStrPropAsLongStr
 0001:0001FA24       TypInfo.SetWideStrPropAsLongStr
 0001:0001FA7C       TypInfo.GetUnicodeStrPropAsLongStr
 0001:0001FAD8       TypInfo.SetUnicodeStrPropAsLongStr
 0001:0001FB30       TypInfo.GetAnsiStrProp
 0001:0001FB7C       TypInfo.SetAnsiStrProp
 0001:0001FBB8       TypInfo.GetWideStrProp
 0001:0001FCCC       TypInfo.SetWideStrProp
 0001:0001FDC8       TypInfo.GetUnicodeStrProp
 0001:0001FEE0       TypInfo.SetRawByteStrProp
 0001:00020034       TypInfo.SetUnicodeStrProp
 0001:00020158       TypInfo.GetFloatProp
 0001:00020270       TypInfo.SetFloatProp
 0001:00020468       TypInfo.AssignVariant
 0001:0002047C       TypInfo.GetVariantProp
 0001:000204BC       TypInfo.SetVariantProp
 0001:000204FC       TypInfo.GetMethodProp
 0001:0002053C       TypInfo.SetMethodProp
 0001:00020574       TypInfo.GetInt64Prop
 0001:0002059C       TypInfo.SetInt64Prop
 0001:000205D8       TypInfo.GetInterfaceProp
 0001:00020658       TypInfo.SetInterfaceProp
 0001:000206CC       TypInfo.Finalization
 0001:000207A4       Classes..EStreamError
 0001:00020840       Classes..EFileStreamError
 0001:0002093C       Classes..EFCreateError
 0001:000209D8       Classes..EFOpenError
 0001:00020A70       Classes..EFilerError
 0001:00020B08       Classes..EReadError
 0001:00020B9C       Classes..EWriteError
 0001:00020C34       Classes..EClassNotFound
 0001:00020CD0       Classes..EInvalidImage
 0001:00020D6C       Classes..EResNotFound
 0001:00020E08       Classes..EListError
 0001:00020E9C       Classes..EStringListError
 0001:00020F40       Classes..EComponentError
 0001:00021144       Classes..TListEnumerator
 0001:00021318       Classes..TList
 0001:00021A2C       Classes..TThreadList
 0001:00021CE4       Classes..TPersistent
 0001:00021E5C       Classes..TCollectionItem
 0001:000220C8       Classes..TCollectionEnumerator
 0001:0002226C       Classes..TCollection
 0001:000227C4       Classes..TStringsEnumerator
 0001:0002296C       Classes..TStrings
 0001:000234E4       Classes.TStrings.Clear
 0001:000234EC       Classes.TStrings.Delete
 0001:000234F4       Classes.TStrings.Insert
 0001:000235E4       Classes..TStringList
 0001:00023C60       Classes..TStream
 0001:0002425C       Classes.TStream.Read
 0001:00024264       Classes.TStream.Write
 0001:0002426C       Classes..THandleStream
 0001:00024484       Classes..TFileStream
 0001:00024668       Classes..TCustomMemoryStream
 0001:000248B0       Classes..TMemoryStream
 0001:00024AF8       Classes..TResourceStream
 0001:00024D70       Classes..TClassFinder
 0001:00025144       Classes..TFiler
 0001:000254F4       Classes.TFiler.DefineProperty
 0001:000254FC       Classes.TFiler.DefineBinaryProperty
 0001:00025504       Classes.TFiler.FlushBuffer
 0001:00025B5C       Classes..TReader
 0001:00026A64       Classes..TWriter
 0001:00027470       Classes..EThread
 0001:00027664       Classes..TThread
 0001:00027E5C       Classes..TComponentEnumerator
 0001:00028234       Classes..TComponent
 0001:00028B7C       Classes..TBasicActionLink
 0001:00028D98       Classes..TBasicAction
 0001:000291A4       Classes..TRegGroup
 0001:00029604       Classes..TRegGroups
 0001:00029AE0       Classes.TRegGroup.AddClass
 0001:00029AEC       Classes.TRegGroup.BestClass
 0001:00029B4C       Classes.TRegGroup.BestGroup
 0001:00029BBC       Classes.TRegGroup.Create
 0001:00029C18       Classes.TRegGroup.Destroy
 0001:00029C58       Classes.TRegGroup.GetClass
 0001:00029CA8       Classes.TRegGroup.GetClasses
 0001:00029CF0       Classes.TRegGroup.IndexOfClass
 0001:00029D68       Classes.TRegGroup.InGroup
 0001:00029DAC       Classes.TRegGroup.RegisterClass
 0001:00029E60       Classes.TRegGroup.RegisterClassAlias
 0001:00029E98       Classes.TRegGroup.Registered
 0001:00029EB0       Classes.TRegGroup.UnregisterClass
 0001:00029F10       Classes.TRegGroup.UnregisterModuleClasses
 0001:0002A050       Classes.TRegGroups.Activate
 0001:0002A09C       Classes.TRegGroups.AddClass
 0001:0002A0BC       Classes.TRegGroups.Create
 0001:0002A130       Classes.TRegGroups.Destroy
 0001:0002A190       Classes.TRegGroups.FindGroup
 0001:0002A1D4       Classes.TRegGroups.GetClass
 0001:0002A218       Classes.TRegGroups.GroupedWith
 0001:0002A238       Classes.Error
 0001:0002A2BC       Classes.TRegGroups.GroupWith
 0001:0002A390       Classes.TRegGroups.Lock
 0001:0002A39C       Classes.TRegGroups.RegisterClass
 0001:0002A3B4       Classes.TRegGroups.RegisterClassAlias
 0001:0002A3D4       Classes.TRegGroups.Registered
 0001:0002A418       Classes.TRegGroups.StartGroup
 0001:0002A468       Classes.TRegGroups.Unlock
 0001:0002A474       Classes.TRegGroups.UnregisterClass
 0001:0002A4A4       Classes.TRegGroups.UnregisterModuleClasses
 0001:0002A4F4       Classes.TClassFinder.Create
 0001:0002A634       Classes.TClassFinder.Destroy
 0001:0002A664       Classes.TClassFinder.GetClass
 0001:0002A700       Classes.TClassFinder.GetClasses
 0001:0002A788       Classes.GetFieldClassTable
 0001:0002A794       Classes.ClassNotFound
 0001:0002A800       Classes.GetClass
 0001:0002A86C       Classes.FindClass
 0001:0002A88C       Classes.UnRegisterModuleClasses
 0001:0002A8F4       Classes.FindIntToIdent
 0001:0002A970       Classes.FindIdentToInt
 0001:0002A9EC       Classes.FindGlobalComponent
 0001:0002AA2C       Classes.IsUniqueGlobalComponentName
 0001:0002AA50       Classes.WriteCollection
 0001:0002AABC       Classes.CollectionsEqual
 0001:0002ABD8       Classes.TListEnumerator.Create
 0001:0002AC1C       Classes.TListEnumerator.GetCurrent
 0001:0002AC28       Classes.TListEnumerator.MoveNext
 0001:0002AC40       Classes.TList.Destroy
 0001:0002AC60       Classes.TList.Add
 0001:0002ACA0       Classes.TList.Clear
 0001:0002ACB8       Classes.TList.Delete
 0001:0002AD20       Classes.ReturnAddr
 0001:0002AD24       Classes.TList.Error
 0001:0002AD5C       Classes.TList.Error
 0001:0002ADB0       Classes.TList.Exchange
 0001:0002AE00       Classes.TList.Expand
 0001:0002AE18       Classes.TList.First
 0001:0002AE20       Classes.TList.Get
 0001:0002AE44       Classes.TList.GetEnumerator
 0001:0002AE54       Classes.TList.Grow
 0001:0002AE88       Classes.TList.IndexOf
 0001:0002AEAC       Classes.TList.IndexOfItem
 0001:0002AED8       Classes.TList.Insert
 0001:0002AF50       Classes.TList.Last
 0001:0002AF74       Classes.TList.Move
 0001:0002AFCC       Classes.TList.Put
 0001:0002B028       Classes.TList.Remove
 0001:0002B030       Classes.TList.RemoveItem
 0001:0002B050       Classes.TList.Pack
 0001:0002B0C4       Classes.TList.SetCapacity
 0001:0002B100       Classes.TList.SetCount
 0001:0002B1A4       Classes.QuickSort
 0001:0002B2DC       Classes..TList.Sort$ActRec
 0001:0002B394       Classes.TList.Sort$ActRec.$0$Body
 0001:0002B3A0       Classes.TList.Sort
 0001:0002B420       Classes.TList.SortList
 0001:0002B440       Classes.TList.Extract
 0001:0002B448       Classes.TList.ExtractItem
 0001:0002B498       Classes.TList.Notify
 0001:0002B49C       Classes.TList.Assign
 0001:0002B768       Classes.TThreadList.Create
 0001:0002B7BC       Classes.TThreadList.Destroy
 0001:0002B838       Classes.TThreadList.Add
 0001:0002B8C0       Classes.TThreadList.Clear
 0001:0002B908       Classes.TThreadList.LockList
 0001:0002B91C       Classes.TThreadList.Remove
 0001:0002B924       Classes.TThreadList.RemoveItem
 0001:0002B978       Classes.TThreadList.UnlockList
 0001:0002B984       Classes.TPersistent.Destroy
 0001:0002B9B0       Classes.TPersistent.Assign
 0001:0002B9C4       Classes.TPersistent.AssignError
 0001:0002BA80       Classes.TPersistent.AssignTo
 0001:0002BA88       Classes.TPersistent.DefineProperties
 0001:0002BA8C       Classes.TPersistent.GetNamePath
 0001:0002BB24       Classes.TPersistent.GetOwner
 0001:0002BB28       Classes.GetDesigner
 0001:0002BBCC       Classes.NotifyDesigner
 0001:0002BC30       Classes.TCollectionItem.Create
 0001:0002BC68       Classes.TCollectionItem.Destroy
 0001:0002BC98       Classes.TCollectionItem.Changed
 0001:0002BCBC       Classes.TCollectionItem.GetIndex
 0001:0002BCD4       Classes.TCollectionItem.GetDisplayName
 0001:0002BCE8       Classes.TCollectionItem.GetNamePath
 0001:0002BD94       Classes.TCollectionItem.GetOwner
 0001:0002BD98       Classes.TCollectionItem.SetCollection
 0001:0002BDC0       Classes.TCollectionItem.SetDisplayName
 0001:0002BDC8       Classes.TCollectionItem.SetIndex
 0001:0002BDF8       Classes.TCollectionEnumerator.Create
 0001:0002BE3C       Classes.TCollectionEnumerator.GetCurrent
 0001:0002BE48       Classes.TCollectionEnumerator.MoveNext
 0001:0002BE64       Classes.TCollection.Create
 0001:0002BEB0       Classes.TCollection.Destroy
 0001:0002BEFC       Classes.TCollection.Add
 0001:0002BF1C       Classes.TCollection.Assign
 0001:0002BFC4       Classes.TCollection.BeginUpdate
 0001:0002BFC8       Classes.TCollection.Changed
 0001:0002BFD8       Classes.TCollection.Clear
 0001:0002C040       Classes.TCollection.EndUpdate
 0001:0002C04C       Classes.TCollection.FindItemID
 0001:0002C07C       Classes.TCollection.GetAttrCount
 0001:0002C080       Classes.TCollection.GetAttr
 0001:0002C090       Classes.TCollection.GetEnumerator
 0001:0002C0A0       Classes.TCollection.GetCapacity
 0001:0002C0A8       Classes.TCollection.GetItemAttr
 0001:0002C0C8       Classes.TCollection.GetCount
 0001:0002C0D0       Classes.TCollection.GetItem
 0001:0002C0E4       Classes.TCollection.GetNamePath
 0001:0002C198       Classes.TCollection.GetPropName
 0001:0002C2EC       Classes.TCollection.Insert
 0001:0002C308       Classes.TCollection.InsertItem
 0001:0002C370       Classes.TCollection.RemoveItem
 0001:0002C3C4       Classes.TCollection.SetCapacity
 0001:0002C3D4       Classes.TCollection.SetItemName
 0001:0002C3D8       Classes.TCollection.Update
 0001:0002C3DC       Classes.TCollection.Delete
 0001:0002C40C       Classes.TCollection.Owner
 0001:0002C418       Classes.TCollection.Added
 0001:0002C41C       Classes.TCollection.Deleting
 0001:0002C420       Classes.TCollection.Notify
 0001:0002C444       Classes.TStringsEnumerator.Create
 0001:0002C488       Classes.TStringsEnumerator.GetCurrent
 0001:0002C4A0       Classes.TStringsEnumerator.MoveNext
 0001:0002C4BC       Classes.TStrings.Destroy
 0001:0002C4EC       Classes.TStrings.Add
 0001:0002C510       Classes.TStrings.AddObject
 0001:0002C534       Classes.TStrings.Append
 0001:0002C540       Classes.TStrings.AddStrings
 0001:0002C5F8       Classes.TStrings.Assign
 0001:0002C6B4       Classes.TStrings.BeginUpdate
 0001:0002C6CC       Classes.DoWrite
 0001:0002C724       Classes.TStrings.DefineProperties
 0001:0002C77C       Classes.TStrings.EndUpdate
 0001:0002C790       Classes.TStrings.Equals
 0001:0002C838       Classes.ReturnAddr
 0001:0002C83C       Classes.TStrings.Error
 0001:0002C874       Classes.TStrings.Error
 0001:0002C8CC       Classes.TStrings.Exchange
 0001:0002C9B8       Classes.TStrings.GetCapacity
 0001:0002C9C0       Classes.TStrings.GetCommaText
 0001:0002CA58       Classes.TStrings.GetDelimitedText
 0001:0002CCC8       Classes.TStrings.GetEnumerator
 0001:0002CCD8       Classes.TStrings.GetObject
 0001:0002CCDC       Classes.TStrings.GetText
 0001:0002CD30       Classes.TStrings.GetTextStr
 0001:0002CEC8       Classes.TStrings.IndexOf
 0001:0002CF54       Classes.TStrings.IndexOfName
 0001:0002D028       Classes.TStrings.IndexOfObject
 0001:0002D05C       Classes.TStrings.InsertObject
 0001:0002D08C       Classes.TStrings.LoadFromFile
 0001:0002D0E0       Classes.TStrings.LoadFromFile
 0001:0002D13C       Classes.TStrings.LoadFromStream
 0001:0002D148       Classes.TStrings.LoadFromStream
 0001:0002D23C       Classes.TStrings.Move
 0001:0002D2EC       Classes.TStrings.Put
 0001:0002D31C       Classes.TStrings.PutObject
 0001:0002D320       Classes.TStrings.ReadData
 0001:0002D3D0       Classes.TStrings.SaveToFile
 0001:0002D3E0       Classes.TStrings.SaveToFile
 0001:0002D440       Classes.TStrings.SaveToStream
 0001:0002D450       Classes.TStrings.SaveToStream
 0001:0002D508       Classes.TStrings.SetCapacity
 0001:0002D50C       Classes.TStrings.SetCommaText
 0001:0002D534       Classes.TStrings.SetStringsAdapter
 0001:0002D568       Classes.TStrings.SetText
 0001:0002D5B8       Classes.TStrings.SetTextStr
 0001:0002D764       Classes.TStrings.SetUpdateState
 0001:0002D768       Classes.TStrings.WriteData
 0001:0002D7EC       Classes.TStrings.SetDelimitedText
 0001:0002D99C       Classes.TStrings.GetDelimiter
 0001:0002D9B8       Classes.TStrings.GetLineBreak
 0001:0002D9F4       Classes.TStrings.GetQuoteChar
 0001:0002DA10       Classes.TStrings.GetStrictDelimiter
 0001:0002DA28       Classes.TStrings.SetDelimiter
 0001:0002DA48       Classes.TStrings.SetLineBreak
 0001:0002DA74       Classes.TStrings.SetQuoteChar
 0001:0002DA94       Classes.TStrings.SetStrictDelimiter
 0001:0002DAB0       Classes.TStrings.CompareStrings
 0001:0002DABC       Classes.TStrings.GetNameValueSeparator
 0001:0002DAD8       Classes.TStrings.SetNameValueSeparator
 0001:0002DAF8       Classes.TStringList.Destroy
 0001:0002DB7C       Classes.TStringList.Add
 0001:0002DB8C       Classes.TStringList.AddObject
 0001:0002DBF0       Classes.TStringList.Changed
 0001:0002DC0C       Classes.TStringList.Changing
 0001:0002DC28       Classes.TStringList.Clear
 0001:0002DC90       Classes.TStringList.Delete
 0001:0002DD10       Classes.TStringList.Exchange
 0001:0002DD6C       Classes.TStringList.ExchangeItems
 0001:0002DD90       Classes.TStringList.Find
 0001:0002DE14       Classes.TStringList.Get
 0001:0002DE44       Classes.TStringList.GetCapacity
 0001:0002DE48       Classes.TStringList.GetCount
 0001:0002DE4C       Classes.TStringList.GetObject
 0001:0002DE70       Classes.TStringList.Grow
 0001:0002DEA4       Classes.TStringList.IndexOf
 0001:0002DEE0       Classes.TStringList.Insert
 0001:0002DEF0       Classes.TStringList.InsertObject
 0001:0002DF44       Classes.TStringList.InsertItem
 0001:0002DFC0       Classes.TStringList.Put
 0001:0002E018       Classes.TStringList.PutObject
 0001:0002E054       Classes.TStringList.QuickSort
 0001:0002E0EC       Classes.TStringList.SetCapacity
 0001:0002E12C       Classes.TStringList.SetSorted
 0001:0002E14C       Classes.TStringList.SetUpdateState
 0001:0002E16C       Classes.StringListCompareStrings
 0001:0002E18C       Classes.TStringList.Sort
 0001:0002E19C       Classes.TStringList.CustomSort
 0001:0002E1D4       Classes.TStringList.CompareStrings
 0001:0002E1F0       Classes.TStringList.Create
 0001:0002E228       Classes.TStringList.Create
 0001:0002E26C       Classes.TStringList.SetCaseSensitive
 0001:0002E294       Classes.TStream.GetPosition
 0001:0002E2B4       Classes.TStream.SetPosition
 0001:0002E2C8       Classes.TStream.GetSize
 0001:0002E314       Classes.TStream.SetSize
 0001:0002E318       Classes.TStream.SetSize64
 0001:0002E32C       Classes.TStream.SetSize
 0001:0002E380       Classes.RaiseException
 0001:0002E3F4       Classes.TStream.Seek
 0001:0002E478       Classes.TStream.Seek
 0001:0002E4E8       Classes.TStream.ReadBuffer
 0001:0002E520       Classes.TStream.WriteBuffer
 0001:0002E558       Classes.TStream.CopyFrom
 0001:0002E64C       Classes.TStream.ReadComponent
 0001:0002E6AC       Classes.TStream.WriteComponent
 0001:0002E6B4       Classes.TStream.WriteDescendent
 0001:0002E710       Classes.TStream.ReadComponentRes
 0001:0002E72C       Classes.TStream.WriteComponentRes
 0001:0002E734       Classes.TStream.WriteResourceHeader
 0001:0002E9C0       Classes.TStream.FixupResourceHeader
 0001:0002EA84       Classes.TStream.WriteDescendentRes
 0001:0002EAB8       Classes.TStream.ReadResHeader
 0001:0002EBA4       Classes.THandleStream.Create
 0001:0002EBE0       Classes.THandleStream.Read
 0001:0002EBF0       Classes.THandleStream.Write
 0001:0002EC00       Classes.THandleStream.Seek
 0001:0002EC2C       Classes.THandleStream.SetSize
 0001:0002EC40       Classes.THandleStream.SetSize
 0001:0002EC68       Classes.TFileStream.Create
 0001:0002ECAC       Classes.TFileStream.Create
 0001:0002EE20       Classes.TFileStream.Destroy
 0001:0002EE54       Classes.TCustomMemoryStream.SetPointer
 0001:0002EE5C       Classes.TCustomMemoryStream.Read
 0001:0002EE94       Classes.TCustomMemoryStream.Seek
 0001:0002EEB8       Classes.TCustomMemoryStream.SaveToStream
 0001:0002EED0       Classes.TCustomMemoryStream.SaveToFile
 0001:0002EF28       Classes.TMemoryStream.Destroy
 0001:0002EF54       Classes.TMemoryStream.Clear
 0001:0002EF6C       Classes.TMemoryStream.LoadFromStream
 0001:0002EFA4       Classes.TMemoryStream.LoadFromFile
 0001:0002EFF8       Classes.TMemoryStream.SetCapacity
 0001:0002F020       Classes.TMemoryStream.SetSize
 0001:0002F04C       Classes.TMemoryStream.Realloc
 0001:0002F0CC       Classes.TMemoryStream.Write
 0001:0002F11C       Classes.TResourceStream.Create
 0001:0002F174       Classes.TResourceStream.CreateFromID
 0001:0002F1C8       Classes.Error
 0001:0002F268       Classes.TResourceStream.Initialize
 0001:0002F2D4       Classes.TResourceStream.Destroy
 0001:0002F304       Classes.TResourceStream.Write
 0001:0002F31C       Classes.TFiler.Create
 0001:0002F364       Classes.TFiler.Destroy
 0001:0002F38C       Classes.TFiler.SetRoot
 0001:0002F390       Classes..TPropFixup
 0001:0002F5BC       Classes..TPropIntfFixup
 0001:0002F6A4       Classes.TPropFixup.Create
 0001:0002F6FC       Classes.TPropFixup.MakeGlobalReference
 0001:0002F75C       Classes.TPropFixup.ResolveReference
 0001:0002F76C       Classes.TPropIntfFixup.ResolveReference
 0001:0002F7F0       Classes.FindNestedComponent
 0001:0002F8E8       Classes.AddFinished
 0001:0002F920       Classes.AddNotFinished
 0001:0002F968       Classes.GlobalFixupReferences
 0001:0002FB3C       Classes.RemoveFixupReferences
 0001:0002FBF0       Classes.RemoveFixups
 0001:0002FC84       Classes.ReadError
 0001:0002FC9C       Classes.PropValueError
 0001:0002FCA8       Classes.PropertyNotFound
 0001:0002FCD4       Classes.SetElementValue
 0001:0002FCEC       Classes.TReader.Destroy
 0001:0002FD28       Classes.TReader.BeginReferences
 0001:0002FD90       Classes.TReader.CheckValue
 0001:0002FDB4       Classes.TReader.DefineProperty
 0001:0002FDF0       Classes.TReader.DefineBinaryProperty
 0001:0002FED8       Classes.TReader.EndOfList
 0001:0002FEEC       Classes.TReader.EndReferences
 0001:0002FF08       Classes.TReader.Error
 0001:0002FF2C       Classes.TReader.FindMethodInstance
 0001:0002FF9C       Classes.TReader.FindMethod
 0001:0002FFEC       Classes.RemoveGlobalFixup
 0001:00030074       Classes.TReader.DoFixupReferences
 0001:000301B8       Classes.TReader.FixupReferences
 0001:000301F0       Classes.TReader.FlushBuffer
 0001:00030214       Classes.TReader.FreeFixups
 0001:00030250       Classes.TReader.GetFieldClass
 0001:000302E4       Classes.TReader.GetPosition
 0001:000302FC       Classes.TReader.NextValue
 0001:0003030C       Classes.TReader.PropertyError
 0001:00030320       Classes.TReader.Read
 0001:0003036C       Classes.TReader.ReadBuffer
 0001:000303A8       Classes.TReader.ReadBoolean
 0001:000303BC       Classes.TReader.ReadChar
 0001:00030450       Classes.TReader.ReadWideChar
 0001:000304B0       Classes.TReader.ReadCollection
 0001:0003058C       Classes.AddSubComponentsToLoaded
 0001:000305C8       Classes.CheckSubComponents
 0001:00030640       Classes.SetSubComponentState
 0001:000306A8       Classes.ComponentCreated
 0001:000306C8       Classes.Recover
 0001:00030728       Classes.CreateComponent
 0001:00030838       Classes.SetCompName
 0001:000308D8       Classes.FindExistingComponent
 0001:0003097C       Classes.TReader.ReadComponent
 0001:00030BBC       Classes.TReader.ReadData
 0001:00030C2C       Classes.TReader.ReadDataInner
 0001:00030CFC       Classes.TReader.ReadFloat
 0001:00030D34       Classes.TReader.ReadDouble
 0001:00030D78       Classes.TReader.ReadSingle
 0001:00030DBC       Classes.TReader.ReadCurrency
 0001:00030E0C       Classes.TReader.ReadDate
 0001:00030E50       Classes.TReader.ReadIdent
 0001:00030FE8       Classes.TReader.ReadInteger
 0001:00031054       Classes.TReader.ReadInt64
 0001:00031098       Classes.TReader.ReadListBegin
 0001:000310A0       Classes.TReader.ReadListEnd
 0001:000310A8       Classes.TReader.ReadPrefix
 0001:000310E8       Classes.HandleException
 0001:000311B8       Classes.PropPathError
 0001:000311D4       Classes.TReader.ReadProperty
 0001:0003144C       Classes.SetIntIdent
 0001:00031494       Classes.SetObjectIdent
 0001:000314D4       Classes.SetVariantReference
 0001:00031530       Classes.SetInterfaceReference
 0001:000315F0       Classes.TReader.ReadPropValue
 0001:00031954       Classes.FindUniqueName
 0001:000319BC       Classes.TReader.ReadRootComponent
 0001:00031CF0       Classes.TReader.ReadComponents
 0001:00031DE0       Classes.TReader.ReadSet
 0001:00031E9C       Classes.TReader.ReadSignature
 0001:00031EC0       Classes.TReader.ReadStr
 0001:00031F50       Classes.TReader.ReadString
 0001:00032038       Classes.TReader.ReadWideString
 0001:00032178       Classes.TReader.ReadValue
 0001:0003218C       Classes.TReader.SetPosition
 0001:000321AC       Classes.TReader.SkipSetBody
 0001:000321F4       Classes.SkipList
 0001:00032220       Classes.SkipBinary
 0001:00032250       Classes.SkipCollection
 0001:000322B4       Classes.TReader.SkipValue
 0001:00032464       Classes.CopySetBody
 0001:000324EC       Classes.CopyList
 0001:00032538       Classes.CopyBytes
 0001:000325C8       Classes.CopyBinary
 0001:00032620       Classes.TReader.CopyValue
 0001:00032808       Classes.TReader.SkipProperty
 0001:00032850       Classes.TReader.SkipComponent
 0001:000328FC       Classes.TReader.FindAncestorComponent
 0001:000329B4       Classes.TReader.ReferenceName
 0001:000329CC       Classes.TReader.SetName
 0001:000329F4       Classes.TReader.FindComponentClass
 0001:00032A68       Classes.TReader.SkipBytes
 0001:00032AB0       Classes.ReadCustomVariant
 0001:00032C78       Classes.TReader.ReadVariant
 0001:00032E98       Classes.TWriter.Destroy
 0001:00032EC4       Classes.TWriter.AddAncestor
 0001:00032ED0       Classes.TWriter.DefineProperty
 0001:00032EF8       Classes.TWriter.DefineBinaryProperty
 0001:00032F24       Classes.TWriter.GetPosition
 0001:00032F34       Classes.TWriter.FindMethodName
 0001:00032F7C       Classes.TWriter.FlushBuffer
 0001:00032F84       Classes.TWriter.SetPosition
 0001:00032FC0       Classes.TWriter.SetRoot
 0001:00032FD8       Classes.TWriter.Write
 0001:00033024       Classes.TWriter.WriteBinary
 0001:000330AC       Classes.TWriter.WriteBuffer
 0001:000330C4       Classes.TWriter.WriteBoolean
 0001:000330D8       Classes.TWriter.WriteChar
 0001:00033128       Classes.TWriter.WriteWideChar
 0001:00033178       Classes.TWriter.WriteCollection
 0001:00033218       Classes.FindAncestor
 0001:00033268       Classes.TWriter.WriteComponent
 0001:000333BC       Classes.TWriter.WriteData
 0001:0003377C       Classes.TWriter.WriteDescendent
 0001:000337A4       Classes.TWriter.WriteFloat
 0001:000337C8       Classes.TWriter.WriteSingle
 0001:000337EC       Classes.TWriter.WriteDouble
 0001:00033810       Classes.TWriter.WriteCurrency
 0001:00033834       Classes.TWriter.WriteDate
 0001:00033858       Classes.TWriter.WriteIdent
 0001:0003393C       Classes.TWriter.WriteInteger
 0001:000339B0       Classes.TWriter.WriteInteger
 0001:00033A08       Classes.TWriter.WriteListBegin
 0001:00033A10       Classes.TWriter.WriteListEnd
 0001:00033A18       Classes.TWriter.WritePrefix
 0001:00033A60       Classes.TWriter.WriteProperties
 0001:00033B28       Classes.AncestorIsValid
 0001:00033B40       Classes.IsDefaultOrdProp
 0001:00033B98       Classes.IsDefaultFloatProp
 0001:00033BF4       Classes.IsDefaultInt64Prop
 0001:00033C4C       Classes.IsDefaultStrProp
 0001:00033CDC       Classes.ObjectAncestorMatch
 0001:00033D1C       Classes.IsDefault
 0001:00033D74       Classes.IsDefaultObjectProp
 0001:00033DF4       Classes.IsDefaultValue
 0001:00033EC0       Classes.IsDefaultInterfaceProp
 0001:00033F9C       Classes.FindMethodName
 0001:00033FF4       Classes.IsDefaultMethodProp
 0001:00034094       Classes.IsDefaultVariantProp
 0001:0003412C       Classes.IsDefaultPropertyValue
 0001:00034290       Classes.WritePropPath
 0001:000342E8       Classes.WriteSet
 0001:0003437C       Classes.WriteIntProp
 0001:000343E8       Classes.WriteCollectionProp
 0001:0003448C       Classes.WriteOrdProp
 0001:00034584       Classes.WriteFloatProp
 0001:000345C4       Classes.WriteInt64Prop
 0001:00034600       Classes.WriteStrProp
 0001:00034678       Classes.OwnedBy
 0001:00034690       Classes.GetComponentValue
 0001:000347D4       Classes.WriteObjectProp
 0001:000349E8       Classes.WriteInterfaceProp
 0001:00034AC4       Classes.WriteMethodProp
 0001:00034B54       Classes.WriteVariantProp
 0001:00034BB8       Classes.TWriter.WriteProperty
 0001:00034D0C       Classes.TWriter.WriteVariant
 0001:000350EC       Classes.TWriter.WritePropName
 0001:00035140       Classes.TWriter.WriteRootComponent
 0001:00035148       Classes.TWriter.WriteSignature
 0001:00035158       Classes.TWriter.WriteStr
 0001:00035214       Classes.TWriter.WriteMinStr
 0001:00035348       Classes.TWriter.WriteString
 0001:00035460       Classes.TWriter.WriteUTF8Str
 0001:00035534       Classes.TWriter.WriteWideString
 0001:0003553C       Classes.TWriter.WriteValue
 0001:00035550       Classes.TWriter.GetLookupInfo
 0001:00035574       Classes.InitThreadSynchronization
 0001:000355A8       Classes.DoneThreadSynchronization
 0001:000355C0       Classes.FreeExternalThreads
 0001:0003564C       Classes.ResetSyncEvent
 0001:00035658       Classes.WaitForSyncEvent
 0001:00035674       Classes.SignalSyncEvent
 0001:00035680       Classes.CheckSynchronize
 0001:00035874       Classes.ThreadProc
 0001:00035928       Classes.TThread.Create
 0001:00035A2C       Classes.TThread.Destroy
 0001:00035AA0       Classes.TThread.Destroy@
 0001:00035AC8       Classes.TThread.AfterConstruction
 0001:00035ADC       Classes.TThread.CheckThreadError
 0001:00035B58       Classes.TThread.CheckThreadError
 0001:00035B70       Classes.TThread.CallOnTerminate
 0001:00035B84       Classes.TThread.DoTerminate
 0001:00035B98       Classes.TThread.GetPriority
 0001:00035BD4       Classes.TThread.InternalStart
 0001:00035C80       Classes.TThread.SetPriority
 0001:00035CAC       Classes.TThread.Queue
 0001:00035D34       Classes.TThread.Queue
 0001:00035E00       Classes.TThread.Queue
 0001:00035EA0       Classes.TThread.RemoveQueuedEvents
 0001:00035F64       Classes.TThread.StaticQueue
 0001:00035F78       Classes.TThread.Synchronize
 0001:0003613C       Classes.TThread.Synchronize
 0001:00036170       Classes.TThread.Synchronize
 0001:000361D8       Classes.TThread.Synchronize
 0001:00036268       Classes.TThread.Queue
 0001:0003634C       Classes.TThread.Synchronize
 0001:000363E8       Classes.TThread.StaticSynchronize
 0001:000363FC       Classes.TThread.RemoveQueuedEvents
 0001:000364A0       Classes.TThread.RemoveQueuedEvents
 0001:000364B4       Classes.TThread.SetSuspended
 0001:000364CC       Classes.TThread.SpinWait
 0001:000364E8       Classes.TThread.Start
 0001:000364F0       Classes.TThread.Suspend
 0001:00036560       Classes.TThread.Resume
 0001:00036588       Classes.TThread.Terminate
 0001:000365AC       Classes.TThread.WaitFor
 0001:0003666C       Classes.TThread.NameThreadForDebugging
 0001:0003670C       Classes.TComponentEnumerator.Create
 0001:00036750       Classes.TComponentEnumerator.GetCurrent
 0001:0003675C       Classes.TComponentEnumerator.MoveNext
 0001:00036778       Classes.TComponent.Create
 0001:000367C4       Classes.TComponent.Destroy
 0001:0003680C       Classes.TComponent.BeforeDestruction
 0001:00036818       Classes.TComponent.RemoveFreeNotifications
 0001:00036858       Classes.TComponent.FreeNotification
 0001:000368AC       Classes.TComponent.ReadLeft
 0001:000368C0       Classes.TComponent.ReadTop
 0001:000368D4       Classes.TComponent.WriteLeft
 0001:000368E0       Classes.TComponent.WriteTop
 0001:000368EC       Classes.TComponent.Insert
 0001:00036928       Classes.TComponent.Remove
 0001:000369A0       Classes.TComponent.InsertComponent
 0001:00036A04       Classes.TComponent.RemoveComponent
 0001:00036A3C       Classes.TComponent.DestroyComponents
 0001:00036AA8       Classes.TComponent.Destroying
 0001:00036AE4       Classes.TComponent.RemoveNotification
 0001:00036B3C       Classes.TComponent.RemoveFreeNotification
 0001:00036B58       Classes.TComponent.Notification
 0001:00036BB8       Classes.TComponent.DefineProperties
 0001:00036C50       Classes.TComponent.HasParent
 0001:00036C54       Classes.TComponent.GetChildren
 0001:00036C5C       Classes.TComponent.GetChildOwner
 0001:00036C60       Classes.TComponent.GetChildParent
 0001:00036C64       Classes.TComponent.GetEnumerator
 0001:00036C74       Classes.TComponent.GetNamePath
 0001:00036C88       Classes.TComponent.GetOwner
 0001:00036C8C       Classes.TComponent.SetChildOrder
 0001:00036C90       Classes.TComponent.GetParentComponent
 0001:00036C94       Classes.TComponent.SetParentComponent
 0001:00036C98       Classes.TComponent.Updating
 0001:00036CA4       Classes.TComponent.Updated
 0001:00036CB0       Classes.TComponent.Loaded
 0001:00036CBC       Classes.TComponent.PaletteCreated
 0001:00036CC0       Classes.TComponent.ReadState
 0001:00036CC8       Classes.TComponent.WriteState
 0001:00036CD0       Classes.TComponent.ValidateRename
 0001:00036D58       Classes.TComponent.ValidateContainer
 0001:00036D6C       Classes.TComponent.ValidateInsert
 0001:00036DC8       Classes..TComponent.FindComponent$ActRec
 0001:00036E80       Classes.TComponent.FindComponent$ActRec.$0$Body
 0001:00036E8C       Classes.TComponent.FindComponent
 0001:00036F78       Classes.TComponent.FindSortedComponent
 0001:00036FF0       Classes.TComponent.AddSortedComponent
 0001:00037014       Classes.TComponent.SetName
 0001:000370A4       Classes.TComponent.ChangeName
 0001:000370DC       Classes.TComponent.GetComponentIndex
 0001:000370F8       Classes.TComponent.GetComponent
 0001:00037124       Classes.TComponent.GetComponentCount
 0001:00037134       Classes.TComponent.SetComponentIndex
 0001:00037188       Classes.TComponent.SetDesigning
 0001:000371D8       Classes.TComponent.SetReference
 0001:00037200       Classes.TComponent.ExecuteAction
 0001:00037228       Classes.TComponent.UpdateAction
 0001:00037250       Classes.TComponent.SetSubComponent
 0001:00037264       Classes.TComponent.GetComObject
 0001:0003731C       Classes.TComponent.SafeCallException
 0001:00037334       Classes.TComponent.FreeOnRelease
 0001:00037344       Classes.TComponent.UpdateRegistry
 0001:0003734C       Classes.TComponent.QueryInterface
 0001:0003738C       Classes.TComponent._AddRef
 0001:000373AC       Classes.TComponent._Release
 0001:000373CC       Classes.TComponent.IntfGetComponent
 0001:000373D0       Classes.TComponent.IsImplementorOf
 0001:00037450       Classes.TComponent.ReferenceInterface
 0001:000374F8       Classes.TBasicActionLink.Create
 0001:0003753C       Classes.TBasicActionLink.AssignClient
 0001:00037540       Classes.TBasicActionLink.Destroy
 0001:00037574       Classes.TBasicActionLink.Change
 0001:0003758C       Classes.TBasicActionLink.Execute
 0001:000375A8       Classes.TBasicActionLink.SetAction
 0001:000375D4       Classes.TBasicActionLink.IsOnExecuteLinked
 0001:000375D8       Classes.TBasicActionLink.SetOnExecute
 0001:000375E0       Classes.TBasicActionLink.Update
 0001:000375EC       Classes.TBasicAction.Create
 0001:00037630       Classes.TBasicAction.Destroy
 0001:00037698       Classes.TBasicAction.HandlesTarget
 0001:0003769C       Classes.TBasicAction.ExecuteTarget
 0001:000376A0       Classes.TBasicAction.Notification
 0001:000376C8       Classes.TBasicAction.UpdateTarget
 0001:000376CC       Classes.TBasicAction.Execute
 0001:000376E8       Classes.TBasicAction.Update
 0001:00037704       Classes.TBasicAction.SetOnExecute
 0001:00037760       Classes.TBasicAction.Change
 0001:00037774       Classes.TBasicAction.RegisterChanges
 0001:00037780       Classes.TBasicAction.UnRegisterChanges
 0001:000377C0       Classes.TBasicAction.SetActionComponent
 0001:000377EC       Classes.FreeIntConstList
 0001:00037864       Classes.ModuleUnload
 0001:0003786C       Classes.CleanupInstFreeList
 0001:000378A8       Classes.GetFreeInstBlockItemCount
 0001:000378D8       Classes.ReleaseObjectInstanceBlocks
 0001:0003793C       Classes.EFileStreamError.Create
 0001:000379EC       Classes.Finalization
 0001:00037ABC       SyncObjs..TSynchroObject
 0001:00037BC0       SyncObjs..TCriticalSection
 0001:00037DC8       SyncObjs.TSynchroObject.Acquire
 0001:00037DCC       SyncObjs.TSynchroObject.Release
 0001:00037DD0       SyncObjs.TCriticalSection.Create
 0001:00037E10       SyncObjs.TCriticalSection.Destroy
 0001:00037E40       SyncObjs.TCriticalSection.Acquire
 0001:00037E4C       SyncObjs.TCriticalSection.Release
 0001:00037E58       SyncObjs.TCriticalSection.TryEnter
 0001:00037E6C       SyncObjs.TCriticalSection.Enter
 0001:00037E74       SyncObjs.TCriticalSection.Leave
 0001:00037E7C       SyncObjs.InternalInitConditionVariable
 0001:00037E8C       SyncObjs.InternalWakeConditionVariable
 0001:00037E9C       SyncObjs.InternalWakeAllConditionVariable
 0001:00037EAC       SyncObjs.InternalSleepConditionVariableCS
 0001:00037EC8       SyncObjs.TInternalConditionVariable.DequeueWaiter
 0001:00037F20       SyncObjs.TInternalConditionVariable.DequeueWaiterNoLock
 0001:00037F3C       SyncObjs.TInternalConditionVariable.LockQueue
 0001:00037FA0       SyncObjs.TInternalConditionVariable.QueueWaiter
 0001:00038008       SyncObjs.TInternalConditionVariable.RemoveWaiter
 0001:00038094       SyncObjs.TInternalConditionVariable.SleepCriticalSection
 0001:0003818C       SyncObjs.TInternalConditionVariable.UnlockQueue
 0001:00038194       SyncObjs.TInternalConditionVariable.Wake
 0001:000381A8       SyncObjs.TInternalConditionVariable.WakeAll
 0001:0003821C       SyncObjs.InitConditionVariableProcs
 0001:00038388       SyncObjs.Finalization
 0001:00038390       Rtti.OnUnloadModule
 0001:000383E0       Rtti.Finalization
 0001:00038CF4       ceflib..TCefBaseOwn
 0001:00038EB0       ceflib..TCefBaseRef
 0001:00039268       ceflib..TCefBrowserRef
 0001:000394C4       ceflib..TCefFrameRef
 0001:00039638       ceflib..TCefPostDataRef
 0001:00039800       ceflib..TCefPostDataElementRef
 0001:00039A10       ceflib..TCefRequestRef
 0001:00039BB0       ceflib..TCefStreamReaderRef
 0001:0003A064       ceflib..TCefv8ValueRef
 0001:0003A5B8       ceflib..TCefv8ContextRef
 0001:0003A784       ceflib..TCefv8HandlerRef
 0001:0003A86C       ceflib..TCefClientOwn
 0001:0003A96C       ceflib..TCefLifeSpanHandlerOwn
 0001:0003AA60       ceflib..TCefLoadHandlerOwn
 0001:0003AB44       ceflib..TCefDisplayHandlerOwn
 0001:0003ACD4       ceflib..TCefCustomStreamReader
 0001:0003AF1C       ceflib..TCefSchemeHandlerOwn
 0001:0003B210       ceflib..TCefSchemeHandlerCallbackRef
 0001:0003B378       ceflib..TCefSchemeHandlerFactoryOwn
 0001:0003B53C       ceflib..TCefv8HandlerOwn
 0001:0003B680       ceflib..TCefDomVisitorOwn
 0001:0003B758       ceflib..TCefFastDomVisitor
 0001:0003B988       ceflib..TCefDomDocumentRef
 0001:0003BBEC       ceflib..TCefDomNodeRef
 0001:0003BD88       ceflib..TCefDomEventRef
 0001:0003BED4       ceflib..TCefDomEventListenerOwn
 0001:0003C07C       ceflib..TCefResponseRef
 0001:0003C160       ceflib..TCefFastDomEventListener
 0001:0003C300       ceflib..TCefV8AccessorOwn
 0001:0003C3DC       ceflib..TCefFastV8Accessor
 0001:0003C524       ceflib..ECefException
 0001:0003C5E4       ceflib.TzSpecificLocalTimeToSystemTime
 0001:0003C5EC       ceflib.SystemTimeToTzSpecificLocalTime
 0001:0003C5F4       ceflib..TSHSyncProcessRequest
 0001:0003C7C4       ceflib.TSHSyncProcessRequest.Execute
 0001:0003C7E0       ceflib.TSHSyncProcessRequest.Create
 0001:0003C83C       ceflib..TSHSyncReadResponse
 0001:0003CA30       ceflib.TSHSyncReadResponse.Execute
 0001:0003CA50       ceflib.TSHSyncReadResponse.Create
 0001:0003CAA8       ceflib..TSHSyncGetResponseHeaders
 0001:0003CC34       ceflib.TSHSyncGetResponseHeaders.Execute
 0001:0003CC48       ceflib.TSHSyncGetResponseHeaders.Create
 0001:0003CC98       ceflib.cef_string_utf16_copy
 0001:0003CCB4       ceflib.CefTimeToSystemTime
 0001:0003CCF4       ceflib.SystemTimeToCefTime
 0001:0003CD2C       ceflib.CefTimeToDateTime
 0001:0003CD64       ceflib.DateTimeToCefTime
 0001:0003CD9C       ceflib.cef_base_add_ref
 0001:0003CDB4       ceflib.cef_base_release
 0001:0003CDCC       ceflib.cef_base_get_refct
 0001:0003CDE0       ceflib.cef_client_get_life_span_handler
 0001:0003CE40       ceflib.cef_client_get_load_handler
 0001:0003CEA0       ceflib.cef_client_get_request_handler
 0001:0003CF00       ceflib.cef_client_get_display_handler
 0001:0003CF60       ceflib.cef_client_get_focus_handler
 0001:0003CFC0       ceflib.cef_client_get_keyboard_handler
 0001:0003D020       ceflib.cef_client_get_menu_handler
 0001:0003D080       ceflib.cef_client_get_print_handler
 0001:0003D0E0       ceflib.cef_client_get_find_handler
 0001:0003D140       ceflib.cef_client_get_jsdialog_handler
 0001:0003D1A0       ceflib.cef_client_get_jsbinding_handler
 0001:0003D200       ceflib.cef_client_get_render_handler
 0001:0003D260       ceflib.cef_client_get_drag_handler
 0001:0003D2C0       ceflib.cef_life_span_handler_on_before_popup
 0001:0003D394       ceflib.cef_life_span_handler_on_after_created
 0001:0003D3F0       ceflib.cef_life_span_handler_on_before_close
 0001:0003D44C       ceflib.cef_life_span_handler_run_modal
 0001:0003D4B0       ceflib.cef_life_span_handler_do_close
 0001:0003D514       ceflib.cef_load_handler_on_load_start
 0001:0003D590       ceflib.cef_load_handler_on_load_end
 0001:0003D610       ceflib.cef_load_handler_on_load_error
 0001:0003D6D4       ceflib.cef_display_handler_on_nav_state_change
 0001:0003D740       ceflib.cef_display_handler_on_address_change
 0001:0003D7D4       ceflib.cef_display_handler_on_title_change
 0001:0003D84C       ceflib.cef_display_handler_on_tooltip
 0001:0003D8F0       ceflib.cef_display_handler_on_status_message
 0001:0003D96C       ceflib.cef_display_handler_on_console_message
 0001:0003DA08       ceflib.cef_read_handler_read
 0001:0003DA28       ceflib.cef_read_handler_seek
 0001:0003DA44       ceflib.cef_read_handler_tell
 0001:0003DA58       ceflib.cef_read_handler_eof
 0001:0003DA78       ceflib.cef_scheme_handler_factory_create
 0001:0003DB2C       ceflib.cef_scheme_handler_process_request
 0001:0003DBCC       ceflib.cef_scheme_handler_process_request_sync
 0001:0003DCB8       ceflib.cef_scheme_handler_cancel
 0001:0003DCCC       ceflib.cef_scheme_handler_read_response
 0001:0003DD3C       ceflib.cef_scheme_handler_read_response_sync
 0001:0003DE08       ceflib.cef_scheme_handler_get_response_headers_sync
 0001:0003DEC0       ceflib.cef_scheme_handler_get_response_headers
 0001:0003DF20       ceflib.cef_v8_handler_execute
 0001:0003E0AC       ceflib.cef_v8_handler_execute_function_with_context
 0001:0003E23C       ceflib.cef_dom_visitor_visite
 0001:0003E298       ceflib.cef_dom_event_listener_handle_event
 0001:0003E2F4       ceflib.cef_v8_accessor_get
 0001:0003E3F8       ceflib.cef_v8_accessor_put
 0001:0003E4A8       ceflib.TCefBaseOwn.CreateData
 0001:0003E528       ceflib.TCefBaseOwn.Destroy
 0001:0003E564       ceflib.TCefBaseOwn.Wrap
 0001:0003E578       ceflib.TCefBaseOwn.Lock
 0001:0003E584       ceflib.TCefBaseOwn.Unlock
 0001:0003E590       ceflib.TCefBaseRef.Create
 0001:0003E660       ceflib.TCefBaseRef.Destroy
 0001:0003E694       ceflib.TCefBaseRef.UnWrap
 0001:0003E6DC       ceflib.TCefBaseRef.Wrap
 0001:0003E6F0       ceflib.TCefBrowserRef.CanGoBack
 0001:0003E704       ceflib.TCefBrowserRef.CanGoForward
 0001:0003E718       ceflib.TCefBrowserRef.ClearHistory
 0001:0003E720       ceflib.TCefBrowserRef.CloseBrowser
 0001:0003E728       ceflib.TCefBrowserRef.CloseDevTools
 0001:0003E730       ceflib.TCefBrowserRef.Find
 0001:0003E770       ceflib.TCefBrowserRef.GetFocusedFrame
 0001:0003E790       ceflib.TCefBrowserRef.GetFrame
 0001:0003E7C4       ceflib.TCefBrowserRef.GetFrameNames
 0001:0003E89C       ceflib.TCefBrowserRef.GetClient
 0001:0003E8BC       ceflib.TCefBrowserRef.GetImage
 0001:0003E8F0       ceflib.TCefBrowserRef.GetMainFrame
 0001:0003E910       ceflib.TCefBrowserRef.GetOpenerWindowHandle
 0001:0003E918       ceflib.TCefBrowserRef.GetSize
 0001:0003E948       ceflib.TCefBrowserRef.GetWindowHandle
 0001:0003E950       ceflib.TCefBrowserRef.GetZoomLevel
 0001:0003E964       ceflib.TCefBrowserRef.GoBack
 0001:0003E96C       ceflib.TCefBrowserRef.GoForward
 0001:0003E974       ceflib.TCefBrowserRef.HasDocument
 0001:0003E988       ceflib.TCefBrowserRef.HidePopup
 0001:0003E994       ceflib.TCefBrowserRef.Invalidate
 0001:0003E9A0       ceflib.TCefBrowserRef.IsPopup
 0001:0003E9B4       ceflib.TCefBrowserRef.IsPopupVisible
 0001:0003E9CC       ceflib.TCefBrowserRef.IsWindowRenderingDisabled
 0001:0003E9E0       ceflib.TCefBrowserRef.ParentWindowWillClose
 0001:0003E9E8       ceflib.TCefBrowserRef.Reload
 0001:0003E9F0       ceflib.TCefBrowserRef.ReloadIgnoreCache
 0001:0003E9F8       ceflib.TCefBrowserRef.SendCaptureLostEvent
 0001:0003EA04       ceflib.TCefBrowserRef.SendFocusEvent
 0001:0003EA14       ceflib.TCefBrowserRef.SendKeyEvent
 0001:0003EA3C       ceflib.TCefBrowserRef.SendMouseClickEvent
 0001:0003EA60       ceflib.TCefBrowserRef.SendMouseMoveEvent
 0001:0003EA7C       ceflib.TCefBrowserRef.SendMouseWheelEvent
 0001:0003EA98       ceflib.TCefBrowserRef.SetFocus
 0001:0003EAA4       ceflib.TCefBrowserRef.SetSize
 0001:0003EAC0       ceflib.TCefBrowserRef.SetZoomLevel
 0001:0003EAD4       ceflib.TCefBrowserRef.ShowDevTools
 0001:0003EADC       ceflib.TCefBrowserRef.StopFinding
 0001:0003EAE8       ceflib.TCefBrowserRef.StopLoad
 0001:0003EAF0       ceflib.TCefBrowserRef.UnWrap
 0001:0003EB38       ceflib.TCefFrameRef.Copy
 0001:0003EB40       ceflib.TCefFrameRef.Cut
 0001:0003EB48       ceflib.TCefFrameRef.Del
 0001:0003EB50       ceflib.TCefFrameRef.ExecuteJavaScript
 0001:0003EB90       ceflib.TCefFrameRef.GetBrowser
 0001:0003EBB0       ceflib.TCefFrameRef.GetName
 0001:0003EBCC       ceflib.TCefFrameRef.GetSource
 0001:0003EBE8       ceflib.TCefFrameRef.getText
 0001:0003EC04       ceflib.TCefFrameRef.GetUrl
 0001:0003EC20       ceflib.TCefFrameRef.IsFocused
 0001:0003EC34       ceflib.TCefFrameRef.IsMain
 0001:0003EC48       ceflib.TCefFrameRef.LoadFile
 0001:0003ED2C       ceflib.TCefFrameRef.LoadRequest
 0001:0003EDC0       ceflib.TCefFrameRef.LoadStream
 0001:0003EEC0       ceflib.TCefFrameRef.LoadString
 0001:0003EEF8       ceflib.TCefFrameRef.LoadUrl
 0001:0003EF18       ceflib.TCefFrameRef.Paste
 0001:0003EF20       ceflib.TCefFrameRef.Print
 0001:0003EF28       ceflib.TCefFrameRef.Redo
 0001:0003EF30       ceflib.TCefFrameRef.SelectAll
 0001:0003EF38       ceflib.TCefFrameRef.Undo
 0001:0003EF40       ceflib.TCefFrameRef.ViewSource
 0001:0003EF48       ceflib.TCefFrameRef.VisitDom
 0001:0003EFDC       ceflib.TCefFrameRef.VisitDomProc
 0001:0003F058       ceflib.TCefFrameRef.UnWrap
 0001:0003F0A0       ceflib.TCefCustomStreamReader.Create
 0001:0003F110       ceflib.TCefCustomStreamReader.Create
 0001:0003F164       ceflib.TCefCustomStreamReader.Destroy
 0001:0003F198       ceflib.TCefCustomStreamReader.Eof
 0001:0003F208       ceflib.TCefCustomStreamReader.Read
 0001:0003F270       ceflib.TCefCustomStreamReader.Seek
 0001:0003F2D0       ceflib.TCefCustomStreamReader.Tell
 0001:0003F324       ceflib.TCefPostDataRef.AddElement
 0001:0003F3BC       ceflib.TCefPostDataRef.GetCount
 0001:0003F3C4       ceflib.TCefPostDataRef.GetElement
 0001:0003F3EC       ceflib.TCefPostDataRef.New
 0001:0003F408       ceflib.TCefPostDataRef.RemoveElement
 0001:0003F4A0       ceflib.TCefPostDataRef.RemoveElements
 0001:0003F4A8       ceflib.TCefPostDataRef.UnWrap
 0001:0003F4F0       ceflib.TCefPostDataElementRef.GetBytes
 0001:0003F4FC       ceflib.TCefPostDataElementRef.GetBytesCount
 0001:0003F504       ceflib.TCefPostDataElementRef.GetFile
 0001:0003F520       ceflib.TCefPostDataElementRef.GetType
 0001:0003F528       ceflib.TCefPostDataElementRef.New
 0001:0003F544       ceflib.TCefPostDataElementRef.SetToBytes
 0001:0003F550       ceflib.TCefPostDataElementRef.SetToEmpty
 0001:0003F558       ceflib.TCefPostDataElementRef.SetToFile
 0001:0003F578       ceflib.TCefPostDataElementRef.UnWrap
 0001:0003F5C0       ceflib.TCefRequestRef.GetFirstPartyForCookies
 0001:0003F5DC       ceflib.TCefRequestRef.GetFlags
 0001:0003F5E4       ceflib.TCefRequestRef.GetHeaderMap
 0001:0003F600       ceflib.TCefRequestRef.GetMethod
 0001:0003F61C       ceflib.TCefRequestRef.GetPostData
 0001:0003F63C       ceflib.TCefRequestRef.GetUrl
 0001:0003F658       ceflib.TCefRequestRef.New
 0001:0003F674       ceflib.TCefRequestRef.SetFirstPartyForCookies
 0001:0003F694       ceflib.TCefRequestRef.SetFlags
 0001:0003F6A0       ceflib.TCefRequestRef.SetHeaderMap
 0001:0003F6BC       ceflib.TCefRequestRef.SetMethod
 0001:0003F6DC       ceflib.TCefRequestRef.SetPostData
 0001:0003F774       ceflib.TCefRequestRef.SetUrl
 0001:0003F794       ceflib.TCefRequestRef.UnWrap
 0001:0003F7DC       ceflib.TCefStreamReaderRef.CreateForCustomStream
 0001:0003F880       ceflib.TCefStreamReaderRef.CreateForData
 0001:0003F8AC       ceflib.TCefStreamReaderRef.CreateForFile
 0001:0003F8DC       ceflib.TCefStreamReaderRef.CreateForStream
 0001:0003F960       ceflib.TCefStreamReaderRef.Eof
 0001:0003F974       ceflib.TCefStreamReaderRef.Read
 0001:0003F98C       ceflib.TCefStreamReaderRef.Seek
 0001:0003F998       ceflib.TCefStreamReaderRef.Tell
 0001:0003F9A0       ceflib.TCefStreamReaderRef.UnWrap
 0001:0003F9E8       ceflib.CefLoadLibDefault
 0001:0003FA34       ceflib.CefLoadLib
 0001:0004183C       ceflib.CefBrowserCreate
 0001:0004187C       ceflib.CefRunMessageLoop
 0001:0004188C       ceflib.CefString
 0001:000418EC       ceflib.CefString
 0001:00041910       ceflib.CefStringAlloc
 0001:00041988       ceflib.CefStringSet
 0001:000419F0       ceflib.CefStringClearAndGet
 0001:00041A0C       ceflib.CefStringFreeAndGet
 0001:00041A38       ceflib.CefRegisterSchemeHandlerFactory
 0001:00041AFC       ceflib.CefRegisterCustomScheme
 0001:00041B44       ceflib.CefRegisterExtension
 0001:00041C10       ceflib.TCefSchemeHandlerFactoryOwn.Create
 0001:00041C6C       ceflib.TCefSchemeHandlerFactoryOwn.New
 0001:00041CB8       ceflib.TCefSchemeHandlerOwn.Cancel
 0001:00041CC0       ceflib.TCefSchemeHandlerOwn.Create
 0001:00041D70       ceflib.TCefSchemeHandlerOwn.GetResponseHeaders
 0001:00041D74       ceflib.TCefSchemeHandlerOwn.ProcessRequest
 0001:00041D80       ceflib.TCefSchemeHandlerOwn.ReadResponse
 0001:00041D8C       ceflib.TCefv8ValueRef.CreateArray
 0001:00041DA8       ceflib.TCefv8ValueRef.CreateBool
 0001:00041DCC       ceflib.TCefv8ValueRef.CreateDate
 0001:00041E04       ceflib.TCefv8ValueRef.CreateDouble
 0001:00041E30       ceflib.TCefv8ValueRef.CreateFunction
 0001:00041EEC       ceflib.TCefv8ValueRef.CreateInt
 0001:00041F0C       ceflib.TCefv8ValueRef.CreateNull
 0001:00041F28       ceflib.TCefv8ValueRef.CreateObject
 0001:00041FCC       ceflib.TCefv8ValueRef.CreateObjectWithAccessor
 0001:000420AC       ceflib.TCefv8ValueRef.CreateObjectWithAccessorProc
 0001:00042138       ceflib.TCefv8ValueRef.CreateString
 0001:00042168       ceflib.TCefv8ValueRef.CreateUndefined
 0001:00042184       ceflib.TCefv8ValueRef.DeleteValueByIndex
 0001:0004219C       ceflib.TCefv8ValueRef.DeleteValueByKey
 0001:000421C4       ceflib.TCefv8ValueRef.ExecuteFunction
 0001:00042378       ceflib.TCefv8ValueRef.ExecuteFunctionWithContext
 0001:00042574       ceflib.TCefv8ValueRef.GetArrayLength
 0001:0004257C       ceflib.TCefv8ValueRef.GetBoolValue
 0001:00042590       ceflib.TCefv8ValueRef.GetDateValue
 0001:000425BC       ceflib.TCefv8ValueRef.GetDoubleValue
 0001:000425D0       ceflib.TCefv8ValueRef.GetFunctionHandler
 0001:000425F4       ceflib.TCefv8ValueRef.GetFunctionName
 0001:00042610       ceflib.TCefv8ValueRef.GetIntValue
 0001:00042618       ceflib.TCefv8ValueRef.GetKeys
 0001:000426F4       ceflib.TCefv8ValueRef.GetStringValue
 0001:00042710       ceflib.TCefv8ValueRef.GetUserData
 0001:00042730       ceflib.TCefv8ValueRef.GetValueByIndex
 0001:00042758       ceflib.TCefv8ValueRef.GetValueByKey
 0001:0004278C       ceflib.TCefv8ValueRef.HasValueByIndex
 0001:000427A4       ceflib.TCefv8ValueRef.HasValueByKey
 0001:000427CC       ceflib.TCefv8ValueRef.IsArray
 0001:000427E0       ceflib.TCefv8ValueRef.IsBool
 0001:000427F4       ceflib.TCefv8ValueRef.IsDate
 0001:00042808       ceflib.TCefv8ValueRef.IsDouble
 0001:0004281C       ceflib.TCefv8ValueRef.IsFunction
 0001:00042830       ceflib.TCefv8ValueRef.IsInt
 0001:00042844       ceflib.TCefv8ValueRef.IsNull
 0001:00042858       ceflib.TCefv8ValueRef.IsObject
 0001:0004286C       ceflib.TCefv8ValueRef.IsSame
 0001:0004290C       ceflib.TCefv8ValueRef.IsString
 0001:00042920       ceflib.TCefv8ValueRef.IsUndefined
 0001:00042934       ceflib.TCefv8ValueRef.SetValueByAccessor
 0001:0004296C       ceflib.TCefv8ValueRef.SetValueByIndex
 0001:00042A14       ceflib.TCefv8ValueRef.SetValueByKey
 0001:00042ACC       ceflib.TCefv8ValueRef.UnWrap
 0001:00042B4C       ceflib.TCefv8HandlerRef.Execute
 0001:00042D38       ceflib.TCefv8HandlerRef.ExecuteFunctionWithContext
 0001:00042F10       ceflib.TCefv8HandlerRef.UnWrap
 0001:00042F58       ceflib.TCefv8HandlerOwn.Create
 0001:00042FA8       ceflib.TCefv8HandlerOwn.Execute
 0001:00042FB4       ceflib.TCefv8HandlerOwn.ExecuteFunctionWithContext
 0001:00042FC0       ceflib.TCefv8ContextRef.Current
 0001:00042FDC       ceflib.TCefv8ContextRef.Enter
 0001:00042FF0       ceflib.TCefv8ContextRef.Entered
 0001:0004300C       ceflib.TCefv8ContextRef.Exit
 0001:00043020       ceflib.TCefv8ContextRef.GetBrowser
 0001:00043040       ceflib.TCefv8ContextRef.GetFrame
 0001:00043060       ceflib.TCefv8ContextRef.GetGlobal
 0001:00043080       ceflib.TCefv8ContextRef.UnWrap
 0001:000430C8       ceflib.TCefDomVisitorOwn.Create
 0001:00043110       ceflib.TCefDomVisitorOwn.visit
 0001:00043114       ceflib.TCefFastDomVisitor.Create
 0001:00043158       ceflib.TCefFastDomVisitor.visit
 0001:00043164       ceflib.TCefDomDocumentRef.GetBaseUrl
 0001:00043180       ceflib.TCefDomDocumentRef.GetBody
 0001:000431A0       ceflib.TCefDomDocumentRef.GetCompleteUrl
 0001:000431CC       ceflib.TCefDomDocumentRef.GetDocument
 0001:000431EC       ceflib.TCefDomDocumentRef.GetElementById
 0001:00043220       ceflib.TCefDomDocumentRef.GetFocusedNode
 0001:00043240       ceflib.TCefDomDocumentRef.GetHead
 0001:00043260       ceflib.TCefDomDocumentRef.GetSelectionAsMarkup
 0001:0004327C       ceflib.TCefDomDocumentRef.GetSelectionAsText
 0001:00043298       ceflib.TCefDomDocumentRef.GetSelectionEndNode
 0001:000432B8       ceflib.TCefDomDocumentRef.GetSelectionEndOffset
 0001:000432C0       ceflib.TCefDomDocumentRef.GetSelectionStartNode
 0001:000432E0       ceflib.TCefDomDocumentRef.GetSelectionStartOffset
 0001:000432E8       ceflib.TCefDomDocumentRef.GetTitle
 0001:00043304       ceflib.TCefDomDocumentRef.GetType
 0001:0004330C       ceflib.TCefDomDocumentRef.HasSelection
 0001:00043320       ceflib.TCefDomDocumentRef.UnWrap
 0001:00043368       ceflib.TCefDomNodeRef.AddEventListener
 0001:00043420       ceflib.TCefDomNodeRef.AddEventListenerProc
 0001:000434A8       ceflib.TCefDomNodeRef.GetAsMarkup
 0001:000434C4       ceflib.TCefDomNodeRef.GetDocument
 0001:000434E4       ceflib.TCefDomNodeRef.GetElementAttribute
 0001:00043510       ceflib.TCefDomNodeRef.GetElementAttributes
 0001:0004352C       ceflib.TCefDomNodeRef.GetElementInnerText
 0001:00043548       ceflib.TCefDomNodeRef.GetElementTagName
 0001:00043564       ceflib.TCefDomNodeRef.GetFirstChild
 0001:00043584       ceflib.TCefDomNodeRef.GetLastChild
 0001:000435A4       ceflib.TCefDomNodeRef.GetName
 0001:000435C0       ceflib.TCefDomNodeRef.GetNextSibling
 0001:000435E0       ceflib.TCefDomNodeRef.GetParent
 0001:00043600       ceflib.TCefDomNodeRef.GetPreviousSibling
 0001:00043620       ceflib.TCefDomNodeRef.GetType
 0001:00043628       ceflib.TCefDomNodeRef.GetValue
 0001:00043644       ceflib.TCefDomNodeRef.HasChildren
 0001:00043658       ceflib.TCefDomNodeRef.HasElementAttribute
 0001:00043680       ceflib.TCefDomNodeRef.HasElementAttributes
 0001:00043694       ceflib.TCefDomNodeRef.IsElement
 0001:000436A8       ceflib.TCefDomNodeRef.IsSame
 0001:00043748       ceflib.TCefDomNodeRef.IsText
 0001:0004375C       ceflib.TCefDomNodeRef.SetElementAttribute
 0001:0004379C       ceflib.TCefDomNodeRef.SetValue
 0001:000437C4       ceflib.TCefDomNodeRef.UnWrap
 0001:0004380C       ceflib.TCefDomEventListenerOwn.Create
 0001:00043854       ceflib.TCefDomEventListenerOwn.HandleEvent
 0001:00043858       ceflib.TCefDomEventRef.CanBubble
 0001:0004386C       ceflib.TCefDomEventRef.CanCancel
 0001:00043880       ceflib.TCefDomEventRef.GetCategory
 0001:00043888       ceflib.TCefDomEventRef.GetCurrentTarget
 0001:000438A8       ceflib.TCefDomEventRef.GetDocument
 0001:000438C8       ceflib.TCefDomEventRef.GetPhase
 0001:000438D0       ceflib.TCefDomEventRef.GetTarget
 0001:000438F0       ceflib.TCefDomEventRef.GetType
 0001:0004390C       ceflib.TCefDomEventRef.UnWrap
 0001:00043954       ceflib.TCefFastDomEventListener.Create
 0001:00043998       ceflib.TCefFastDomEventListener.HandleEvent
 0001:000439B4       ceflib.TCefResponseRef.GetHeader
 0001:000439E0       ceflib.TCefResponseRef.GetHeaderMap
 0001:000439FC       ceflib.TCefResponseRef.GetMimeType
 0001:00043A18       ceflib.TCefResponseRef.GetStatus
 0001:00043A20       ceflib.TCefResponseRef.GetStatusText
 0001:00043A3C       ceflib.TCefResponseRef.SetHeaderMap
 0001:00043A58       ceflib.TCefResponseRef.SetMimeType
 0001:00043A78       ceflib.TCefResponseRef.SetStatus
 0001:00043A84       ceflib.TCefResponseRef.SetStatusText
 0001:00043AA4       ceflib.TCefResponseRef.UnWrap
 0001:00043AEC       ceflib.TCefV8AccessorOwn.Create
 0001:00043B3C       ceflib.TCefV8AccessorOwn.Get
 0001:00043B50       ceflib.TCefV8AccessorOwn.Put
 0001:00043B5C       ceflib.TCefFastV8Accessor.Create
 0001:00043BA8       ceflib.TCefFastV8Accessor.Get
 0001:00043BEC       ceflib.TCefFastV8Accessor.Put
 0001:00043C10       ceflib.TCefClientOwn.Create
 0001:00043CB8       ceflib.TCefClientOwn.GetDisplayHandler
 0001:00043CC4       ceflib.TCefClientOwn.GetDragHandler
 0001:00043CD0       ceflib.TCefClientOwn.GetFindHandler
 0001:00043CDC       ceflib.TCefClientOwn.GetFocusHandler
 0001:00043CE8       ceflib.TCefClientOwn.GetJsbindingHandler
 0001:00043CF4       ceflib.TCefClientOwn.GetJsdialogHandler
 0001:00043D00       ceflib.TCefClientOwn.GetKeyboardHandler
 0001:00043D0C       ceflib.TCefClientOwn.GetLifeSpanHandler
 0001:00043D18       ceflib.TCefClientOwn.GetLoadHandler
 0001:00043D24       ceflib.TCefClientOwn.GetMenuHandler
 0001:00043D30       ceflib.TCefClientOwn.GetPrintHandler
 0001:00043D3C       ceflib.TCefClientOwn.GetRenderHandler
 0001:00043D48       ceflib.TCefClientOwn.GetRequestHandler
 0001:00043D54       ceflib.TCefLifeSpanHandlerOwn.Create
 0001:00043DBC       ceflib.TCefLifeSpanHandlerOwn.OnAfterCreated
 0001:00043DC0       ceflib.TCefLifeSpanHandlerOwn.OnBeforeClose
 0001:00043DC4       ceflib.TCefLifeSpanHandlerOwn.OnBeforePopup
 0001:00043DD0       ceflib.TCefLifeSpanHandlerOwn.DoClose
 0001:00043DD4       ceflib.TCefLifeSpanHandlerOwn.RunModal
 0001:00043DD8       ceflib.TCefLoadHandlerOwn.Create
 0001:00043E30       ceflib.TCefLoadHandlerOwn.OnLoadEnd
 0001:00043E38       ceflib.TCefLoadHandlerOwn.OnLoadError
 0001:00043E44       ceflib.TCefLoadHandlerOwn.OnLoadStart
 0001:00043E48       ceflib.TCefDisplayHandlerOwn.Create
 0001:00043EB8       ceflib.TCefDisplayHandlerOwn.OnAddressChange
 0001:00043EC0       ceflib.TCefDisplayHandlerOwn.OnConsoleMessage
 0001:00043ECC       ceflib.TCefDisplayHandlerOwn.OnNavStateChange
 0001:00043ED4       ceflib.TCefDisplayHandlerOwn.OnStatusMessage
 0001:00043EDC       ceflib.TCefDisplayHandlerOwn.OnTitleChange
 0001:00043EE0       ceflib.TCefDisplayHandlerOwn.OnTooltip
 0001:00043EE4       ceflib.TCefSchemeHandlerCallbackRef.BytesAvailable
 0001:00043EEC       ceflib.TCefSchemeHandlerCallbackRef.Cancel
 0001:00043EF4       ceflib.TCefSchemeHandlerCallbackRef.HeadersAvailable
 0001:00043EFC       ceflib.TCefSchemeHandlerCallbackRef.UnWrap
 0001:00043F44       ceflib.Finalization
 0001:00044030       IOUtils.TPath.Destroy@
 0001:00044038       IOUtils.Finalization
 0001:00044100       IniFiles.Finalization
 0001:00044150       Registry..ERegistryException
 0001:00044344       Registry..TRegistry
 0001:00045300       Registry.ReadError
 0001:0004532C       Registry.IsRelative
 0001:000453A0       Registry.RegDataToDataType
 0001:000453D0       Registry.DataTypeToRegData
 0001:000453F8       Registry.BinaryToHexString
 0001:00045548       Registry.TRegistry.Create
 0001:0004558C       Registry.TRegistry.Create
 0001:000455C8       Registry.TRegistry.Destroy
 0001:000455F4       Registry.TRegistry.CheckResult
 0001:00045600       Registry.TRegistry.CloseKey
 0001:00045630       Registry.TRegistry.SetRootKey
 0001:0004565C       Registry.TRegistry.ChangeKey
 0001:00045680       Registry.TRegistry.GetBaseKey
 0001:00045694       Registry.TRegistry.SetCurrentKey
 0001:00045698       Registry.TRegistry.CreateKey
 0001:00045778       Registry.TRegistry.OpenKey
 0001:000458AC       Registry.TRegistry.OpenKeyReadOnly
 0001:00045A94       Registry.TRegistry.DeleteKey
 0001:00045C20       Registry.TRegistry.DeleteValue
 0001:00045C44       Registry.TRegistry.GetKeyInfo
 0001:00045CB0       Registry.TRegistry.GetKeyNames
 0001:00045D78       Registry.TRegistry.GetLastErrorMsg
 0001:00045EEC       Registry.TRegistry.GetRootKeyName
 0001:00045F24       Registry.TRegistry.GetValueNames
 0001:00045FEC       Registry.TRegistry.GetDataInfo
 0001:00046040       Registry.TRegistry.GetDataSize
 0001:00046068       Registry.TRegistry.GetDataType
 0001:00046090       Registry.TRegistry.WriteString
 0001:0004611C       Registry.TRegistry.WriteExpandString
 0001:000461A8       Registry.TRegistry.ReadString
 0001:0004625C       Registry.TRegistry.GetDataAsString
 0001:00046414       Registry.TRegistry.WriteInteger
 0001:00046428       Registry.TRegistry.ReadInteger
 0001:00046458       Registry.TRegistry.WriteBool
 0001:00046464       Registry.TRegistry.ReadBool
 0001:0004647C       Registry.TRegistry.WriteFloat
 0001:00046490       Registry.TRegistry.ReadFloat
 0001:000464C4       Registry.TRegistry.WriteCurrency
 0001:000464D8       Registry.TRegistry.ReadCurrency
 0001:0004650C       Registry.TRegistry.WriteDateTime
 0001:00046520       Registry.TRegistry.ReadDateTime
 0001:00046554       Registry.TRegistry.WriteDate
 0001:00046568       Registry.TRegistry.ReadDate
 0001:0004657C       Registry.TRegistry.WriteTime
 0001:00046590       Registry.TRegistry.ReadTime
 0001:000465A4       Registry.TRegistry.WriteBinaryData
 0001:000465B8       Registry.TRegistry.ReadBinaryData
 0001:0004661C       Registry.TRegistry.PutData
 0001:00046690       Registry.TRegistry.GetData
 0001:0004670C       Registry.TRegistry.HasSubKeys
 0001:00046730       Registry.TRegistry.ValueExists
 0001:00046740       Registry.TRegistry.GetKey
 0001:000467D8       Registry.TRegistry.RegistryConnect
 0001:00046814       Registry.TRegistry.LoadKey
 0001:000468A4       Registry.TRegistry.UnLoadKey
 0001:00046928       Registry.TRegistry.RestoreKey
 0001:000469A0       Registry.TRegistry.ReplaceKey
 0001:00046A44       Registry.TRegistry.SaveKey
 0001:00046ABC       Registry.TRegistry.KeyExists
 0001:00046B34       Registry.TRegistry.RenameValue
 0001:00046BD0       Registry.MoveValue
 0001:00046CF0       Registry.CopyValues
 0001:00046E28       Registry.CopyKeys
 0001:00047084       Registry.TRegistry.MoveKey
 0001:00047198       Registry.Finalization
 0001:000471F4       Contnrs..TObjectList
 0001:00047660       Contnrs.TObjectList.Add
 0001:00047668       Contnrs.TObjectList.Create
 0001:000476A4       Contnrs.TObjectList.Create
 0001:000476E8       Contnrs.TObjectList.Extract
 0001:000476FC       Contnrs.TObjectList.ExtractItem
 0001:00047714       Contnrs.TObjectList.FindInstanceOf
 0001:0004779C       Contnrs.TObjectList.First
 0001:000477AC       Contnrs.TObjectList.GetItem
 0001:000477C0       Contnrs.TObjectList.IndexOf
 0001:000477C8       Contnrs.TObjectList.IndexOfItem
 0001:000477D0       Contnrs.TObjectList.Insert
 0001:000477D8       Contnrs.TObjectList.Last
 0001:000477E4       Contnrs.TObjectList.Notify
 0001:00047810       Contnrs.TObjectList.Remove
 0001:00047818       Contnrs.TObjectList.RemoveItem
 0001:00047820       ceffilescheme..TFileScheme
 0001:00047A08       ceffilescheme.Escape
 0001:00047B04       ceffilescheme..TFileInfo
 0001:00047D14       ceffilescheme.TFileInfo.Create
 0001:00047D80       ceffilescheme.TFileInfo.DisplaySize
 0001:00048020       ceffilescheme.TFileInfo.DisplayDate
 0001:000480C4       ceffilescheme.TFileInfo.Display
 0001:000481F8       ceffilescheme.FileSortCompare
 0001:00048240       ceffilescheme.HTTPDecode
 0001:00048394       ceffilescheme.ParseFileUrl
 0001:00048598       ceffilescheme.TFileScheme.Cancel
 0001:000485A0       ceffilescheme.TFileScheme.Create
 0001:000485EC       ceffilescheme.TFileScheme.Destroy
 0001:00048620       ceffilescheme.TFileScheme.GetResponseHeaders
 0001:00048658       ceffilescheme.OutPut
 0001:00048704       ceffilescheme.OutputUTF8
 0001:000487B0       ceffilescheme.TFileScheme.ProcessRequest
 0001:00048F7C       ceffilescheme.TFileScheme.ReadResponse
 0001:00048FA4       cefclient..TCustomClient
 0001:0004910C       cefclient..TCustomLifeSpan
 0001:000491C0       cefclient..TCustomLoad
 0001:00049264       cefclient..TCustomDisplay
 0001:0004931C       cefclient..TScheme
 0001:00049484       cefclient..TExtension
 0001:0004958C       cefclient.CefWndProc
 0001:00049B2C       cefclient.TCustomClient.Create
 0001:00049BB8       cefclient.TCustomClient.GetDisplayHandler
 0001:00049BCC       cefclient.TCustomClient.GetLifeSpanHandler
 0001:00049BE0       cefclient.TCustomClient.GetLoadHandler
 0001:00049BF4       cefclient.TCustomLifeSpan.OnAfterCreated
 0001:00049C20       cefclient.TCustomLoad.OnLoadEnd
 0001:00049C44       cefclient.TCustomLoad.OnLoadStart
 0001:00049C78       cefclient.TCustomDisplay.OnAddressChange
 0001:00049CB8       cefclient.TCustomDisplay.OnTitleChange
 0001:00049CE4       cefclient.TScheme.Create
 0001:00049D3C       cefclient.TScheme.Destroy
 0001:00049D6C       cefclient.TScheme.ProcessRequest
 0001:0004A220       cefclient.TScheme.GetResponseHeaders
 0001:0004A294       cefclient.TScheme.ReadResponse
 0001:0004A2BC       cefclient.TScheme.Output
 0001:0004A348       cefclient.TExtension.Execute
 0001:0004A66C       cefclient.Finalization
 0002:00000000       System.System
 0002:000000AC       Windows.Windows
 0002:000000C4       SysUtils.TEncoding.Create@
 0002:000000CC       SysUtils.Exception.Create@
 0002:000000DC       SysUtils.SysUtils
 0002:00000178       VarUtils.VarUtils
 0002:00000188       Variants.Variants
 0002:00000234       TypInfo.TypInfo
 0002:0000023C       Classes.TThread.Create@
 0002:0000024C       Classes.Classes
 0002:000002DC       SyncObjs.SyncObjs
 0002:000002EC       Rtti.Rtti
 0002:00000338       ceflib.ceflib
 0002:0000034C       IOUtils.TPath.Create@
 0002:000007A4       IOUtils.IOUtils
 0002:000007AC       IniFiles.IniFiles
 0002:000007B4       Registry.Registry
 0002:000007BC       cefclient.cefclient
 0003:00000000       System.ExitCode
 0003:00000004       System.ErrorAddr
 0003:00000008       System.RandSeed
 0003:0000000C       System.FileMode
 0003:00000010       System.VarClearProc
 0003:00000014       System.VarAddRefProc
 0003:00000018       System.VarCopyProc
 0003:0000001C       System.VarToLStrProc
 0003:00000020       System.VarToWStrProc
 0003:00000024       System.Default8087CW
 0003:00000028       System.DebugHook
 0003:0000002C       System.JITEnable
 0003:00000030       System.NoErrMsg
 0003:00000034       System.SystemThreadFuncProc
 0003:00000038       System.SystemThreadEndProc
 0003:0000003C       System.LibModuleList
 0003:00000040       System.ModuleUnloadList
 0003:00000044       System.ObjCastGUID
 0003:00000054       System.Copyright
 0003:00000058       System.LeakMessageHeader
 0003:0000005C       System.SmallLeakDetail
 0003:00000060       System.LargeLeakDetail
 0003:00000064       System.BytesMessage
 0003:00000068       System.UnknownClassNameMsg
 0003:0000006C       System.AnsiStringBlockMessage
 0003:00000070       System.UnicodeStringBlockMessage
 0003:00000074       System.LeakMessageFooter
 0003:00000078       System.LeakMessageTitle
 0003:0000007C       System.SmallBlockTypes
 0003:0000075C       System.MemoryManager
 0003:00000774       System.reMap
 0003:00000790       System.errCaption
 0003:00000798       System.runErrMsg
 0003:000007B8       System.hexDigits
 0003:000007C8       System.EmptyStringW
 0003:000007D8       System.LocaleTable
 0003:000009E0       System.hexdig
 0003:000009E4       System...
 0003:000009E8       System.@__pfnDliFailureHook
 0003:000009EC       System.@__pfnDliNotifyHook
 0003:000009F0       SysInit.TlsIndex
 0003:000009F4       SysInit.PtrToNil
 0003:000009F8       SysInit.Module
 0003:00000A14       Windows.Win32MajorVersion
 0003:00000A18       Windows.Win32MinorVersion
 0003:00000A1C       Windows.Win32Platform
 0003:00000A20       Character.Latin1Categories
 0003:00000B20       SysUtils.EmptyStr
 0003:00000B24       SysUtils.EmptyWideStr
 0003:00000B28       SysUtils.EmptyAnsiStr
 0003:00000B2C       SysUtils.Win32Platform
 0003:00000B30       SysUtils.Win32MajorVersion
 0003:00000B34       SysUtils.Win32MinorVersion
 0003:00000B38       SysUtils.Win32BuildNumber
 0003:00000B3C       SysUtils.Win32CSDVersion
 0003:00000B40       SysUtils.TwoDigitYearCenturyWindow
 0003:00000B44       SysUtils.MonthDays
 0003:00000B74       SysUtils.LeadBytes
 0003:00000B94       SysUtils.HexDisplayPrefix
 0003:00000B98       SysUtils.GetDiskFreeSpaceEx
 0003:00000B9C       SysUtils.cSimpleBoolStrs
 0003:00000BA4       SysUtils.AccessMode
 0003:00000BB0       SysUtils.ShareMode
 0003:00000BC4       SysUtils.ShareMode
 0003:00000BD8       SysUtils.FormatErrorStrs
 0003:00000BE0       SysUtils.FCon1E18
 0003:00000BEC       SysUtils.DCon10
 0003:00000BF0       SysUtils.CWNear
 0003:00000BF4       SysUtils.FMSecsPerDay
 0003:00000BF8       SysUtils.IMSecsPerDay
 0003:00000BFC       SysUtils.Format
 0003:00000C04       SysUtils.DefShortMonthNames
 0003:00000C34       SysUtils.DefLongMonthNames
 0003:00000C64       SysUtils.DefShortDayNames
 0003:00000C80       SysUtils.DefLongDayNames
 0003:00000C9C       SysUtils.ErrorMap
 0003:00000CD4       SysUtils.ExceptTypes
 0003:00000D20       SysUtils.ExceptMap
 0003:00000DE0       SysUtils.MonitorSupport
 0003:00000DF4       SysUtils.TerminateProcList
 0003:00000DF8       SysUtils.DefaultFallbackLanguages
 0003:00000DFC       VarUtils.CResult
 0003:00000E04       Variants.NullEqualityRule
 0003:00000E08       Variants.NullMagnitudeRule
 0003:00000E0C       Variants.NullStrictConvert
 0003:00000E10       Variants.NullAsStringValue
 0003:00000E14       Variants.PackVarCreation
 0003:00000E18       Variants.BooleanToStringRule
 0003:00000E1C       Variants.BaseTypeMap
 0003:00000E34       Variants.CInvalidCustomVariantType
 0003:00000E38       Variants.CRangeToType
 0003:00000E4C       Variants.CBooleanToRelationship
 0003:00000E58       Variants.CmpTypeMap
 0003:00000EE8       Variants.CText
 0003:00000F40       Variants.LNextVarType
 0003:00000F44       Variants.CRelationshipToBoolean
 0003:00000F58       TypInfo.BooleanIdents
 0003:00000F60       TypInfo.DotSep
 0003:00000F64       Classes.CreateVCLComObjectProc
 0003:00000F68       Classes.WakeMainThread
 0003:00000F70       Classes.FilerSignature
 0003:00000F74       Classes.Dummy32bitResHeader
 0003:00000F94       Classes.NilMethod
 0003:00000F9C       Classes.SyncList
 0003:00000FA0       Classes.Priorities
 0003:00000FBC       Rtti.Kind
 0003:00000FC4       ceflib.CefLibrary
 0003:00000FC8       ceflib.CefCache
 0003:00000FCC       ceflib.CefUserAgent
 0003:00000FD0       ceflib.CefProductVersion
 0003:00000FD4       ceflib.CefLocale
 0003:00000FD8       ceflib.CefLogFile
 0003:00000FDC       ceflib.CefLogSeverity
 0003:00000FE0       ceflib.CefGraphicsImplementation
 0003:00000FE4       ceflib.CefExtraPluginPaths
 0003:00000FE8       ceflib.LibHandle
 0003:00000FEC       IOUtils.TPath.FCCurrentDir
 0003:00000FF0       IOUtils.TPath.FCParentDir
 0003:00000FF4       IOUtils.TPath.FCExtendedPrefix
 0003:00000FF8       IOUtils.TPath.FCExtendedUNCPrefix
 0003:00000FFC       IniFiles.TCustomIniFile.SectionNameSeparator
 0003:00001000       IniFiles.Values
 0003:00001008       Registry.KeyNames
 0003:00001024       Registry.Values
 0003:0000102C       ceffilescheme.s
 0003:0000105C       cefclient.handl
 0003:00001060       cefclient.brows
 0003:00001064       cefclient.browsrHwnd
 0003:00001068       cefclient.navigateto
 0004:00000000       System.DispCallByIDProc
 0004:00000004       System.ExceptProc
 0004:00000008       System.ErrorProc
 0004:0000000C       System.ExceptClsProc
 0004:00000010       System.ExceptObjProc
 0004:00000014       System.RaiseExceptionProc
 0004:00000018       System.RTLUnwindProc
 0004:0000001C       System.RaiseExceptObjProc
 0004:00000020       System.ExceptionAcquired
 0004:00000024       System.ExceptionClass
 0004:00000028       System.AssertErrorProc
 0004:0000002C       System.ExitProcessProc
 0004:00000030       System.AbstractErrorProc
 0004:00000034       System.MainInstance
 0004:00000038       System.MainThreadID
 0004:0000003C       System.IsLibrary
 0004:00000040       System.CmdShow
 0004:00000044       System.CmdLine
 0004:00000048       System.ExitProc
 0004:0000004C       System.IsConsole
 0004:0000004D       System.IsMultiThread
 0004:0000004E       System.Test8086
 0004:00000050       System.CPUCount
 0004:00000054       System.Input
 0004:00000324       System.Output
 0004:000005F4       System.ErrOutput
 0004:000008C4       System.MonitorSupport
 0004:000008C8       System.DefaultSystemCodePage
 0004:000008CC       System.DefaultUnicodeCodePage
 0004:000008D0       System.UTF8CompareLocale
 0004:000008D4       System.ReportMemoryLeaksOnShutdown
 0004:000008D5       System.NeverSleepOnMMThreadContention
 0004:000008D8       System..8
 0004:000008DC       System.AllocSize2SmallBlockTypeIndX4
 0004:00000A22       System.MinimumBlockAlignment
 0004:00000A24       System.MediumBlockPoolsCircularList
 0004:00000A34       System.MediumBlocksLocked
 0004:00000A38       System.LastSequentiallyFedMediumBlock
 0004:00000A3C       System.MediumSequentialFeedBytesLeft
 0004:00000A40       System.MediumBlockBinGroupBitmap
 0004:00000A44       System.MediumBlockBinBitmaps
 0004:00000AC4       System.MediumBlockBins
 0004:00002AC4       System.LargeBlocksLocked
 0004:00002AC8       System.LargeBlocksCircularList
 0004:00002AD8       System.ExpectedMemoryLeaks
 0004:00002ADC       System.ExpectedMemoryLeaksListLocked
 0004:00002AE0       System.MappingObjectHandle
 0004:00002AE4       System.InitContext
 0004:00002B14       System.DLLThreadContext
 0004:00002B44       System.GetThreadPreferredUILanguages
 0004:00002B48       System.SetThreadPreferredUILanguages
 0004:00002B4C       System.GetThreadUILanguage
 0004:00002B50       System.UseThreadUILanguageAPI
 0004:00002B54       System.CrSec
 0004:00002B6C       System.CachedLangID
 0004:00002B70       System.CachedLanguageNames
 0004:00002C1C       System...
 0004:00002C34       SysInit.ModuleIsLib
 0004:00002C35       SysInit.ModuleIsCpp
 0004:00002C38       SysInit.HInstance
 0004:00002C3C       SysInit.tlsBuffer
 0004:00002C40       Windows..2
 0004:00002C44       Windows.HtmlHelpModule
 0004:00002C48       Character.DataTable
 0004:00002C4C       Character.CatIndexPrimary
 0004:00002C50       Character.CatIndexSecondary
 0004:00002C54       Character.CategoryTable
 0004:00002C58       Character.NumIndexPrimary
 0004:00002C5C       Character.NumIndexSecondary
 0004:00002C60       Character.NumericValueTable
 0004:00002C64       SysUtils.Exception.$ClassInitFlag
 0004:00002C68       SysUtils.Exception.GetExceptionStackInfoProc
 0004:00002C6C       SysUtils.Exception.GetStackInfoStringProc
 0004:00002C70       SysUtils.Exception.CleanUpStackInfoProc
 0004:00002C74       SysUtils.CurrencyString
 0004:00002C78       SysUtils.CurrencyFormat
 0004:00002C79       SysUtils.NegCurrFormat
 0004:00002C7A       SysUtils.ThousandSeparator
 0004:00002C7C       SysUtils.DecimalSeparator
 0004:00002C7E       SysUtils.CurrencyDecimals
 0004:00002C80       SysUtils.DateSeparator
 0004:00002C84       SysUtils.ShortDateFormat
 0004:00002C88       SysUtils.LongDateFormat
 0004:00002C8C       SysUtils.TimeSeparator
 0004:00002C90       SysUtils.TimeAMString
 0004:00002C94       SysUtils.TimePMString
 0004:00002C98       SysUtils.ShortTimeFormat
 0004:00002C9C       SysUtils.LongTimeFormat
 0004:00002CA0       SysUtils.ShortMonthNames
 0004:00002CD0       SysUtils.LongMonthNames
 0004:00002D00       SysUtils.ShortDayNames
 0004:00002D1C       SysUtils.LongDayNames
 0004:00002D38       SysUtils.SysLocale
 0004:00002D46       SysUtils.ListSeparator
 0004:00002D48       SysUtils.EraNames
 0004:00002D64       SysUtils.EraYearOffsets
 0004:00002D80       SysUtils.TrueBoolStrs
 0004:00002D84       SysUtils.FalseBoolStrs
 0004:00002D88       SysUtils.TEncoding.FASCIIEncoding
 0004:00002D8C       SysUtils.TEncoding.FBigEndianUnicodeEncoding
 0004:00002D90       SysUtils.TEncoding.FDefaultEncoding
 0004:00002D94       SysUtils.TEncoding.FUnicodeEncoding
 0004:00002D98       SysUtils.TEncoding.FUTF7Encoding
 0004:00002D9C       SysUtils.TEncoding.FUTF8Encoding
 0004:00002DA0       SysUtils.TEncoding.$ClassInitFlag
 0004:00002DA4       SysUtils..76
 0004:00002DA8       SysUtils.OutOfMemory
 0004:00002DAC       SysUtils.InvalidPointer
 0004:00002DB0       SysUtils.SyncEventCache
 0004:00002EB0       SysUtils.EventCache
 0004:00002EB4       SysUtils.EventItemHolders
 0004:00002EB8       SysUtils.ValidatedUnitHashBuckets
 0004:00003EAC       SysUtils.UnitHashBuckets
 0004:00004EA0       SysUtils.LanguageArray
 0004:00004EA4       VarUtils.VariantChangeTypeEx
 0004:00004EA8       VarUtils.VarNeg
 0004:00004EAC       VarUtils.VarNot
 0004:00004EB0       VarUtils.VarAdd
 0004:00004EB4       VarUtils.VarSub
 0004:00004EB8       VarUtils.VarMul
 0004:00004EBC       VarUtils.VarDiv
 0004:00004EC0       VarUtils.VarIDiv
 0004:00004EC4       VarUtils.VarMod
 0004:00004EC8       VarUtils.VarAnd
 0004:00004ECC       VarUtils.VarOr
 0004:00004ED0       VarUtils.VarXor
 0004:00004ED4       VarUtils.VarCmp
 0004:00004ED8       VarUtils.VarI4FromStr
 0004:00004EDC       VarUtils.VarR4FromStr
 0004:00004EE0       VarUtils.VarR8FromStr
 0004:00004EE4       VarUtils.VarDateFromStr
 0004:00004EE8       VarUtils.VarCyFromStr
 0004:00004EEC       VarUtils.VarBoolFromStr
 0004:00004EF0       VarUtils.VarBstrFromCy
 0004:00004EF4       VarUtils.VarBstrFromDate
 0004:00004EF8       VarUtils.VarBstrFromBool
 0004:00004EFC       VarUtils..5
 0004:00004F00       Variants.EmptyParam
 0004:00004F10       Variants.VarDispProc
 0004:00004F14       Variants.ClearAnyProc
 0004:00004F18       Variants.ChangeAnyProc
 0004:00004F1C       Variants.RefAnyProc
 0004:00004F20       Variants..81
 0004:00004F24       Variants.LVarTypes
 0004:00004F28       Variants.LVarTypeSync
 0004:00004F40       TypInfo..5
 0004:00004F44       Classes.TThread.$ClassInitFlag
 0004:00004F48       Classes.GlobalNameSpace
 0004:00004F4C       Classes.IsUniqueGlobalComponentNameProc
 0004:00004F50       Classes.SyncEvent
 0004:00004F54       Classes..66
 0004:00004F58       Classes.IntConstList
 0004:00004F5C       Classes.RegGroups
 0004:00004F60       Classes.FindGlobalComponentProcs
 0004:00004F64       Classes.GlobalFixupList
 0004:00004F68       Classes.ThreadLock
 0004:00004F80       Classes.ExternalThreads
 0004:00004F84       Classes.InstBlockList
 0004:00004F88       Classes.InstFreeList
 0004:00004F8C       SyncObjs..01
 0004:00004F90       SyncObjs.InitializeConditionVariableProc
 0004:00004F94       SyncObjs.SleepConditionVariableCSProc
 0004:00004F98       SyncObjs.WakeConditionVariableProc
 0004:00004F9C       SyncObjs.WakeAllConditionVariableProc
 0004:00004FA0       Rtti..23
 0004:00004FA4       Rtti.ModListRemovals
 0004:00004FA8       Rtti.StringEqCmpCI
 0004:00004FAC       Rtti.PoolLock
 0004:00004FB0       ceflib.CefLocalStorageQuota
 0004:00004FB4       ceflib.CefSessionStorageQuota
 0004:00004FB8       ceflib..85
 0004:00004FBC       ceflib.cef_string_wide_set
 0004:00004FC0       ceflib.cef_string_utf8_set
 0004:00004FC4       ceflib.cef_string_utf16_set
 0004:00004FC8       ceflib.cef_string_set
 0004:00004FCC       ceflib.cef_string_wide_clear
 0004:00004FD0       ceflib.cef_string_utf8_clear
 0004:00004FD4       ceflib.cef_string_utf16_clear
 0004:00004FD8       ceflib.cef_string_clear
 0004:00004FDC       ceflib.cef_string_wide_cmp
 0004:00004FE0       ceflib.cef_string_utf8_cmp
 0004:00004FE4       ceflib.cef_string_utf16_cmp
 0004:00004FE8       ceflib.cef_string_wide_to_utf8
 0004:00004FEC       ceflib.cef_string_utf8_to_wide
 0004:00004FF0       ceflib.cef_string_wide_to_utf16
 0004:00004FF4       ceflib.cef_string_utf16_to_wide
 0004:00004FF8       ceflib.cef_string_utf8_to_utf16
 0004:00004FFC       ceflib.cef_string_utf16_to_utf8
 0004:00005000       ceflib.cef_string_to_utf8
 0004:00005004       ceflib.cef_string_from_utf8
 0004:00005008       ceflib.cef_string_to_utf16
 0004:0000500C       ceflib.cef_string_from_utf16
 0004:00005010       ceflib.cef_string_to_wide
 0004:00005014       ceflib.cef_string_from_wide
 0004:00005018       ceflib.cef_string_ascii_to_wide
 0004:0000501C       ceflib.cef_string_ascii_to_utf16
 0004:00005020       ceflib.cef_string_from_ascii
 0004:00005024       ceflib.cef_string_userfree_wide_alloc
 0004:00005028       ceflib.cef_string_userfree_utf8_alloc
 0004:0000502C       ceflib.cef_string_userfree_utf16_alloc
 0004:00005030       ceflib.cef_string_userfree_alloc
 0004:00005034       ceflib.cef_string_userfree_wide_free
 0004:00005038       ceflib.cef_string_userfree_utf8_free
 0004:0000503C       ceflib.cef_string_userfree_utf16_free
 0004:00005040       ceflib.cef_string_userfree_free
 0004:00005044       ceflib.cef_browser_create
 0004:00005048       ceflib.cef_browser_create_sync
 0004:0000504C       ceflib.cef_do_message_loop_work
 0004:00005050       ceflib.cef_run_message_loop
 0004:00005054       ceflib.cef_initialize
 0004:00005058       ceflib.cef_shutdown
 0004:0000505C       ceflib.cef_string_map_alloc
 0004:00005060       ceflib.cef_string_map_size
 0004:00005064       ceflib.cef_string_map_find
 0004:00005068       ceflib.cef_string_map_key
 0004:0000506C       ceflib.cef_string_map_value
 0004:00005070       ceflib.cef_string_map_append
 0004:00005074       ceflib.cef_string_map_clear
 0004:00005078       ceflib.cef_string_map_free
 0004:0000507C       ceflib.cef_string_list_alloc
 0004:00005080       ceflib.cef_string_list_size
 0004:00005084       ceflib.cef_string_list_value
 0004:00005088       ceflib.cef_string_list_append
 0004:0000508C       ceflib.cef_string_list_clear
 0004:00005090       ceflib.cef_string_list_free
 0004:00005094       ceflib.cef_string_list_copy
 0004:00005098       ceflib.cef_register_extension
 0004:0000509C       ceflib.cef_register_custom_scheme
 0004:000050A0       ceflib.cef_register_scheme_handler_factory
 0004:000050A4       ceflib.cef_clear_scheme_handler_factories
 0004:000050A8       ceflib.cef_add_cross_origin_whitelist_entry
 0004:000050AC       ceflib.cef_remove_cross_origin_whitelist_entry
 0004:000050B0       ceflib.cef_clear_cross_origin_whitelist
 0004:000050B4       ceflib.cef_currently_on
 0004:000050B8       ceflib.cef_post_task
 0004:000050BC       ceflib.cef_post_delayed_task
 0004:000050C0       ceflib.cef_parse_url
 0004:000050C4       ceflib.cef_create_url
 0004:000050C8       ceflib.cef_visit_all_cookies
 0004:000050CC       ceflib.cef_visit_url_cookies
 0004:000050D0       ceflib.cef_set_cookie
 0004:000050D4       ceflib.cef_delete_cookies
 0004:000050D8       ceflib.cef_visit_storage
 0004:000050DC       ceflib.cef_set_storage
 0004:000050E0       ceflib.cef_delete_storage
 0004:000050E4       ceflib.cef_request_create
 0004:000050E8       ceflib.cef_post_data_create
 0004:000050EC       ceflib.cef_post_data_element_create
 0004:000050F0       ceflib.cef_stream_reader_create_for_file
 0004:000050F4       ceflib.cef_stream_reader_create_for_data
 0004:000050F8       ceflib.cef_stream_reader_create_for_handler
 0004:000050FC       ceflib.cef_stream_writer_create_for_file
 0004:00005100       ceflib.cef_stream_writer_create_for_handler
 0004:00005104       ceflib.cef_v8context_get_current_context
 0004:00005108       ceflib.cef_v8context_get_entered_context
 0004:0000510C       ceflib.cef_v8value_create_undefined
 0004:00005110       ceflib.cef_v8value_create_null
 0004:00005114       ceflib.cef_v8value_create_bool
 0004:00005118       ceflib.cef_v8value_create_int
 0004:0000511C       ceflib.cef_v8value_create_double
 0004:00005120       ceflib.cef_v8value_create_date
 0004:00005124       ceflib.cef_v8value_create_string
 0004:00005128       ceflib.cef_v8value_create_object
 0004:0000512C       ceflib.cef_v8value_create_object_with_accessor
 0004:00005130       ceflib.cef_v8value_create_array
 0004:00005134       ceflib.cef_v8value_create_function
 0004:00005138       ceflib.cef_web_urlrequest_create
 0004:0000513C       ceflib.cef_xml_reader_create
 0004:00005140       ceflib.cef_zip_reader_create
 0004:00005144       IOUtils.TPath.FAltDirectorySeparatorChar
 0004:00005146       IOUtils.TPath.FDirectorySeparatorChar
 0004:00005148       IOUtils.TPath.FPathSeparator
 0004:0000514A       IOUtils.TPath.FVolumeSeparatorChar
 0004:0000514C       IOUtils.TPath.FExtensionSeparatorChar
 0004:00005150       IOUtils.TPath.FInvalidPathChars
 0004:00005154       IOUtils.TPath.FInvalidFileNameChars
 0004:00005158       IOUtils.TPath.FPathWildcardChars
 0004:0000515C       IOUtils.TPath.FFileNameWildCardChars
 0004:00005160       IOUtils.TPath.$ClassInitFlag
 0004:00005164       IOUtils..1
 0004:00005168       IniFiles..7
 0004:0000516C       Registry..5
 0004:00005170       cefclient.Window
 0004:00005174       cefclient.backWnd
 0004:00005178       cefclient.forwardWnd
 0004:0000517C       cefclient.reloadWnd
 0004:00005180       cefclient.stopWnd
 0004:00005184       cefclient.editWnd
 0004:00005188       cefclient.editWndOldProc
 0004:0000518C       cefclient.isLoading
 0004:0000518D       cefclient.canGoBack
 0004:0000518E       cefclient.canGoForward
 0004:00005190       cefclient.wndClass
 0005:00000000       System.RaiseListPtr
 0005:00000004       System.InOutRes
 0005:00000008       Classes.TThread.FCurrentThread
 0005:0000000C       Classes.GlobalLoaded
 0005:00000010       Classes.GlobalLists
 0005:00000014       SysInit.TlsLast


Line numbers for ceflib(..\src\ceflib.pas) segment .text

  4220 0001:0003C5E4  4224 0001:0003C5EC  4241 0001:0003C7C4  4242 0001:0003C7C8
  4243 0001:0003C7DD  4247 0001:0003C7E0  4248 0001:0003C7F5  4249 0001:0003C7F8
  4250 0001:0003C803  4251 0001:0003C807  4252 0001:0003C811  4253 0001:0003C81C
  4271 0001:0003CA30  4272 0001:0003CA34  4273 0001:0003CA4D  4277 0001:0003CA50
  4278 0001:0003CA65  4279 0001:0003CA68  4280 0001:0003CA6E  4281 0001:0003CA74
  4282 0001:0003CA7A  4283 0001:0003CA85  4284 0001:0003CA89  4298 0001:0003CC34
  4299 0001:0003CC35  4300 0001:0003CC43  4304 0001:0003CC48  4305 0001:0003CC5D
  4306 0001:0003CC60  4307 0001:0003CC6B  4308 0001:0003CC79  4390 0001:0003CC98
  4391 0001:0003CC9B  4392 0001:0003CCB2  4790 0001:0003CCB4  4791 0001:0003CCBA
  4792 0001:0003CCC2  4793 0001:0003CCCA  4794 0001:0003CCD2  4795 0001:0003CCDA
  4796 0001:0003CCE2  4797 0001:0003CCEA  4798 0001:0003CCF2  4802 0001:0003CCF4
  4803 0001:0003CCF9  4804 0001:0003CD00  4805 0001:0003CD07  4806 0001:0003CD0E
  4807 0001:0003CD15  4808 0001:0003CD1C  4809 0001:0003CD23  4810 0001:0003CD2A
  4815 0001:0003CD2C  4816 0001:0003CD32  4817 0001:0003CD3D  4818 0001:0003CD4E
  4819 0001:0003CD5B  4824 0001:0003CD64  4825 0001:0003CD6D  4826 0001:0003CD7B
  4827 0001:0003CD8A  4828 0001:0003CD94  4925 0001:0003CD9C  4926 0001:0003CD9F
  4927 0001:0003CDAD  4930 0001:0003CDB4  4931 0001:0003CDB7  4932 0001:0003CDC5
  4935 0001:0003CDCC  4936 0001:0003CDCF  4937 0001:0003CDDA  4942 0001:0003CDE0
  4943 0001:0003CDF4  4944 0001:0003CDFE  4945 0001:0003CE1A  4948 0001:0003CE40
  4949 0001:0003CE54  4950 0001:0003CE5E  4951 0001:0003CE7A  4954 0001:0003CEA0
  4955 0001:0003CEB4  4956 0001:0003CEBE  4957 0001:0003CEDA  4960 0001:0003CF00
  4961 0001:0003CF14  4962 0001:0003CF1E  4963 0001:0003CF3A  4966 0001:0003CF60
  4967 0001:0003CF74  4968 0001:0003CF7E  4969 0001:0003CF9A  4972 0001:0003CFC0
  4973 0001:0003CFD4  4974 0001:0003CFDE  4975 0001:0003CFFA  4978 0001:0003D020
  4979 0001:0003D034  4980 0001:0003D03E  4981 0001:0003D05A  4984 0001:0003D080
  4985 0001:0003D094  4986 0001:0003D09E  4987 0001:0003D0BA  4990 0001:0003D0E0
  4991 0001:0003D0F4  4992 0001:0003D0FE  4993 0001:0003D11A  4996 0001:0003D140
  4997 0001:0003D154  4998 0001:0003D15E  4999 0001:0003D17A  5002 0001:0003D1A0
  5003 0001:0003D1B4  5004 0001:0003D1BE  5005 0001:0003D1DA  5008 0001:0003D200
  5009 0001:0003D214  5010 0001:0003D21E  5011 0001:0003D23A  5014 0001:0003D260
  5015 0001:0003D274  5016 0001:0003D27E  5017 0001:0003D29A  5027 0001:0003D2C0
  5028 0001:0003D2DC  5029 0001:0003D2E6  5030 0001:0003D2F8  5031 0001:0003D302
  5039 0001:0003D334  5040 0001:0003D33E  5041 0001:0003D355  5042 0001:0003D35D
  5045 0001:0003D394  5046 0001:0003D3A8  5047 0001:0003D3B2  5048 0001:0003D3CC
  5051 0001:0003D3F0  5052 0001:0003D404  5053 0001:0003D40E  5054 0001:0003D428
  5057 0001:0003D44C  5058 0001:0003D460  5059 0001:0003D46A  5060 0001:0003D489
  5063 0001:0003D4B0  5064 0001:0003D4C4  5065 0001:0003D4CE  5066 0001:0003D4ED
  5072 0001:0003D514  5073 0001:0003D52A  5074 0001:0003D534  5075 0001:0003D563
  5079 0001:0003D590  5080 0001:0003D5A6  5081 0001:0003D5B0  5082 0001:0003D5E3
  5089 0001:0003D610  5090 0001:0003D628  5091 0001:0003D633  5092 0001:0003D63D
  5094 0001:0003D688  5095 0001:0003D68C  5096 0001:0003D697  5234 0001:0003D6D4
  5235 0001:0003D6E8  5236 0001:0003D6F2  5237 0001:0003D71B  5241 0001:0003D740
  5242 0001:0003D758  5243 0001:0003D762  5247 0001:0003D7A0  5251 0001:0003D7D4
  5252 0001:0003D7EA  5253 0001:0003D7F4  5254 0001:0003D81E  5260 0001:0003D84C
  5261 0001:0003D86D  5262 0001:0003D877  5263 0001:0003D881  5265 0001:0003D8A3
  5266 0001:0003D8BF  5270 0001:0003D8F0  5271 0001:0003D906  5272 0001:0003D910
  5273 0001:0003D93E  5278 0001:0003D96C  5279 0001:0003D984  5280 0001:0003D98E
  5282 0001:0003D9D0  5524 0001:0003DA08  5525 0001:0003DA0C  5526 0001:0003DA14
  5527 0001:0003DA23  5530 0001:0003DA28  5531 0001:0003DA2C  5532 0001:0003DA34
  5533 0001:0003DA3F  5536 0001:0003DA44  5537 0001:0003DA47  5538 0001:0003DA4F
  5539 0001:0003DA54  5542 0001:0003DA58  5543 0001:0003DA5C  5544 0001:0003DA66
  5545 0001:0003DA70  5596 0001:0003DA78  5597 0001:0003DA90  5598 0001:0003DA9A
  5600 0001:0003DAEE  5608 0001:0003DB2C  5609 0001:0003DB44  5610 0001:0003DB4E
  5612 0001:0003DB84  5613 0001:0003DB8A  5614 0001:0003DB95  5621 0001:0003DBCC
  5622 0001:0003DBE9  5624 0001:0003DC2A  5625 0001:0003DC38  5626 0001:0003DC48
  5627 0001:0003DC52  5628 0001:0003DC5B  5630 0001:0003DC76  5632 0001:0003DC86
  5635 0001:0003DCB8  5636 0001:0003DCBB  5637 0001:0003DCC3  5638 0001:0003DCC8
  5643 0001:0003DCCC  5644 0001:0003DCE0  5645 0001:0003DCEA  5647 0001:0003DD14
  5654 0001:0003DD3C  5655 0001:0003DD5A  5657 0001:0003DD92  5658 0001:0003DDA0
  5659 0001:0003DDB0  5660 0001:0003DDBA  5662 0001:0003DDCF  5664 0001:0003DDDF
  5670 0001:0003DE08  5671 0001:0003DE22  5673 0001:0003DE4F  5674 0001:0003DE5D
  5675 0001:0003DE6D  5677 0001:0003DE8B  5679 0001:0003DE9B  5683 0001:0003DEC0
  5684 0001:0003DED4  5685 0001:0003DEDE  5686 0001:0003DEFB  5699 0001:0003DF20
  5700 0001:0003DF47  5701 0001:0003DF5E  5702 0001:0003DF68  5701 0001:0003DF87
  5704 0001:0003DF8A  5706 0001:0003DFCF  5707 0001:0003E006  5708 0001:0003E00E
  5709 0001:0003E02D  5720 0001:0003E0AC  5721 0001:0003E0D3  5722 0001:0003E0EA
  5723 0001:0003E0F4  5722 0001:0003E113  5725 0001:0003E116  5727 0001:0003E160
  5728 0001:0003E197  5729 0001:0003E19F  5730 0001:0003E1BE  5754 0001:0003E23C
  5755 0001:0003E250  5756 0001:0003E272  5761 0001:0003E298  5762 0001:0003E2AC
  5763 0001:0003E2CE  5825 0001:0003E2F4  5826 0001:0003E30E  5828 0001:0003E35D
  5829 0001:0003E394  5834 0001:0003E3F8  5835 0001:0003E410  5837 0001:0003E46A
  5874 0001:0003E4A8  5875 0001:0003E4C2  5876 0001:0003E4CB  5877 0001:0003E4D8
  5878 0001:0003E4DA  5879 0001:0003E4DE  5880 0001:0003E4EA  5881 0001:0003E4EF
  5882 0001:0003E4F7  5883 0001:0003E4FF  5884 0001:0003E507  5887 0001:0003E528
  5888 0001:0003E533  5889 0001:0003E537  5890 0001:0003E53F  5891 0001:0003E548
  5892 0001:0003E554  5895 0001:0003E564  5896 0001:0003E565  5897 0001:0003E56A
  5898 0001:0003E570  5899 0001:0003E574  5903 0001:0003E578  5904 0001:0003E581
  5908 0001:0003E584  5909 0001:0003E58D  5914 0001:0003E590  5915 0001:0003E5A5
  5916 0001:0003E5BD  5917 0001:0003E5C0  5920 0001:0003E660  5921 0001:0003E66B
  5922 0001:0003E674  5923 0001:0003E678  5924 0001:0003E684  5927 0001:0003E694
  5928 0001:0003E69D  5929 0001:0003E6A1  5930 0001:0003E6C0  5931 0001:0003E6C7
  5934 0001:0003E6DC  5935 0001:0003E6DD  5936 0001:0003E6E2  5937 0001:0003E6E8
  5938 0001:0003E6EC  5943 0001:0003E6F0  5944 0001:0003E6F4  5945 0001:0003E700
  5948 0001:0003E704  5949 0001:0003E708  5950 0001:0003E714  5954 0001:0003E718
  5955 0001:0003E71F  5959 0001:0003E720  5960 0001:0003E727  5964 0001:0003E728
  5965 0001:0003E72F  5971 0001:0003E730  5972 0001:0003E73F  5973 0001:0003E749
  5975 0001:0003E767  5978 0001:0003E770  5979 0001:0003E777  5980 0001:0003E78C
  5985 0001:0003E790  5986 0001:0003E79C  5987 0001:0003E7A5  5988 0001:0003E7BB
  5995 0001:0003E7C4  5996 0001:0003E7E4  5997 0001:0003E7ED  5998 0001:0003E7FB
  5999 0001:0003E806  6000 0001:0003E815  6002 0001:0003E82A  6003 0001:0003E83C
  6004 0001:0003E851  6000 0001:0003E852  6006 0001:0003E862  6008 0001:0003E875
  6011 0001:0003E89C  6012 0001:0003E8A3  6013 0001:0003E8B8  6017 0001:0003E8BC
  6018 0001:0003E8CA  6019 0001:0003E8E6  6022 0001:0003E8F0  6023 0001:0003E8F7
  6024 0001:0003E90C  6028 0001:0003E910  6029 0001:0003E917  6033 0001:0003E918
  6034 0001:0003E928  6035 0001:0003E93D  6039 0001:0003E948  6040 0001:0003E94F
  6043 0001:0003E950  6044 0001:0003E953  6045 0001:0003E95E  6049 0001:0003E964
  6050 0001:0003E96B  6054 0001:0003E96C  6055 0001:0003E973  6058 0001:0003E974
  6059 0001:0003E978  6060 0001:0003E984  6064 0001:0003E988  6065 0001:0003E992
  6069 0001:0003E994  6070 0001:0003E99F  6073 0001:0003E9A0  6074 0001:0003E9A4
  6075 0001:0003E9B0  6078 0001:0003E9B4  6079 0001:0003E9B8  6080 0001:0003E9C7
  6083 0001:0003E9CC  6084 0001:0003E9D0  6085 0001:0003E9DC  6089 0001:0003E9E0
  6090 0001:0003E9E7  6094 0001:0003E9E8  6095 0001:0003E9EF  6099 0001:0003E9F0
  6100 0001:0003E9F7  6104 0001:0003E9F8  6105 0001:0003EA02  6109 0001:0003EA04
  6110 0001:0003EA12  6113 0001:0003EA14  6114 0001:0003EA19  6115 0001:0003EA33
  6119 0001:0003EA3C  6120 0001:0003EA41  6121 0001:0003EA5A  6124 0001:0003EA60
  6125 0001:0003EA65  6126 0001:0003EA76  6129 0001:0003EA7C  6130 0001:0003EA81
  6131 0001:0003EA91  6135 0001:0003EA98  6136 0001:0003EAA3  6140 0001:0003EAA4
  6141 0001:0003EAA9  6142 0001:0003EAB9  6145 0001:0003EAC0  6146 0001:0003EAC3
  6147 0001:0003EAD0  6151 0001:0003EAD4  6152 0001:0003EADB  6156 0001:0003EADC
  6157 0001:0003EAE7  6161 0001:0003EAE8  6162 0001:0003EAEF  6165 0001:0003EAF0
  6166 0001:0003EAF9  6167 0001:0003EAFD  6168 0001:0003EB1C  6169 0001:0003EB23
  6175 0001:0003EB38  6176 0001:0003EB3F  6180 0001:0003EB40  6181 0001:0003EB47
  6185 0001:0003EB48  6186 0001:0003EB4F  6192 0001:0003EB50  6193 0001:0003EB5F
  6194 0001:0003EB69  6195 0001:0003EB73  6196 0001:0003EB86  6199 0001:0003EB90
  6200 0001:0003EB97  6201 0001:0003EBAC  6204 0001:0003EBB0  6205 0001:0003EBB7
  6206 0001:0003EBC5  6209 0001:0003EBCC  6210 0001:0003EBD3  6211 0001:0003EBE1
  6214 0001:0003EBE8  6215 0001:0003EBEF  6216 0001:0003EBFD  6219 0001:0003EC04
  6220 0001:0003EC0B  6221 0001:0003EC19  6224 0001:0003EC20  6225 0001:0003EC24
  6226 0001:0003EC30  6229 0001:0003EC34  6230 0001:0003EC38  6231 0001:0003EC44
  6237 0001:0003EC48  6238 0001:0003EC70  6239 0001:0003EC7A  6240 0001:0003EC94
  6242 0001:0003EC9A  6243 0001:0003ECA4  6245 0001:0003ECE2  6248 0001:0003ED2C
  6249 0001:0003ED47  6250 0001:0003ED7F  6256 0001:0003EDC0  6257 0001:0003EDEB
  6258 0001:0003EE0F  6260 0001:0003EE15  6261 0001:0003EE20  6263 0001:0003EE5E
  6268 0001:0003EEC0  6269 0001:0003EECC  6270 0001:0003EED5  6271 0001:0003EEE0
  6272 0001:0003EEF1  6277 0001:0003EEF8  6278 0001:0003EF01  6279 0001:0003EF0A
  6280 0001:0003EF12  6284 0001:0003EF18  6285 0001:0003EF1F  6289 0001:0003EF20
  6290 0001:0003EF27  6294 0001:0003EF28  6295 0001:0003EF2F  6299 0001:0003EF30
  6300 0001:0003EF37  6304 0001:0003EF38  6305 0001:0003EF3F  6309 0001:0003EF40
  6310 0001:0003EF47  6313 0001:0003EF48  6314 0001:0003EF63  6315 0001:0003EF9B
  6318 0001:0003EFDC  6319 0001:0003EFF5  6320 0001:0003F023  6323 0001:0003F058
  6324 0001:0003F061  6325 0001:0003F065  6326 0001:0003F084  6327 0001:0003F08B
  6332 0001:0003F0A0  6333 0001:0003F0B9  6334 0001:0003F0C7  6335 0001:0003F0CA
  6336 0001:0003F0D1  6338 0001:0003F0D4  6339 0001:0003F0DB  6340 0001:0003F0E2
  6341 0001:0003F0E9  6343 0001:0003F0F0  6346 0001:0003F110  6347 0001:0003F129
  6348 0001:0003F146  6351 0001:0003F164  6352 0001:0003F16F  6353 0001:0003F175
  6354 0001:0003F17D  6355 0001:0003F189  6358 0001:0003F198  6359 0001:0003F1A1
  6360 0001:0003F1A9  6361 0001:0003F1B7  6363 0001:0003F1ED  6365 0001:0003F1FD
  6368 0001:0003F208  6369 0001:0003F217  6370 0001:0003F21F  6371 0001:0003F22D
  6373 0001:0003F254  6375 0001:0003F264  6378 0001:0003F270  6379 0001:0003F27F
  6380 0001:0003F287  6381 0001:0003F295  6383 0001:0003F2B4  6385 0001:0003F2C4
  6388 0001:0003F2D0  6389 0001:0003F2D9  6390 0001:0003F2E1  6391 0001:0003F2EF
  6393 0001:0003F30A  6395 0001:0003F31A  6401 0001:0003F324  6402 0001:0003F33F
  6403 0001:0003F379  6407 0001:0003F3BC  6408 0001:0003F3C3  6411 0001:0003F3C4
  6412 0001:0003F3CE  6413 0001:0003F3E4  6416 0001:0003F3EC  6417 0001:0003F3F2
  6418 0001:0003F403  6422 0001:0003F408  6423 0001:0003F423  6424 0001:0003F45D
  6428 0001:0003F4A0  6429 0001:0003F4A7  6432 0001:0003F4A8  6433 0001:0003F4B1
  6434 0001:0003F4B5  6435 0001:0003F4D4  6436 0001:0003F4DB  6442 0001:0003F4F0
  6443 0001:0003F4F1  6444 0001:0003F4FA  6448 0001:0003F4FC  6449 0001:0003F503
  6452 0001:0003F504  6453 0001:0003F50B  6454 0001:0003F519  6458 0001:0003F520
  6459 0001:0003F527  6462 0001:0003F528  6463 0001:0003F52E  6464 0001:0003F53F
  6467 0001:0003F544  6468 0001:0003F545  6469 0001:0003F54E  6473 0001:0003F550
  6474 0001:0003F557  6479 0001:0003F558  6480 0001:0003F561  6481 0001:0003F56A
  6482 0001:0003F572  6485 0001:0003F578  6486 0001:0003F581  6487 0001:0003F585
  6488 0001:0003F5A4  6489 0001:0003F5AB  6617 0001:0003F5C0  6618 0001:0003F5C7
  6619 0001:0003F5D5  6623 0001:0003F5DC  6624 0001:0003F5E3  6627 0001:0003F5E4
  6628 0001:0003F5EB  6629 0001:0003F5FA  6632 0001:0003F600  6633 0001:0003F607
  6634 0001:0003F615  6637 0001:0003F61C  6638 0001:0003F623  6639 0001:0003F638
  6642 0001:0003F63C  6643 0001:0003F643  6644 0001:0003F651  6647 0001:0003F658
  6648 0001:0003F65E  6649 0001:0003F66F  6654 0001:0003F674  6655 0001:0003F67D
  6656 0001:0003F686  6657 0001:0003F68E  6661 0001:0003F694  6662 0001:0003F69C
  6665 0001:0003F6A0  6666 0001:0003F6A7  6667 0001:0003F6B6  6672 0001:0003F6BC
  6673 0001:0003F6C5  6674 0001:0003F6CE  6675 0001:0003F6D6  6678 0001:0003F6DC
  6679 0001:0003F6F7  6680 0001:0003F6FB  6681 0001:0003F733  6686 0001:0003F774
  6687 0001:0003F77D  6688 0001:0003F786  6689 0001:0003F78E  6692 0001:0003F794
  6693 0001:0003F79D  6694 0001:0003F7A1  6695 0001:0003F7C0  6696 0001:0003F7C7
  6702 0001:0003F7DC  6703 0001:0003F7FA  6704 0001:0003F83F  6707 0001:0003F880
  6708 0001:0003F88C  6709 0001:0003F8A3  6714 0001:0003F8AC  6715 0001:0003F8B8
  6716 0001:0003F8C1  6717 0001:0003F8D4  6721 0001:0003F8DC  6722 0001:0003F8F8
  6723 0001:0003F92A  6726 0001:0003F960  6727 0001:0003F964  6728 0001:0003F970
  6731 0001:0003F974  6732 0001:0003F979  6733 0001:0003F986  6736 0001:0003F98C
  6737 0001:0003F98D  6738 0001:0003F996  6742 0001:0003F998  6743 0001:0003F99F
  6746 0001:0003F9A0  6747 0001:0003F9A9  6748 0001:0003F9AD  6749 0001:0003F9CC
  6750 0001:0003F9D3  6759 0001:0003F9E8  6760 0001:0003F9F1  6763 0001:0003FA31
  6773 0001:0003FA34  6774 0001:0003FA5C  6777 0001:0003FA65  6779 0001:0003FA73
  6780 0001:0003FA85  6781 0001:0003FA8A  6783 0001:0003FA8F  6784 0001:0003FAA1
  6785 0001:0003FAB3  6786 0001:0003FAC5  6787 0001:0003FAD7  6788 0001:0003FAE9
  6789 0001:0003FAFB  6790 0001:0003FB0D  6791 0001:0003FB1F  6792 0001:0003FB31
  6793 0001:0003FB43  6794 0001:0003FB55  6795 0001:0003FB67  6796 0001:0003FB79
  6797 0001:0003FB8B  6798 0001:0003FB9D  6799 0001:0003FBAF  6800 0001:0003FBC1
  6801 0001:0003FBD3  6802 0001:0003FBE5  6803 0001:0003FBF7  6804 0001:0003FC09
  6805 0001:0003FC1B  6822 0001:0003FC2D  6823 0001:0003FC37  6824 0001:0003FC41
  6825 0001:0003FC4B  6826 0001:0003FC55  6827 0001:0003FC5F  6828 0001:0003FC69
  6829 0001:0003FC73  6830 0001:0003FC7D  6831 0001:0003FC87  6832 0001:0003FC91
  6849 0001:0003FC9B  6850 0001:0003FCAD  6851 0001:0003FCBF  6852 0001:0003FCD1
  6853 0001:0003FCE3  6854 0001:0003FCF5  6855 0001:0003FD07  6856 0001:0003FD19
  6857 0001:0003FD2B  6858 0001:0003FD3D  6859 0001:0003FD4F  6860 0001:0003FD61
  6861 0001:0003FD73  6862 0001:0003FD85  6863 0001:0003FD97  6864 0001:0003FDA9
  6865 0001:0003FDBB  6866 0001:0003FDCD  6867 0001:0003FDDF  6868 0001:0003FDF1
  6869 0001:0003FE03  6870 0001:0003FE15  6871 0001:0003FE27  6872 0001:0003FE39
  6873 0001:0003FE4B  6874 0001:0003FE5D  6875 0001:0003FE6F  6876 0001:0003FE81
  6877 0001:0003FE93  6878 0001:0003FEA5  6879 0001:0003FEB7  6880 0001:0003FEC9
  6881 0001:0003FEDB  6882 0001:0003FEED  6883 0001:0003FEFF  6884 0001:0003FF11
  6885 0001:0003FF23  6886 0001:0003FF35  6887 0001:0003FF47  6888 0001:0003FF59
  6889 0001:0003FF6B  6890 0001:0003FF7D  6891 0001:0003FF8F  6892 0001:0003FFA1
  6893 0001:0003FFB3  6894 0001:0003FFC5  6895 0001:0003FFD7  6896 0001:0003FFE9
  6897 0001:0003FFFB  6898 0001:0004000D  6899 0001:0004001F  6900 0001:00040031
  6901 0001:00040043  6902 0001:00040055  6903 0001:00040067  6904 0001:00040079
  6905 0001:0004008B  6906 0001:0004009D  6907 0001:000400AF  6908 0001:000400C1
  6909 0001:000400D3  6910 0001:000400E5  6911 0001:000400F7  6912 0001:00040109
  6914 0001:0004011B  7003 0001:0004054A  7005 0001:00040560  7006 0001:0004056F
  7008 0001:00040576  7012 0001:0004057A  7013 0001:00040596  7014 0001:000405B2
  7015 0001:000405CF  7016 0001:000405EC  7018 0001:000405F6  7019 0001:000405FF
  7020 0001:0004060E  7021 0001:0004061C  7022 0001:00040628  7023 0001:00040633
  7025 0001:00040645  7026 0001:0004065D  7027 0001:0004066E  7023 0001:0004066F
  7029 0001:0004067F  7032 0001:0004068F  7033 0001:000406AC  7034 0001:000406B2
  7035 0001:000406B8  7036 0001:000406BE  7037 0001:000406C4  7038 0001:000406CF
  7039 0001:000406D6  7041 0001:000406DE  7047 0001:0004183C  7048 0001:0004184B
  7049 0001:00041850  7050 0001:0004185A  7056 0001:00041872  7082 0001:0004187C
  7083 0001:00041885  7084 0001:0004188B  7089 0001:0004188C  7090 0001:000418AC
  7091 0001:000418B6  7092 0001:000418C6  7093 0001:000418CB  7096 0001:000418EC
  7097 0001:000418EF  7098 0001:000418F3  7099 0001:00041902  7100 0001:0004190B
  7118 0001:00041910  7119 0001:00041930  7120 0001:0004193E  7121 0001:00041944
  7122 0001:00041965  7125 0001:00041988  7126 0001:000419A8  7127 0001:000419AC
  7128 0001:000419CF  7131 0001:000419F0  7132 0001:000419F6  7133 0001:000419FF
  7134 0001:00041A07  7137 0001:00041A0C  7138 0001:00041A12  7140 0001:00041A16
  7141 0001:00041A1F  7143 0001:00041A2A  7144 0001:00041A33  7156 0001:00041A38
  7157 0001:00041A5A  7158 0001:00041A5F  7159 0001:00041A69  7160 0001:00041A73
  7164 0001:00041AC4  7176 0001:00041AFC  7177 0001:00041B0B  7178 0001:00041B10
  7179 0001:00041B1A  7181 0001:00041B3A  7218 0001:00041B44  7219 0001:00041B69
  7220 0001:00041B6E  7221 0001:00041B78  7222 0001:00041B82  7223 0001:00041BCD
  7243 0001:00041C10  7244 0001:00041C29  7245 0001:00041C37  7246 0001:00041C3A
  7247 0001:00041C42  7248 0001:00041C45  7249 0001:00041C4C  7253 0001:00041C6C
  7254 0001:00041C78  7255 0001:00041CA0  7262 0001:00041CB8  7263 0001:00041CBC
  7267 0001:00041CC0  7268 0001:00041CD9  7269 0001:00041CE7  7270 0001:00041CEB
  7271 0001:00041CF6  7272 0001:00041D01  7273 0001:00041D0C  7275 0001:00041D0F
  7277 0001:00041D13  7278 0001:00041D1B  7279 0001:00041D23  7282 0001:00041D2D
  7283 0001:00041D35  7284 0001:00041D3D  7286 0001:00041D45  7288 0001:00041D4D
  7294 0001:00041D70  7298 0001:00041D74  7299 0001:00041D77  7300 0001:00041D79
  7304 0001:00041D80  7305 0001:00041D83  7306 0001:00041D85  7311 0001:00041D8C
  7312 0001:00041D92  7313 0001:00041DA3  7316 0001:00041DA8  7317 0001:00041DB1
  7318 0001:00041DC7  7323 0001:00041DCC  7324 0001:00041DD8  7325 0001:00041DE6
  7326 0001:00041DFC  7329 0001:00041E04  7330 0001:00041E0D  7331 0001:00041E27
  7337 0001:00041E30  7338 0001:00041E55  7339 0001:00041E5F  7340 0001:00041EAB
  7343 0001:00041EEC  7344 0001:00041EF5  7345 0001:00041F08  7348 0001:00041F0C
  7349 0001:00041F12  7350 0001:00041F23  7353 0001:00041F28  7354 0001:00041F46
  7355 0001:00041F8B  7359 0001:00041FCC  7360 0001:00041FEE  7361 0001:00042069
  7366 0001:000420AC  7367 0001:000420C8  7369 0001:00042100  7374 0001:00042138
  7375 0001:00042144  7376 0001:0004214D  7377 0001:00042160  7380 0001:00042168
  7381 0001:0004216E  7382 0001:0004217F  7385 0001:00042184  7386 0001:0004218B
  7387 0001:00042198  7392 0001:0004219C  7393 0001:000421A5  7394 0001:000421AE
  7395 0001:000421BB  7405 0001:000421C4  7406 0001:000421F7  7407 0001:0004220A
  7408 0001:00042218  7409 0001:00042229  7408 0001:00042262  7410 0001:00042265
  7411 0001:0004226A  7412 0001:00042279  7414 0001:000422D5  7415 0001:000422F0
  7417 0001:00042313  7419 0001:00042323  7429 0001:00042378  7430 0001:000423B5
  7431 0001:000423C8  7432 0001:000423D6  7433 0001:000423E7  7432 0001:00042420
  7434 0001:00042423  7435 0001:00042428  7436 0001:00042437  7438 0001:000424CE
  7439 0001:000424E9  7441 0001:0004250C  7443 0001:0004251C  7447 0001:00042574
  7448 0001:0004257B  7451 0001:0004257C  7452 0001:00042580  7453 0001:0004258C
  7456 0001:00042590  7457 0001:00042597  7458 0001:000425B0  7461 0001:000425BC
  7462 0001:000425BF  7463 0001:000425CA  7466 0001:000425D0  7467 0001:000425D7
  7468 0001:000425EF  7471 0001:000425F4  7472 0001:000425FB  7473 0001:0004260C
  7477 0001:00042610  7478 0001:00042617  7485 0001:00042618  7486 0001:00042638
  7487 0001:00042641  7488 0001:0004264F  7489 0001:0004265D  7490 0001:0004266C
  7492 0001:00042681  7493 0001:00042693  7494 0001:000426A8  7490 0001:000426A9
  7496 0001:000426B9  7498 0001:000426CC  7501 0001:000426F4  7502 0001:000426FB
  7503 0001:00042709  7506 0001:00042710  7507 0001:00042717  7508 0001:0004272C
  7511 0001:00042730  7512 0001:0004273A  7513 0001:00042750  7518 0001:00042758
  7519 0001:00042764  7520 0001:0004276D  7521 0001:00042783  7524 0001:0004278C
  7525 0001:00042793  7526 0001:000427A0  7531 0001:000427A4  7532 0001:000427AD
  7533 0001:000427B6  7534 0001:000427C3  7537 0001:000427CC  7538 0001:000427D0
  7539 0001:000427DC  7542 0001:000427E0  7543 0001:000427E4  7544 0001:000427F0
  7547 0001:000427F4  7548 0001:000427F8  7549 0001:00042804  7552 0001:00042808
  7553 0001:0004280C  7554 0001:00042818  7557 0001:0004281C  7558 0001:00042820
  7559 0001:0004282C  7562 0001:00042830  7563 0001:00042834  7564 0001:00042840
  7567 0001:00042844  7568 0001:00042848  7569 0001:00042854  7572 0001:00042858
  7573 0001:0004285C  7574 0001:00042868  7577 0001:0004286C  7578 0001:00042888
  7579 0001:000428C9  7582 0001:0004290C  7583 0001:00042910  7584 0001:0004291C
  7587 0001:00042920  7588 0001:00042924  7589 0001:00042930  7595 0001:00042934
  7596 0001:00042943  7597 0001:0004294D  7598 0001:00042962  7602 0001:0004296C
  7603 0001:0004298D  7604 0001:000429D2  7610 0001:00042A14  7611 0001:00042A39
  7612 0001:00042A43  7613 0001:00042A88  7616 0001:00042ACC  7617 0001:00042AD5
  7618 0001:00042AD9  7619 0001:00042AF8  7620 0001:00042AFF  7633 0001:00042B4C
  7634 0001:00042B86  7635 0001:00042BA4  7636 0001:00042BB5  7635 0001:00042BEE
  7637 0001:00042BF1  7638 0001:00042BF6  7639 0001:00042C05  7640 0001:00042C10
  7642 0001:00042C6E  7643 0001:00042C89  7644 0001:00042C9F  7655 0001:00042D38
  7656 0001:00042D69  7657 0001:00042D87  7658 0001:00042D98  7657 0001:00042DD1
  7659 0001:00042DD4  7660 0001:00042DD9  7661 0001:00042DE8  7663 0001:00042E7D
  7664 0001:00042E98  7665 0001:00042EAE  7668 0001:00042F10  7669 0001:00042F19
  7670 0001:00042F1D  7671 0001:00042F3C  7672 0001:00042F43  7677 0001:00042F58
  7678 0001:00042F6A  7679 0001:00042F78  7681 0001:00042F7B  7682 0001:00042F83
  7684 0001:00042F8B  7689 0001:00042FA8  7690 0001:00042FAB  7691 0001:00042FAD
  7697 0001:00042FB4  7698 0001:00042FB7  7699 0001:00042FB9  8108 0001:00042FC0
  8109 0001:00042FC6  8110 0001:00042FD7  8113 0001:00042FDC  8114 0001:00042FE0
  8115 0001:00042FEC  8118 0001:00042FF0  8119 0001:00042FF6  8120 0001:00043007
  8123 0001:0004300C  8124 0001:00043010  8125 0001:0004301C  8128 0001:00043020
  8129 0001:00043027  8130 0001:0004303C  8133 0001:00043040  8134 0001:00043047
  8135 0001:0004305C  8138 0001:00043060  8139 0001:00043067  8140 0001:0004307C
  8143 0001:00043080  8144 0001:00043089  8145 0001:0004308D  8146 0001:000430AC
  8147 0001:000430B3  8152 0001:000430C8  8153 0001:000430DA  8154 0001:000430E8
  8155 0001:000430EB  8156 0001:000430F3  8161 0001:00043110  8166 0001:00043114
  8167 0001:00043129  8168 0001:00043132  8169 0001:0004313C  8173 0001:00043158
  8174 0001:00043160  8179 0001:00043164  8180 0001:0004316B  8181 0001:00043179
  8184 0001:00043180  8185 0001:00043187  8186 0001:0004319C  8191 0001:000431A0
  8192 0001:000431AC  8193 0001:000431B5  8194 0001:000431C4  8197 0001:000431CC
  8198 0001:000431D3  8199 0001:000431E8  8204 0001:000431EC  8205 0001:000431F8
  8206 0001:00043201  8207 0001:00043217  8210 0001:00043220  8211 0001:00043227
  8212 0001:0004323C  8215 0001:00043240  8216 0001:00043247  8217 0001:0004325C
  8220 0001:00043260  8221 0001:00043267  8222 0001:00043275  8225 0001:0004327C
  8226 0001:00043283  8227 0001:00043291  8230 0001:00043298  8231 0001:0004329F
  8232 0001:000432B4  8236 0001:000432B8  8237 0001:000432BF  8240 0001:000432C0
  8241 0001:000432C7  8242 0001:000432DC  8246 0001:000432E0  8247 0001:000432E7
  8250 0001:000432E8  8251 0001:000432EF  8252 0001:000432FD  8256 0001:00043304
  8257 0001:0004330B  8260 0001:0004330C  8261 0001:00043310  8262 0001:0004331C
  8265 0001:00043320  8266 0001:00043329  8267 0001:0004332D  8268 0001:0004334C
  8269 0001:00043353  8277 0001:00043368  8278 0001:00043391  8279 0001:0004339B
  8280 0001:000433DC  8284 0001:00043420  8285 0001:0004343C  8286 0001:00043470
  8289 0001:000434A8  8290 0001:000434AF  8291 0001:000434BD  8294 0001:000434C4
  8295 0001:000434CB  8296 0001:000434E0  8301 0001:000434E4  8302 0001:000434F0
  8303 0001:000434F9  8304 0001:00043508  8307 0001:00043510  8308 0001:00043517
  8309 0001:00043526  8312 0001:0004352C  8313 0001:00043533  8314 0001:00043541
  8317 0001:00043548  8318 0001:0004354F  8319 0001:0004355D  8322 0001:00043564
  8323 0001:0004356B  8324 0001:00043580  8327 0001:00043584  8328 0001:0004358B
  8329 0001:000435A0  8332 0001:000435A4  8333 0001:000435AB  8334 0001:000435B9
  8337 0001:000435C0  8338 0001:000435C7  8339 0001:000435DC  8342 0001:000435E0
  8343 0001:000435E7  8344 0001:000435FC  8347 0001:00043600  8348 0001:00043607
  8349 0001:0004361C  8353 0001:00043620  8354 0001:00043627  8357 0001:00043628
  8358 0001:0004362F  8359 0001:0004363D  8362 0001:00043644  8363 0001:00043648
  8364 0001:00043654  8369 0001:00043658  8370 0001:00043661  8371 0001:0004366A
  8372 0001:00043677  8375 0001:00043680  8376 0001:00043684  8377 0001:00043690
  8380 0001:00043694  8381 0001:00043698  8382 0001:000436A4  8385 0001:000436A8
  8386 0001:000436C4  8387 0001:00043705  8390 0001:00043748  8391 0001:0004374C
  8392 0001:00043758  8398 0001:0004375C  8399 0001:00043768  8400 0001:00043771
  8401 0001:0004377C  8402 0001:00043792  8407 0001:0004379C  8408 0001:000437A5
  8409 0001:000437AE  8410 0001:000437BB  8413 0001:000437C4  8414 0001:000437CD
  8415 0001:000437D1  8416 0001:000437F0  8417 0001:000437F7  8422 0001:0004380C
  8423 0001:0004381E  8424 0001:0004382C  8425 0001:0004382F  8426 0001:00043837
  8431 0001:00043854  8436 0001:00043858  8437 0001:0004385C  8438 0001:00043868
  8441 0001:0004386C  8442 0001:00043870  8443 0001:0004387C  8447 0001:00043880
  8448 0001:00043887  8451 0001:00043888  8452 0001:0004388F  8453 0001:000438A4
  8456 0001:000438A8  8457 0001:000438AF  8458 0001:000438C4  8462 0001:000438C8
  8463 0001:000438CF  8466 0001:000438D0  8467 0001:000438D7  8468 0001:000438EC
  8471 0001:000438F0  8472 0001:000438F7  8473 0001:00043905  8476 0001:0004390C
  8477 0001:00043915  8478 0001:00043919  8479 0001:00043938  8480 0001:0004393F
  8486 0001:00043954  8487 0001:00043969  8488 0001:00043972  8489 0001:0004397C
  8492 0001:00043998  8493 0001:0004399E  8494 0001:000439A7  8495 0001:000439B1
  8502 0001:000439B4  8503 0001:000439C0  8504 0001:000439C9  8505 0001:000439D8
  8508 0001:000439E0  8509 0001:000439E7  8510 0001:000439F6  8513 0001:000439FC
  8514 0001:00043A03  8515 0001:00043A11  8519 0001:00043A18  8520 0001:00043A1F
  8523 0001:00043A20  8524 0001:00043A27  8525 0001:00043A35  8528 0001:00043A3C
  8529 0001:00043A43  8530 0001:00043A52  8535 0001:00043A58  8536 0001:00043A61
  8537 0001:00043A6A  8538 0001:00043A72  8542 0001:00043A78  8543 0001:00043A80
  8548 0001:00043A84  8549 0001:00043A8D  8550 0001:00043A96  8551 0001:00043A9E
  8554 0001:00043AA4  8555 0001:00043AAD  8556 0001:00043AB1  8557 0001:00043AD0
  8558 0001:00043AD7  9343 0001:00043AEC  9344 0001:00043AFE  9345 0001:00043B0C
  9346 0001:00043B17  9347 0001:00043B1F  9351 0001:00043B3C  9352 0001:00043B4A
  9353 0001:00043B4C  9357 0001:00043B50  9358 0001:00043B53  9359 0001:00043B55
  9366 0001:00043B5C  9367 0001:00043B74  9368 0001:00043B7E  9369 0001:00043B89
  9373 0001:00043BA8  9374 0001:00043BBF  9375 0001:00043BC5  9376 0001:00043BE0
  9377 0001:00043BE2  9381 0001:00043BEC  9382 0001:00043BF0  9383 0001:00043BF6
  9384 0001:00043C08  9385 0001:00043C0A  9451 0001:00043C10  9452 0001:00043C22
  9453 0001:00043C30  9455 0001:00043C33  9456 0001:00043C3B  9457 0001:00043C43
  9458 0001:00043C4B  9459 0001:00043C53  9460 0001:00043C5B  9461 0001:00043C63
  9462 0001:00043C6B  9463 0001:00043C73  9464 0001:00043C7B  9465 0001:00043C83
  9466 0001:00043C8B  9467 0001:00043C93  9469 0001:00043C9B  9472 0001:00043CB8
  9473 0001:00043CBB  9474 0001:00043CC2  9477 0001:00043CC4  9478 0001:00043CC7
  9479 0001:00043CCE  9482 0001:00043CD0  9483 0001:00043CD3  9484 0001:00043CDA
  9487 0001:00043CDC  9488 0001:00043CDF  9489 0001:00043CE6  9492 0001:00043CE8
  9493 0001:00043CEB  9494 0001:00043CF2  9497 0001:00043CF4  9498 0001:00043CF7
  9499 0001:00043CFE  9502 0001:00043D00  9503 0001:00043D03  9504 0001:00043D0A
  9507 0001:00043D0C  9508 0001:00043D0F  9509 0001:00043D16  9512 0001:00043D18
  9513 0001:00043D1B  9514 0001:00043D22  9517 0001:00043D24  9518 0001:00043D27
  9519 0001:00043D2E  9522 0001:00043D30  9523 0001:00043D33  9524 0001:00043D3A
  9527 0001:00043D3C  9528 0001:00043D3F  9529 0001:00043D46  9532 0001:00043D48
  9533 0001:00043D4B  9534 0001:00043D52  9539 0001:00043D54  9540 0001:00043D66
  9541 0001:00043D74  9543 0001:00043D77  9544 0001:00043D7F  9545 0001:00043D87
  9546 0001:00043D8F  9547 0001:00043D97  9549 0001:00043D9F  9554 0001:00043DBC
  9559 0001:00043DC0  9565 0001:00043DC4  9566 0001:00043DC7  9567 0001:00043DC9
  9571 0001:00043DD0  9572 0001:00043DD2  9576 0001:00043DD4  9577 0001:00043DD6
  9583 0001:00043DD8  9584 0001:00043DEA  9585 0001:00043DF8  9587 0001:00043DFB
  9588 0001:00043E03  9589 0001:00043E0B  9591 0001:00043E13  9595 0001:00043E30
  9597 0001:00043E33  9602 0001:00043E38  9603 0001:00043E3B  9604 0001:00043E3D
  9610 0001:00043E44  9697 0001:00043E48  9698 0001:00043E5A  9699 0001:00043E68
  9701 0001:00043E6B  9702 0001:00043E73  9703 0001:00043E7B  9704 0001:00043E83
  9705 0001:00043E8B  9706 0001:00043E93  9708 0001:00043E9B  9712 0001:00043EB8
  9714 0001:00043EBB  9718 0001:00043EC0  9719 0001:00043EC3  9720 0001:00043EC5
  9724 0001:00043ECC  9726 0001:00043ECF  9730 0001:00043ED4  9732 0001:00043ED7
  9738 0001:00043EDC  9743 0001:00043EE0  9744 0001:00043EE2  9994 0001:00043EE4
  9995 0001:00043EEB  9999 0001:00043EEC 10000 0001:00043EF3 10004 0001:00043EF4
 10005 0001:00043EFB 10009 0001:00043EFC 10010 0001:00043F05 10011 0001:00043F09
 10012 0001:00043F28 10013 0001:00043F2F 10102 0001:00043F44 10104 0001:00043F66
 10105 0001:00043F6C 10108 0001:00043F77

Line numbers for ceflib(..\src\ceflib.pas) segment .itext

 10098 0002:00000338 10099 0002:00000341 10101 0002:00000349

Line numbers for ceffilescheme(..\filescheme\ceffilescheme.pas) segment .text

    55 0001:00047A08    56 0001:00047A26    57 0001:00047A2F    60 0001:00047A3A
    61 0001:00047A41    62 0001:00047A69    63 0001:00047A74    64 0001:00047A96
    65 0001:00047AAA    58 0001:00047AAD    67 0001:00047AB5    82 0001:00047D14
    83 0001:00047D37    84 0001:00047D41    85 0001:00047D4D    86 0001:00047D59
    87 0001:00047D5F    98 0001:00047D80    99 0001:00047D89   100 0001:00047DC5
   101 0001:00047E12   102 0001:00047E5F   103 0001:00047EAC   104 0001:00047EF6
   105 0001:00047F40   106 0001:00047F4C   113 0001:00048020   114 0001:0004803C
   115 0001:00048049   116 0001:00048056   118 0001:00048088   119 0001:000480A2
   124 0001:000480C4   125 0001:000480EA   126 0001:000480F5   127 0001:000480FE
   128 0001:00048155   132 0001:000481F8   134 0001:00048203   135 0001:0004820E
   136 0001:0004821B   138 0001:0004821F   139 0001:0004822A   140 0001:00048237
   141 0001:0004823C   147 0001:00048240   148 0001:00048261   149 0001:00048270
   150 0001:000482A3   151 0001:000482AD   154 0001:000482BB   155 0001:000482C5
   157 0001:000482CA   158 0001:000482CB   159 0001:000482D0   162 0001:000482D5
   163 0001:000482D8   164 0001:000482D9   165 0001:000482E6   168 0001:00048323
   169 0001:0004832B   174 0001:0004832D   176 0001:0004832F   177 0001:00048330
   152 0001:00048331   179 0001:00048338   180 0001:00048350   188 0001:00048394
   189 0001:000483B9   190 0001:000483BB   193 0001:000483C4   194 0001:000483F6
   195 0001:00048405   196 0001:00048414   197 0001:00048423   198 0001:00048432
   199 0001:00048441   200 0001:00048450   201 0001:0004845F   203 0001:00048465
   205 0001:00048468   212 0001:000484AB   221 0001:00048500   222 0001:00048503
   191 0001:00048504   225 0001:00048509   226 0001:00048512   232 0001:00048598
   234 0001:0004859D   238 0001:000485A0   239 0001:000485B5   240 0001:000485CA
   241 0001:000485CF   244 0001:000485EC   245 0001:000485F7   246 0001:000485FE
   247 0001:00048603   248 0001:0004860F   252 0001:00048620   253 0001:00048629
   254 0001:00048633   255 0001:0004863D   256 0001:00048647   257 0001:00048653
   273 0001:00048658   275 0001:0004866E   276 0001:0004867D   280 0001:000486E3
   285 0001:00048704   287 0001:0004871A   291 0001:00048729   292 0001:0004878F
   294 0001:000487B0   295 0001:000487EA   297 0001:000487F1   298 0001:00048820
   300 0001:0004883B   301 0001:00048845   302 0001:00048855   304 0001:00048860
   305 0001:00048872   306 0001:00048880   307 0001:00048890   308 0001:000488B8
   309 0001:000488E1   310 0001:00048915   312 0001:00048932   314 0001:00048945
   315 0001:0004894E   316 0001:0004895E   318 0001:0004897D   320 0001:00048990
   321 0001:0004899A   322 0001:000489AA   323 0001:000489BE   324 0001:000489CC
   325 0001:000489EE   326 0001:00048A00   327 0001:00048A1F   328 0001:00048A2D
   330 0001:00048A4B   333 0001:00048A5E   335 0001:00048AA8   338 0001:00048AD8
   339 0001:00048AEA   340 0001:00048B23   341 0001:00048B32   343 0001:00048B3D
   345 0001:00048B4D   346 0001:00048B5E   345 0001:00048B84   348 0001:00048B87
   349 0001:00048B96   351 0001:00048BB3   355 0001:00048BC6   356 0001:00048BD0
   359 0001:00048BE0   361 0001:00048BF2   363 0001:00048C1F   364 0001:00048C2F
   367 0001:00048C3E   368 0001:00048C46   369 0001:00048C4E   373 0001:00048F7C
   374 0001:00048F89   375 0001:00048F9B   376 0001:00048F9D   378 0001:00048FAB

Line numbers for cefclient(cefclient.dpr) segment .text

   115 0001:0004958C   116 0001:000495BA   117 0001:000495C6   119 0001:000495D3
   122 0001:000495DD   123 0001:000495EF   124 0001:000495FB   125 0001:0004960F
   127 0001:00049613   128 0001:0004961D   130 0001:00049656   132 0001:0004965D
   134 0001:00049679   136 0001:00049695   139 0001:000496E1   140 0001:000496EB
   141 0001:000496F5   145 0001:000496FC   146 0001:0004971B   147 0001:0004971D
   149 0001:0004972A   153 0001:00049758   155 0001:0004975B   160 0001:00049789
   162 0001:0004978C   167 0001:000497BA   169 0001:000497BD   173 0001:000497EB
   175 0001:000497EE   183 0001:0004981D   184 0001:0004982F   186 0001:00049841
   187 0001:00049850   188 0001:00049854   189 0001:0004985B   190 0001:0004985E
   191 0001:00049867   192 0001:0004986D   193 0001:00049875   194 0001:0004987D
   195 0001:00049899   196 0001:000498A0   197 0001:000498A7   198 0001:000498AE
   199 0001:000498BA   204 0001:000498C1   205 0001:000498CE   206 0001:000498E4
   207 0001:000498FA   208 0001:00049913   209 0001:00049929   212 0001:00049930
   215 0001:0004994B   216 0001:00049955   220 0001:0004995C   221 0001:00049966
   225 0001:0004996D   226 0001:00049977   230 0001:0004997E   231 0001:00049988
   234 0001:0004998F   238 0001:000499A5   239 0001:000499AF   240 0001:000499B6
   244 0001:000499BD   245 0001:000499C6   246 0001:000499D9   250 0001:000499E0
   254 0001:000499E9   255 0001:000499F6   256 0001:000499FA   257 0001:00049A06
   258 0001:00049A0D   259 0001:00049A29   261 0001:00049A51   263 0001:00049A57
   267 0001:00049A6A   268 0001:00049A73   269 0001:00049A7D   272 0001:00049A90
   274 0001:00049AA1   280 0001:00049B2C   281 0001:00049B3E   282 0001:00049B47
   283 0001:00049B64   284 0001:00049B81   285 0001:00049B9E   288 0001:00049BB8
   289 0001:00049BBE   290 0001:00049BC8   293 0001:00049BCC   294 0001:00049BD2
   295 0001:00049BDC   298 0001:00049BE0   299 0001:00049BE6   300 0001:00049BF0
   305 0001:00049BF4   306 0001:00049BF7   309 0001:00049C02   310 0001:00049C0E
   312 0001:00049C1D   318 0001:00049C20   319 0001:00049C26   320 0001:00049C35
   321 0001:00049C3C   325 0001:00049C44   326 0001:00049C47   328 0001:00049C56
   329 0001:00049C5D   330 0001:00049C69   332 0001:00049C75   338 0001:00049C78
   339 0001:00049C81   340 0001:00049C9B   341 0001:00049CAF   345 0001:00049CB8
   346 0001:00049CBE   347 0001:00049CCD   348 0001:00049CE0   354 0001:00049CE4
   355 0001:00049CF9   356 0001:00049D0E   357 0001:00049D1D   360 0001:00049D3C
   361 0001:00049D47   362 0001:00049D4F   363 0001:00049D5B   367 0001:00049D6C
   368 0001:00049D76   369 0001:00049D82   370 0001:00049D8E   371 0001:00049D9A
   372 0001:00049DA6   373 0001:00049DB2   374 0001:00049DBE   375 0001:00049DCA
   376 0001:00049DD6   377 0001:00049DE2   378 0001:00049DEE   379 0001:00049DFA
   380 0001:00049E06   381 0001:00049E12   382 0001:00049E1E   383 0001:00049E25
   384 0001:00049E2C   385 0001:00049E2E   389 0001:0004A220   390 0001:0004A229
   391 0001:0004A235   392 0001:0004A241   393 0001:0004A24D   394 0001:0004A259
   398 0001:0004A294   399 0001:0004A2A1   400 0001:0004A2B3   401 0001:0004A2B5
   406 0001:0004A2BC   408 0001:0004A2D5   412 0001:0004A2E4   413 0001:0004A324
   418 0001:0004A348   419 0001:0004A36F   423 0001:0004A37D   425 0001:0004A392
   426 0001:0004A394   428 0001:0004A399   429 0001:0004A3AE   431 0001:0004A3B5
   435 0001:0004A3C3   436 0001:0004A3DE   438 0001:0004A3E5   442 0001:0004A3F3
   444 0001:0004A40D   447 0001:0004A431   449 0001:0004A45F   451 0001:0004A463
   454 0001:0004A471   456 0001:0004A48E   458 0001:0004A492   459 0001:0004A494

Line numbers for cefclient(cefclient.dpr) segment .itext

   488 0002:000007BC   489 0002:000007E5   490 0002:000007F4   492 0002:000007F9
   493 0002:00000809   495 0002:00000819   496 0002:00000830   498 0002:00000844
   501 0002:00000878   502 0002:00000886   503 0002:0000088C   504 0002:00000893
   505 0002:00000898   506 0002:0000089D   507 0002:000008A5   508 0002:000008B4
   509 0002:000008C3   510 0002:000008C8   511 0002:000008CD   513 0002:000008D5
   515 0002:000008DB   528 0002:00000914   529 0002:00000921   532 0002:0000092C
   541 0002:0000093E   543 0002:00000950

Bound resource files

g:\program files\embarcadero\rad studio\7.0\lib\character.res
ceffilescheme.res
cefclient.drf


Program entry point at 0002:000007BC
